:020000040802F0
:100000003ADE002405030208A9020208A902020838
:10001000A9020208A9020208A9020208A90202080C
:10002000A9020208A9020208A9020208A9020208FC
:10003000A9020208A9020208A9020208A9020208EC
:10004000A9020208A9020208A9020208A9020208DC
:10029000A9020208A90202080000000000000000F4
:1002A000FFECC2925D7D05C5EFF305801EF0040FE3
:1002B00002D0EFF309818D466A4602F16802EFF33E
:1002C00011831EF0100F0CBF2DED108A90B02DE998
:1002D000FC4F6946DFF828D000F090FBB0E8FC4FF7
:1002E0001EF0100F0CBFB0EC108A40301EF0040F4F
:1002F0000CBF80F3088880F3098883F31188704766
:10030000C010002408B500F02DFC1D4B1D48DA1C60
:10031000C11E121A22F00302994288BF0022002156
:1003200001F0C9F8184B1948DA1CC11E121A22F044
:100330000302994288BF0022154900F051FF00F0E6
:1003400019F900F073FB00F087F9BFF34F8FBFF38B
:100350006F8F4FF0E023D3F8902F22F00102C3F803
:10036000902F0522C3F8942FBFF34F8FBFF36F8FE9
:1003700032F132FA00F08EFA00F0A0FA01F096F9AC
:100380004CDB0024C00D0024780D00240000002464
:10039000A4121C08704A82B0D2F8003423F48023DF
:1003A00043F48033C2F800346C4B0193019B002B63
:1003B00003DDD2F800349B0304D5019B002B04DC41
:1003C00002B07047019B013BEFE7634BD3F8182461
:1003D00022F4706222F00F0242F00802C3F81824DF
:1003E000D3F81C2422F4E06242F04002C3F81C243B
:1003F000D3F81C2422F4E06242F48062C3F81C2487
:10040000D3F8182422F0700242F04002C3F81824F6
:10041000D3F8202422F0700242F04002C3F82024D6
:10042000D3F8102422F47C5242F40062C3F8102462
:100430004B4AC3F828244B4AC3F830244A4AC3F82D
:10044000382402F50032C3F84024484AC3F82C246B
:10045000D3F8002442F0A852C3F80024D3F80024B3
:100460009001FBD5D3F800241101FBD53A4BD3F80A
:1004700000249200FBD5D3F80C2842F00602C3F802
:100480000C28D3F8182842F44042C3F81828D3F8AF
:1004900018289004FBD5304BD3F804289104FBD5E1
:1004A000D3F8F4244FF0B04142F00202C3F8F42430
:1004B000D1F82C2442F00102C1F82C24D3F81828DA
:1004C0009204FBD52A4A22211160D3F8102422F08D
:1004D000070242F00302C3F810241F4BD3F8102484
:1004E00002F03802182AF9D1D3F8542422F44052E9
:1004F00042F40052C3F85424D3F8582422F4407232
:1005000042F40072C3F85824D3F8502422F4E04295
:1005100042F48052C3F85024D3F8502422F4E0224D
:1005200042F48032C3F85024D3F8582422F0E04239
:1005300042F08052C3F85824D3F8542422F44012D5
:1005400042F40012C3F85424D3F8502422F040524D
:10055000C3F8502434E700BF00400258F82F910040
:1005600012202000770203072F0201018808BF0034
:100570000020005210B52F4C00200122D4F8003486
:1005800043F00103C4F800342B4BC3F80821C4F82E
:1005900010042A4BD4F80024134043F01003C4F88D
:1005A0000034274BC4F82C34D4F8003423F48023CF
:1005B000C4F80034C4F8600400F0CEF8FFF7EAFE97
:1005C000D4F8D83443F0006343F02303C4F8D8349C
:1005D000D4F8DC34C4F8DC34D4F8D43443F48033B5
:1005E000C4F8D434D4F8E03443F0895343F09F0383
:1005F000C4F8E034D4F8E83443F4C10343F480434E
:10060000C4F8E834D4F8EC34C4F8EC34D4F8F0345A
:1006100043F4405343F03003C4F8F034D4F8E434E6
:10062000C4F8E434D4F8F43443F00203C4F8F434E6
:1006300010BD00BF004002580080005167EFFEEA85
:100640000000FF01034BD3F81C241206FBD5C3F8AE
:10065000280470470010014020220021184808B5E6
:1006600000F0C4F8174800F0A7FA174800F0A4FA01
:10067000164BD3F8042422F4FE4222F07002120436
:10068000120CC3F80424D3F8002422F04F4222F4C1
:100690007F0222F47F4222F0FC02C3F800240C4ABD
:1006A000D3F808140A40C3F8082440F62302C3F81C
:1006B0000C24D3F8002442F00D02C3F8002408BD36
:1006C000F0440258267C0900277C090000100140F4
:1006D0000000F1FF30B4EFF3118400238022EFF328
:1006E000108372B682F3118883F31088BFF34F8FA3
:1006F000174B1849D3F800280B8802F4807578B19D
:1007000001339BB20B8075B1CBB10023BFF34F8F88
:10071000E4B284F31188C3B1042030BC00F07CB88B
:100720005BB1013BEDE70B88002BEED0084B42F4A8
:100730008072C3F800280123E8E7002DE5D022F4F9
:100740008072034BC3F80028DFE730BC704700BF5E
:1007500000400258C0100024EFF3118200238021D2
:10076000EFF3108372B681F3118883F31088074981
:10077000D1F8003823F48073C1F800380021044B0D
:100780001980D3B283F31188FFF7A4BF0040025849
:10079000C010002470B50446EFF3118500238022B9
:1007A000EFF3108372B682F3118883F310880E4A38
:1007B000D2F8083860B143F001034FF47A740A4E5E
:1007C000C2F80838013C06D2EDB285F3118870BD3D
:1007D00023F00103F3E7D6F80838DB07F4D401204F
:1007E00000F01AF8EEE700BF0040025830B5EFF312
:1007F000118400238025EFF3108372B685F31188EE
:1008000083F31088036823EA0101E3B20A4302601C
:1008100083F3118830BDFFEC82B000221C49B0F593
:100820007A7F0BD8002242F22A51642811D8002284
:100830000A2818D8002208BB02B070470192019B19
:100840008B4202DDA0F57A70E9E7019B0133019349
:10085000F5E70192019B8B4201DD6438E5E7019BDE
:1008600001330193F6E70192019BB3F56E7F01DB43
:100870000A38DDE7019B01330193F5E70192019B03
:100880005E2B01DD0138D6E7019B01330193F6E7CA
:10089000AD730100BFF34F8FBFF36F8F4FF0E023B5
:1008A0000022C3F8502FD3F8142D42F40032C3F8BD
:1008B000142DBFF34F8FBFF36F8F70474FF0E022BF
:1008C000F0B5D2F8803D03F00704C3F34E31C3F313
:1008D000C9030434B3FA83F505F01F05BFF34F8F46
:1008E000184601FA04F700FA05F6013846EA070649
:1008F000C2F8606FF7D20139F2D2BFF34F8FD2F84E
:10090000143D43F48033C2F8143DBFF34F8FBFF35F
:100910006F8FF0BD10B54FF0E0240123D4F8802D87
:1009200002F0070204329340BFF34F8F5A1E024277
:1009300004D05A421040C4F8700F18444FF0E0241D
:10094000C2188A420AD9884203D24FF0E023C3F882
:10095000700FBFF34F8FBFF36F8F10BDC4F85C0FE4
:100960001046EDE7F0B54FF0E026D6F8803D03F0F5
:100970000700C3F34E32C3F3C9030430B3FA83F460
:1009800004F01F04BFF34F8F194602FA00F701FA73
:1009900004F5013945EA0705C6F86C5FF7D2013A5C
:1009A000F2D2BFF34F8FBFF36F8FF0BDF0B44FF0B3
:1009B000E0260F1A0124D6F8802D02F00705C2F3B5
:1009C0004E33C2F3C90204350133AB40AC4002FBE5
:1009D00003339F4202D3F0BCFFF7C4BF6342184009
:1009E000BFF34F8FC6F8680F20448142FAD8BFF397
:1009F0004F8FBFF36F8FF0BC7047FFEC70B50A4D9F
:100A000006460C462B680BB91C462960304600F0A0
:100A1000B5FA2968304600F029FF14B900232C6884
:100A20002B60204670BD00BFC4100024EFF3148378
:100A300043F0040383F314884FF0E023D3F8342FFA
:100A400022F04042C3F8342FD3F8882D42F47002CC
:100A5000C3F8882D7047FFEC024B1878421C1A70BF
:100A6000704700BFC2100024202810B50CD90623FF
:100A70000121202B0AD001FA03F25C1C824201D32F
:100A8000D8B210BD2346F4E70520FAE71846F8E788
:100A9000072A1CD901231F2A03FA02F3A2F1030239
:100AA00003F1FF3300EA030094BFDB106FF06043F3
:100AB000014420EA0300194421EA030120FA02F369
:100AC000D140044A505C044AD35C1843704700206C
:100AD000704700BF7D3616087436160840B10029ED
:100AE000C2F1000214BF0320012002F004021043EF
:100AF0004FF0E023C3F8940D70472DE9F04780468E
:100B00004FF0FF3A1446FFF7A7FF08EB010628F065
:100B10001F0705468946F01BFFF7A6FF0AFA00FAF1
:100B20000AEA070A4FF0E027A6EB0A00FFF79CFF4E
:100B3000C7F8985D45EA0A0506460246494645F06B
:100B400010054046013EC7F89C5DFFF7A1FF00027B
:100B500044EA460480B2044344F00104C7F8A04DBF
:100B6000BDE8F0874FF0E0230022D3F8900D114646
:100B7000C0F30720904202DCC3F8941D7047C3F80D
:100B8000982D0132C3F8A01DC3F89C1DF2E7FFECBD
:100B900003060BD4C0F30312064B53F822202AB1EC
:100BA00000F00F00012311B18340936170471030B2
:100BB000FAE700BF883616082DE9F04710F08006E6
:100BC0000446C0F3031840F0D9806E4B53F8285008
:100BD000002D00F0D38000F4402300F00F07B3F5A0
:100BE000002F00F0B780B3F5402F00F0B580B3F5CB
:100BF000802F40F0B380C0F30021FFF7C9FF01212F
:100C0000EFF3118200238020EFF3108372B680F39C
:100C1000118883F31088022940F0A28014F4704FE9
:100C2000C4F3033E14D023074FF00F094BBFA7F1C5
:100C300008033B46242020209B0050F805C009FAF9
:100C400003F90EFA03F32CEA090C43EA0C034351AF
:100C50004FEA470C0323D5F80090032903FA0CF35D
:100C600029EA03096FEA030001FA0CF343EA0903D6
:100C70002B6078D004F44033B3F5803F75D0A3F5F2
:100C80000039D9F1000343EB09035B00D5F80C9060
:100C900003FA0CF300EA090943EA0903EB60BEF129
:100CA000000F13D123074FF00F0A4BBFA7F1080322
:100CB0003B464FF0240E4FF0200E9B005EF805904F
:100CC0000AFA03F329EA03034EF8053001F1FF3E67
:100CD000BEF1010F0DD804F44066B6F5006F46D0A2
:100CE000B6F5406F45D0A6F58069D9F1000646EB10
:100CF0000906AB6806FA0CF6BEF1010F00EA030024
:100D000046EA00064FF00100AE6000FA07F06B689B
:100D100031D8A6052FD5034301296B6014D0E30514
:100D200012D504F00C04BF000F2104F1B04407F009
:100D30000C07D4F80834B94008FA07F823EA01038D
:100D400048EA0303C4F80834D2B282F311880020C1
:100D5000BDE8F087022153E7032151E731464FE711
:100D60004FF0000E74E7002390E701238EE7022680
:100D7000BFE70326BDE723EA0003CDE76FF01500C8
:100D8000E6E700BF88361608C0B2FFF715BFFFECD4
:100D90000206034610D4C0F30311084A52F821009A
:100DA00058B1012203F00F03016902FA03F30B4269
:100DB00014BF104600207047002070478836160880
:100DC0000F2810B52DDDA0F110041F2C08DC03F155
:100DD000604303F561430B600123A340136009E006
:100DE0003F2C09DC1D4C30381C440C60012303FAF5
:100DF00000F01060002010BD5F2C04DC184C50384F
:100E00001C440C60F2E77F2C04DC164C70381C4448
:100E10000C60EBE7952C1EDC134C90381C440C60E6
:100E2000E4E7124B04380B600B2814D8DFE800F01D
:100E300006090C13131313131313130F4FF48033FA
:100E4000CCE74FF40033C9E74FF48023C6E7084BE3
:100E50000B600123C2E74FF0FF30CCE704E100E074
:100E600008E100E00CE100E010E100E024ED00E02A
:100E700010E000E013B5802301AA69460446FFF79D
:100E80009FFF20B90F2CDDE9003102DD196002B0AF
:100E900010BD1A6822EA01021A60F8E713B50023B0
:100EA00001AA69460446FFF78BFF20B90F2CDDE944
:100EB000003102DD196002B010BD1A680A431A60E1
:100EC000F9E7FFEC4FF0E02325494FF0FF3010B574
:100ED0005B6803F00F035A1C03F1382361339B0056
:100EE00041F8040B9942FBD14FF0E0231D49C3F8B0
:100EF000081D4FF08031C3F8181DC3F81C1DC3F83E
:100F0000201D5301184A03F1604303F5644342F87E
:100F1000041B9342FBD10024144B15490B2022469D
:100F20001C6000F07BFC22461249032000F076FC96
:100F30004FF0E02210490420D2F81C3D23F07F43FB
:100F400043F0E043C2F81C3D224600F067FC042059
:100F5000FFF7A4FFF02383F3118862B610BD00BF32
:100F600080E100E00000020800E400E0C41000247A
:100F700085110208810F0208851002087047FFECF6
:100F80002DE9FF414FF0E02305460E461746D3F802
:100F90002C4DD3F8288D63000FD5304A00203049FE
:100FA00000F0E2FA5FFA88F33BB13A463146284650
:100FB00004B0BDE8F04100F065B8284A0020294996
:100FC00000F0D2FA2B46254A00202749009600F06F
:100FD000CBFAEFF31183EFF31082EFF30581EFF318
:100FE0001480D2B2DBB200921C4ACDE901101F4935
:100FF000002000F0B9FA4FF0E0230020D3F8302DA4
:10100000D3F8381DD3F83C3DCDE90042CDE90213B9
:10101000124A4346164900F0A7FA00200F4A154924
:1010200000F0A2FA14F0020013D00C4A002012497A
:1010300000F09AFAEFF3118300238022EFF310837C
:1010400072B682F3118883F31088AD210B4800F04B
:10105000CFF9002CEEDA014A0949E9E7F57A1708D9
:10106000A8361608C4361608DE361608F5361608F1
:10107000303716086D37160885371608BD3716083D
:10108000AB371608F0B54FF0E02585B006460F46A1
:10109000304A00203049D5F8284D00F065FA334633
:1010A0002C4A2E490020009700F05EFAD5F8283D22
:1010B000D5F8342D00202A490092264A00F054FA2F
:1010C000EFF31183EFF31082EFF30581EFF3148058
:1010D000D2B2DBB200921F4ACDE9011021490020B3
:1010E00000F042FA1B4A2049002000F03DFAE507D3
:1010F00004D5184A00201D4900F036FAA00704D58F
:10110000144A00201A4900F02FFA210704D5114A89
:101110000020184900F028FAE20604D50D4A002004
:10112000154900F021FAA30604D50A4A0020134904
:1011300000F01AFAEFF3118300238022EFF31083FB
:1011400072B682F3118883F3108865210C4800F091
:101150004FF900BF037B1708D5371608FC37160870
:1011600016381608F5361608333816085838160893
:101170007B38160897381608BB381608DD3816086D
:1011800010391608CA6E012A08B508D0022A0AD0FA
:101190001AB9D422086F00F023F8002008BD0A6FA6
:1011A000034B1A60F9E70A6F11604A6FF8E700BF56
:1011B000C4100024FFECC2925D7D05C5FFECC29215
:1011C00018DF88DFCD06CD767CD30CD3D982D91237
:1011D0002C00050A0F14191E232800BFAFF300804E
:1011E00000B501B400F004F801BC00BDAFF300800D
:1011F00000B5042A60DB00F0030E61F3830E7A4B26
:10120000D3E80EF0AFF30080AFF30080AFF30080BF
:1012100011F8013B00F8013BA2F1010211F8013B7A
:1012200000F8013BA2F1010211F8013B00F8013B7B
:10123000A2F101022DE9F01F282A07DBB1E8F81F0F
:10124000A0E8F81FA2F12802282AF7DADFF89CE1CB
:101250004FEA920BDEE80BF051F8043B40F8043BF8
:1012600026E0B1E81800A0E8180021E0B1E8380055
:10127000A0E838001CE0B1E87800A0E8780017E0AA
:10128000B1E8F800A0E8F80012E0B1E8F801A0E841
:10129000F8010DE0B1E8F803A0E8F80308E0B1E8D0
:1012A000F807A0E8F80703E0B1E8F80FA0E8F80FA6
:1012B000BDE8F01F02F00302002A08BF00BD11F8CC
:1012C000013B00F8013B013A08BF00BD11F8013BAA
:1012D00000F8013B013A08BF00BD11F8013B00F8DE
:1012E000013B00BDAFF30080AFF30080AFF300809F
:1012F00011F8013B00F8013BA2F1010211F8013B9A
:1013000000F8013BA2F1010211F8013B00F8013B9A
:10131000A2F10102282A35DB2DE9F01FB1E8F81F00
:1013200020F8023B4FEA134364F31F434FEA14448F
:1013300065F31F444FEA154566F31F454FEA16460D
:1013400067F31F464FEA174768F31F474FEA1848ED
:1013500069F31F484FEA19496AF31F494FEA1A4ACD
:101360006BF31F4A4FEA1B4B6CF31F4BA0E8F80FBF
:101370004FEA1C4C20F802CBA2F12802282ACDDA31
:10138000BDE8F01F042A97DB51F8043B20F8023B2C
:101390004FEA134320F8023BA2F10402BAE711F826
:1013A000013B00F8013BA2F1010211F8013B00F8FA
:1013B000013BA2F1010211F8013B00F8013BA2F14F
:1013C0000102042AFFF678AF51F8043B00F8013B14
:1013D0004FEA132320F8023B4FEA134300F8013B86
:1013E000A2F10402EDE70000C0110208D0110208CA
:1013F00008B507F007FE012000F004F8002008B54A
:1014000000F0DAF8044608B500F032F8204601F0A2
:1014100043FA2DE9F0410E468046174600F0B1F838
:10142000054616B300F0ADF800F0AEFB002809DB6E
:10143000EB6B002B0FDD4FF0FF3400F0A2F800F053
:10144000FFFB05E000F0AEF80468002CF0DD64421C
:101450002046BDE8F0810C2404FB03540133C4E9A9
:101460001086A7640024EB63E7E74FF0FF34EFE753
:10147000F8B5064600F085F80C22C46B0027651EFF
:1014800002FB0404002D00DAF8BDD4E90D23E16B62
:10149000C4E90E7713B1012A03D19847013D0C3CF2
:1014A000F0E7022A02D130469847F7E7032AF5D140
:1014B00008469847F2E7002A44D010F0010F03468F
:1014C0003AD0013A03F8011B012A39D9F0B541EAB3
:1014D00001259E07ADB22CD0023A23F8025B032A05
:1014E00019D95C0705EB054616BF141F144643F8CF
:1014F000046BB446224604EB030E072A13D8E20815
:101500006FF0070707FB02423C40032A234484BFD5
:10151000043A43F8046B012A02D9023A23F8025B29
:1015200002B11970F0BDAEEB0207083AC7E900C678
:10153000E3E7032AD5D8F0E7012AC7D1197070472D
:10154000002AFBD17047FFEC064B07B51B7803411F
:10155000DB0703D5019201AA00F053F803B05DF850
:1015600004FB00BF040000240EB403B503AA52F824
:10157000041B0192FFF7E8FF02B05DF804EB03B033
:10158000704708B500F002F8006808BD1FB50020DC
:1015900001A900F079FA0028ACBF0298002005B03C
:1015A0005DF804FB08B5FFF7F1FF08B1143008BD82
:1015B0000048FCE7C8100024044608B500F003F812
:1015C000204600F083F92DE9F041FFF7DAFF0546E8
:1015D0000024FFF7DBFF4FF001082F7B061D08FA00
:1015E00004F31F4208D056F8240028B105F1100377
:1015F00053F8243003B198470134042CEFD1BDE8EF
:10160000F08130B585B00C461546684600F018F8F4
:101610002A68214668460AF085F805B030BD0D29D4
:1016200038B504460D4607D0284600F015F8031ECD
:1016300003DBE3680133E36038BD0433F4D0FBE738
:10164000034B0360034B83600023C360704700BFFC
:101650001F16020845CB020838B50C4B04460C4D4A
:101660001B681BB1286858B9204638BD00F000FA45
:101670000028F7D128680028F6D003681B6801E02D
:1016800003685B6821469847EEE700BFC41000245A
:101690000800002410B514460846114607F054FE11
:1016A000204610BD084607F0DFB9FFEC3F4C012390
:1016B0003F4DA82204F18C062B7083B500212046F3
:1016C000FFF7F9FE032318223A49237730463A4BB5
:1016D0003A4FC4E905330623A3860BF072FB384961
:1016E00020463E6009F0C9FE364B374E1C6002238F
:1016F0002B7000F0B2FA01A9684606F0EFFDDDE9B3
:10170000000109F093FA042333603368012B49DDAB
:101710003068800009F0B8FA2C4B18603368046018
:10172000224894F8341001F065FAA3681F489B6AB8
:101730009F6007F057FF1D4801F0BCF81B4801F0FF
:1017400087FAA36805221A720022214B1A6003232C
:101750002B7000F04FF90DF04DFE1E4B0BB101F058
:10176000BDFA1D4B0BB102F0F7F91C4B0BB101F0A8
:10177000C9FC02F003FA07F0CDFD0CF015F90423C3
:101780000A482B7031F188FC084801F091FA0523D2
:101790002B7000F025F806232B7000F03BF907F0C2
:1017A0001FFFFCE733685B00AEE700BFD4100024E6
:1017B0007C110024247B1708AD160208CC100024ED
:1017C000B8110024B41100248011002484110024D5
:1017D00088110024DD2C0208593B0208053102085B
:1017E00013B5002401220949094801F06FF901F0FD
:1017F0000DF901F017F9074B40F67A426421009485
:10180000054800F013FE204602B010BD7ADA160833
:101810003A501608E53B020827391608A52870B586
:1018200005460C461AD8EFF3118600238021EFF30A
:10183000108372B681F3118883F310881CB9FFF707
:1018400019FB2246074C084BF6B243F8354003EB30
:10185000C5035A6086F31188002070BD6FF0150033
:10186000FBE700BFA918020844140024A52808B506
:101870000CD8094A52F830305BB102EBC002526812
:101880009847064B1A68064B1A6008BD0022054BA4
:10189000F6E71A46FBE700BF44140024B811002401
:1018A000B4110024A918020808B5EFF3118300232E
:1018B0008022EFF3108372B682F3118883F31088CD
:1018C00036210148FFF794FD303916080E4B37B525
:1018D00004461D684FF0FF33002201A90320019345
:1018E00000F030FB00F0BEFF214600F033F8044664
:1018F00010B10120FFF786FD02460146284600F0A0
:1019000073FF204607F0E6FCB811002438B50C46FA
:101910008D680023016A39B18A6895420A6810D13E
:10192000A3B98AB9C0E9083304F1140000F0CEF875
:1019300004F10C0000F0CAF82046BDE8384009F078
:101940008BB90B461146E6E70262EDE702B9436246
:101950001A60E9E7F7B504460F4600F07CFF00F196
:1019600018060546304600F007F92146284600F0E3
:1019700038F8044630B9304601F0CFF94FF0FF3067
:1019800003B0F0BDC761012300F10C0701A9837109
:10199000384609F0D1FD014630B16379E3B1214603
:1019A0002846FFF7B3FF17E0019A002AF5DA14344E
:1019B0000132204609F0A5FD384601F0AEF918B90C
:1019C00001A9384609F0B8FD019B002B01DA002877
:1019D000F2D0204600F0D0F8304601F09EF9002009
:1019E000CEE7006A10B183688B4200D1704700686F
:1019F000F8E7FFEC054B1B682BB1054A126812B9DA
:101A0000DA8E0132DA860020704700BFB811002458
:101A1000C4100024134B10B51A68C2B1124B1B68D6
:101A2000ABB9EFF311848021EFF3108372B681F329
:101A3000118883F31088B2F93630002B09DC0023BB
:101A4000D3860A4B1B6853B9E4B284F31188002093
:101A500010BD013B1BB2D386002BF5D1EFE707F099
:101A60007FFCF1E7B8110024C4100024AC1100245D
:101A7000044B1B6823B11868B0FA80F04009704726
:101A800001207047B811002438B50F4B0C461D6873
:101A900070B101F08DF9A0B1AB8E03F00303022BFE
:101AA00007D0AA6883689A4203D06FF00C0007E061
:101AB0002846C36C2360036D6360436D0020A36000
:101AC00038BD6FF00100FBE7B811002408B540B144
:101AD00003881B0401D40123038000F0A3F9002034
:101AE00008BD6FF01500FBE710B5FFF7EFFF041E10
:101AF00005DA6442FFF756FD04604FF0FF342046DC
:101B000010BDFFEC1B4B70B504461D68EFF311864A
:101B100000238022EFF3108372B682F3118883F3DF
:101B2000108820B303881BB2002B038803F1FF3316
:101B30001BB2038008DD002400F0A2F9AC65F6B208
:101B400086F31188204670BDA865FFF753FF204635
:101B500000F09EF90023052128462B8707F05CFB47
:101B6000B5F9384004B16442FFF754FFE7E76FF07E
:101B70001504E4E7B811002410B504462046FFF729
:101B8000C1FF031DFAD010BD10B5FFF7BBFF041E47
:101B900006DA6442FFF706FD04604FF0FF3010BD27
:101BA0000020FCE770B50546002844D0EFF311860D
:101BB00000238022EFF3108372B682F3118883F33F
:101BC0001088038847F6FF721BB2934205D1F6B224
:101BD00086F311886FF08A0070BD00F063F92B88DE
:101BE00001331BB22B80FFF705FF2B881BB2002BA4
:101BF0001FDC124B1C687CB1A36DAB4217D1294688
:101C0000204600F015F904F13C0000F061FE0023CD
:101C10002046A36507F042FC2946204600F066F9FD
:101C2000F6B2FFF7F7FE86F311880020D4E72468A8
:101C3000E1E70024F0E76FF01500CDE7A4110024E0
:101C400010B5FFF7AFFF041E05DA6442FFF7AAFCE8
:101C500004604FF0FF34204610BD00F0CFB8FFEC19
:101C6000CB6803F130021B6B1BB18B4212D14B6866
:101C700013600023021DC1E90133CB600B8243686E
:101C80001BB18B4209D10B681360054B1A681960B0
:101C90000A6070471A1D5B68E6E71A461B68EFE7A3
:101CA000C011002408B503460846B3F91020002AE5
:101CB00004DC1946FFF7D4FF012008BD0020FCE733
:101CC00008B50B4601461846FFF7CAFF002008BDBD
:101CD00010B5C068117C90F82E3099420ED9047C62
:101CE000A1420DD9A34206D2437F0F2B9FBFC1183B
:101CF00001338C774377117C01F0AEF8002010BDE2
:101D0000437F0F2B9FBFC218013391774377F5E7CD
:101D10000346084670B51546B3F91020DC68002A62
:101D200002DC1946FFF79CFF227C94F82E108A42B1
:101D300004D0637F23B9204601F0D6F8002070BD9F
:101D4000297C8A4218D804F11E0600200122251899
:101D50009342A97F09DC013B20461EBFE218927F17
:101D6000AA77637701F078F8E8E716F8015F8D420B
:101D700088BF10460132EAE704F11D00002210F886
:101D8000015F8D4207D1013B1FBFE1181219897F06
:101D900091776377D2E701329342F0DCCEE7FFEC34
:101DA000054B10B51B68C4689C4203D1FFF7B0FF18
:101DB000012010BD0020FCE7B8110024064B10B430
:101DC0001B68C4689C4203D05DF8044BFFF7A0BFBA
:101DD00000205DF8044B7047B8110024F8B50446A4
:101DE0000D4616464068002300B103B1F8BD0768F0
:101DF00032462146A84703463846F5E7074A002100
:101E0000074B1A6002F11403013143F8143C1433F8
:101E10001F29F9D10023C2F86C327047C411002485
:101E2000C011002400220149FFF7D8BFC11C0208DD
:101E3000036830B5DBB18B78DB0718D44A681346EA
:101E4000B3B90E4C236893B11D681A6000224B6031
:101E50001A822560C3E90210026B5A600363B3F96A
:101E6000102047F6FF718A421CBF01321A8230BD32
:101E7000DC68A042F3D01B68E2E700BFC011002479
:101E8000024B01461868FFF7D3BF00BFB81100240A
:101E9000024B03491A68FFF7A1BF00BFB811002425
:101EA000D11C02080C4B002210B511461C68436877
:101EB00033B9012A02BF0B8A03F1FF330B8205E01D
:101EC000D968A14203D11A8A013A1A8210BD194673
:101ED00001321B68ECE700BFB81100240246084637
:101EE0000149FFF77BBF00BF111D020838B504464A
:101EF0000D4690B10A4B1B681BB1BDE83840FFF797
:101F0000EDBF024607492846FFF768FF224606490B
:101F10002846BDE83840FFF761BF02460349F7E7AE
:101F2000C4100024BD1D0208A11D0208A51C020842
:101F300010B50446216B01B910BD8868FFF790FE0B
:101F4000F8E7FFECF8B51746194B06460C461D6836
:101F5000FFF750FD0FB1EB6D3B60D4B1EFF3118390
:101F600000228021EFF3108272B681F3118882F390
:101F70001088022E11D0032E14D0012E14D1EA6D38
:101F800021680A430024EA65DBB283F3118800F07C
:101F900011F8FFF73FFD2046F8BD2168EA6D22EAFF
:101FA0000102EFE72268EDE76FF01504ECE700BFF0
:101FB000B8110024174B37B51D68FFF71BFDEC6DFA
:101FC000284601F0FDF8E4430440019424B9FFF7EA
:101FD00021FD204603B030BD01A800F06FF8431C7E
:101FE000044610D0014601A809F0C9FA2146284646
:101FF00000F012F8044630B1011D284600F06EF8DA
:10200000204600F02DF8019B002BE5D1FFF702FDE3
:102010000120DFE7B811002438B58368EFF311859C
:1020200000228020EFF3108272B680F3118882F3D1
:10203000108800205C6B3CB122798A4209D103F1FF
:10204000340148B109F0FEF9EDB285F3118820465C
:1020500038BD20462468EEE7084609F0E9F9F3E7C1
:1020600010B5037B83B9EFF311848022EFF3108363
:1020700072B682F3118883F310880E4909F0A4F92F
:10208000E4B284F3118810BD022B0CD1EFF311845C
:1020900000238022EFF3108372B682F3118883F35A
:1020A00010880549EAE7012BEDD1BDE8104008F0A2
:1020B000D3BD00BF7C1900247419002438B505462F
:1020C00001242146284609F06AFA20B90134202C5F
:1020D000F7D14FF0FF34204638BDFFEC2DE9F04139
:1020E0000D460978044629B35C3009F058FA0128F6
:1020F00007467ED1EFF3118600238022EFF3108391
:1021000072B682F3118883F31088237FF6B2062B10
:1021100012D1297804F1600009F041FA60B12B680E
:10212000204663676B68A3670023236607F0B6F950
:1021300086F311880026C0E086F31188A468297808
:10214000EFF3118200238020EFF3108372B680F347
:10215000118883F31088636B13B11879884208D112
:10216000D2B282F3118833B12A685A606A689A60E1
:10217000E0E71B68F0E7564B1B68FBB1554809F0D8
:1021800057F920B9544809F053F90028D2D02B68E8
:1021900043606B688360EFF3118500238022EFF3C7
:1021A000108372B682F3118883F3108804F134012E
:1021B000EDB209F009F985F31188BBE7EFF3118659
:1021C00000238022EFF3108372B682F3118883F329
:1021D00010884048F6B209F02BF986F311880028E0
:1021E000D5D1102008F040FD0028A3D001230373AF
:1021F000CDE7FFF7FFFB2978A06800F0FDFF06465A
:1022000058B343684BB301F009F8002858D07368FD
:102210004360B2688260F3689B0604D42978012386
:102220008B40134383602B68C3606B680361EFF3DB
:10223000118600238022EFF3108372B682F3118897
:1022400083F3108804F16401F6B209F0BDF8234964
:10225000204607F00DFA86F311880026FFF7DAFB17
:10226000EFF3118800238022EFF3108372B682F31C
:10227000118883F31088237F062B08D12B68204612
:1022800063676B68A3670023236607F007F95FFAAB
:1022900088F888F31188002F15D1237F052B03D1EF
:1022A0000421204600F0E5FE237F072B05D12B7883
:1022B000082B02D1204600F021FE3046BDE8F08117
:1022C0006FF00B06CAE7F8DA6FF01506F5E700BF06
:1022D000C41000247C19002474190024FB22020875
:1022E00010B50C4600F064FD20B12146BDE8104059
:1022F000FFF7F4BE6FF0020010BD2DE9F04F87B07C
:102300000446FFF74FF903684FF0800A04F16C09A7
:102310000193B4F93830029304F164030593EFF3A9
:102320001183EFF3108772B68AF3118887F3108850
:10233000B4F8348018F400725FFA83F804920AD07B
:1023400088F31188FFF72EF9019B0360029B238716
:1023500007B0BDE8F08F059809F06AF80646002836
:10236000EED0A28E494642F40072A28609F02CF803
:10237000D4F85CB0B5684BEA0505E56588F31188CB
:10238000736806F10C01049A307B9847EFF31188CB
:10239000039BEFF3108372B68AF3118883F31088DE
:1023A00003934946A38E30465FFA88F823F40073FE
:1023B000A386E36D5D4083EA0B031D4085EA0B05B0
:1023C000E56509F01FF888F31188FFF7F3FD304643
:1023D00000F050FFA3E72DE9FF410546A8208846FD
:1023E00016461F4608F050FC0446E0B10023A0F852
:1023F00034802946324603930C9B02930B9B019336
:102400000A9B00933B4600F045F8051E06DA20467D
:1024100008F022FC284604B0BDE8F0812046E568BB
:1024200000F09CF9F6E76FF00B05F3E71FB5069C8B
:1024300000920A46CDE9013400231946FFF7CBFF8D
:1024400004B010BD13B5049C0094FFF7EFFF041E09
:1024500005DA6442FFF7A6F804604FF0FF34204627
:1024600002B010BD1FB5079C0294069CCDE9003454
:1024700013460A460221FFF7AEFF04B010BD13B5A4
:10248000049CCDE9003413460022FFF7EBFF02B0B5
:1024900010BDFFEC2DE9F34790F8346088460546FF
:1024A000914631461F46DDF828A000F0A3FB041E2C
:1024B00040DB0D9906F00306A86800F0BFFA041E81
:1024C00011DB284600F0F6FB041E0CDB87B15246F8
:1024D0003946284607F00CF8041E05DB284600F0B4
:1024E000E9F9041E13DA57B1284600F0B7FB21E0E2
:1024F00032465146284606F0C7FE041EEEDA2B6D22
:10250000002BF1D03146284606F050FFECE70B9B3C
:1025100049460A4A2846009600F0A4F8041EE2DB69
:102520000C9A4146284600F0ADF8041EDBDB284635
:1025300000F08EFB204602B0BDE8F0879527020828
:102540002DE9F74F04460E4601929946EFF31187A5
:1025500000238022EFF3108372B682F3118883F395
:102560001088DFF8F8A0DFF8F880DAF800500020D3
:10257000D8F800300135374A116888420DDB106801
:10258000C00008F081FB334A0546002844D1FFB261
:1025900087F311886FF00B0038E0012D1168B8BF88
:1025A00001250139294053F821B0BBF1000F30D18A
:1025B00043F82140FFB2E560CAF8005087F3118864
:1025C000019BF6B29DF830205946032026746674AC
:1025D00084F82E60C4E90539A38E62F3010304F187
:1025E0005C0223F06003A386FFF7ACFC204684F86E
:1025F0001CB006F0F7FFFFF7FDF91749204608F079
:102600003CFF04232377FFF705FA584603B0BDE8E3
:10261000F08F01350130AFE711684FF0000C0D4B22
:10262000490011601A68D8F8000002EBD272BCEBC6
:10263000620F04DB08F010FBC8F8005095E750F873
:102640002C000CF1010C1A68C168013A0A4045F8E7
:102650002200E7E7801100248C1100248811002457
:102660008411002410B49DF8044001945DF8044BDB
:10267000FFF766BF13B501240094FFF761FF02B0B6
:1026800010BDFFEC344B2DE9F74F002914BF8846ED
:102690009846074600241546414618228C300AF019
:1026A000ACFB404687F8A4400AF09FFB461C4DBB9C
:1026B0002C460234384606EB840106F0CBFE064673
:1026C0004FEA8409002844D000EB090AA9F108095F
:1026D000B346043DC0F800A040460AF086FB04461D
:1026E000B1444146013450460AF063FB5444CB45A3
:1026F0001BD100204AF8040CBB689B6A9E6003B0A3
:10270000BDE8F08F40F2011955F824000028D0D020
:1027100001360AF06AFBFB6C06449E4216D2013475
:102720004C45F1D16FF00600E9E74BF8044F55F83E
:10273000041F084601910AF058FB80460199204683
:1027400008F101080AF035FB4444D0E76FF05A0065
:10275000D5E76FF00B00D2E7707B170838B5044659
:10276000EFF3118500238022EFF3108372B682F31A
:10277000118883F31088037F042B01D030F1AEFC65
:102780002046EDB230F188FC204606F087FE85F346
:10279000118838BD38B5134B1C68A38E03F00303B2
:1027A000022B02D0204600F04DFEA368012040F22B
:1027B00001119B6A9A6852F820304BB9A38EA56923
:1027C00003F00303022B08D11146A847FEF71AFEB7
:1027D00001308842EFD10120F8E70146284608F091
:1027E00085FEF8E7B811002470B5838E0E460446C6
:1027F000190517D43AB9806828B1437A012B02D160
:10280000543009F0EDFE204600F03AF8A56855B9BD
:10281000204600F023FA204600F05AFDA38E43F430
:102820000063A38670BDA38E03F00303012B03D0C6
:102830006B690BB136021E606B7A012BE8D1002365
:1028400005F10C066B61EB72AB891B04E0D53046D9
:10285000FFF7A8F9F8E708B500F0AAFA00B1806818
:1028600008BDFFEC054B186830B1037F032B01D185
:10287000C06870476FF00200704700BFB8110024B5
:1028800010B5044600F06DFA204600F055F82046D9
:10289000BDE8104000F0CCBB0446002208B5E4B20D
:1028A000034B21461868FFF79FFF204606F012FDF4
:1028B000B811002410B51821044606F0CBFD20B154
:1028C000A3689B6A0360002010BD6FF00B00FBE75C
:1028D00038B50446EFF3118500238022EFF310830F
:1028E00072B682F3118883F31088F0B14368E3B1C4
:1028F000104B00201B68DBB1A3420FD123681BB132
:102900009A68A1680A449A6058B10A4908F09AFD89
:1029100000206060EDB285F3118838BD18461B6851
:10292000E9E7044808F084FDF2E76FF01500F1E7ED
:102930001B68FFDE9C1900243C30FFF7C9BF2DE95E
:10294000F84300220B46114658680AF028F805465D
:10295000EFF311848026E4B20023EFF3108372B604
:1029600086F3118883F31088002700F10808404699
:10297000FFF702F9284608F05BFD03460028F6D071
:102980000269002AF3D040691F6184F311889047DF
:10299000EFF31184E4B24B46EFF3108372B686F383
:1029A000118883F310889946E1E7FFEC2DE9F041A7
:1029B0008CB004460E4617460DF11008114A20212E
:1029C0001D46404608F071FECDF808804FF0000823
:1029D000CDF80C80FFF70EF802AB20463A463146A0
:1029E0000093094BFFF74BFD041E07DB2C614446A7
:1029F000FFF710F820460CB0BDE8F081FFF70AF8A9
:102A0000F8E700BF483916083F290208034B4FF486
:102A1000A062F9210248FFF7C9BF00BF24000024CB
:102A20004D391608034B4FF4CC6232210248FFF7B0
:102A3000BDBF00BF10000024543916082DE9F04135
:102A4000214B0C4606461D68FEF7D4FF7CBBAB68E5
:102A50001C6C64BBFEF7DEFF2046BDE8F08101354B
:102A600054F82570002FFAD15DB34FEA850808F1BC
:102A7000040008F0F9F80746B0B10023444440F8D8
:102A80002530013D54F8040D0AF0AFF9013008F08B
:102A9000EBF847F8250078B907EB850555F8040FE2
:102AA00038B9384608F0D8F86FF00B040AE0002572
:102AB000D6E708F0D1F8F1E721680AF07AF9013D8C
:102AC000E0D200243764C5E7B81100242DE9F843AB
:102AD0000F4614460546002860D009B10B782BB983
:102AE000B4B12846BDE8F84300F05EB8FEF782FFB7
:102AF0002B4B1B68D3F80880D8F8403073B12946B7
:102B0000404600F0ADFD011E08DB24B9FEF782FF50
:102B10000020BDE8F883404600F0B9FD28460AF0E1
:102B200064F9044638460AF060F92044023008F09F
:102B30009BF8064638B3D8F84090B9F1000F2BD176
:102B4000082008F091F8D8B14C4640F824600023E2
:102B500000EB84042A46134963603B46C8F84000F2
:102B6000304608F07EFDD1E7013459F82430002BBF
:102B7000FAD1A11C4846890008F07EF80028E4D16B
:102B8000304608F069F80C24FEF744FFFEF70AFD12
:102B900004604FF0FF30BCE70024E6E71624F5E7B9
:102BA000B81100245B39160838B5114B04461B6870
:102BB0009D6828B103781BB13D210AF0E5F830B1DA
:102BC000FEF7F0FC162303604FF0FF3038BDFEF730
:102BD00011FF45B12146284600F042FD011E02DBEF
:102BE000284600F054FDFEF715FF0020EEE700BF79
:102BF000B811002470B506464FF47D7008F044F813
:102C0000044610B300F046FC051E04DA204608F026
:102C100023F8284670BD04F14400B4600CF01BFC9E
:102C2000204609F0E7FD0122002104F1180008F018
:102C300068FC0C34002200252046114608F061FC97
:102C40000021204600F038FAE3E76FF00B05E0E7DB
:102C5000D0E902321A6001225A72704738B584688E
:102C6000054634B1637A012B04D9013B637200231A
:102C7000AB6038BD204600F01EFC204600F041FB52
:102C8000204600F056F804F144000CF0E8FB204622
:102C900009F0CFFD204600F0CFFCA37A23B1237AC0
:102CA00043F008032372E2E7204607F0D5FFDEE792
:102CB00000F00BBD084B10B51B680446816898688E
:102CC000443144300CF065FC002804DB2046BDE8AC
:102CD000104000F0FABC10BDB81100240023044AD3
:102CE000044942F833100133A62BFAD1FEF7EAB8B3
:102CF00044140024A918020808B53AB119B9FEF71E
:102D000001FF404208BD00F00BF9FAE711B9FEF7E8
:102D100033FFF6E700F008F9F3E708B528B1FEF74E
:102D200041FF002803DA404208BD1620FCE70020DE
:102D3000FAE738B50446256A2DB904F11800BDE854
:102D40003840FEF7C3BE284650F8143B2362FEF716
:102D5000BDFE05F10C00FEF7B9FE284607F07CFF2A
:102D6000E9E7F8B5802600270446FEF743FEE36F47
:102D70001BB9BDE8F840FEF74DBEEFF311832A46BC
:102D8000EFF3108272B686F3118882F31088E06F39
:102D90001546DBB20268E267076083F31188037CA3
:102DA000043043F002030373FFF7B7FFDFE7FFECE4
:102DB0000346EFF3118100228020EFF3108272B6F8
:102DC00080F3118882F310880A4A106860B1002BE2
:102DD0000EDB094A1268013A1A4050F8220018B175
:102DE000C2689A4218BF0020CBB283F311887047A3
:102DF0000020F9E7841100248011002438B504462E
:102E000018B3C068B0B1EFF3118200238025EFF34F
:102E1000108372B685F3118883F310880C4B00255C
:102E20001B68013B03400B48006840F82350D3B2B5
:102E300083F31188236D13B1204606F0B7FA2046BC
:102E4000FFF70CFF204607F007FF002038BD00BF4A
:102E50008011002484110024F8B54B1E0446FE2B7B
:102E60003BD8EFF3118600238022EFF3108372B674
:102E700082F3118883F31088027FCDB2022A0DD02D
:102E8000032A17D103681B7C994224DC294606F0EB
:102E90009FFAF6B286F311880020F8BD104B1B682C
:102EA0001B7C9942F2DC00F04BFC2046257400F0BC
:102EB00023FCEEE70B4B53F8327003EBC2031B7994
:102EC000DB0708D5394608F0E3FA39462046257471
:102ED00000F04AFCDDE72574DBE76FF01500DCE766
:102EE000B8110024307B170838B504460D46FFF7AB
:102EF000B3FF10B984F82E50607738BD10B5EFF3EA
:102F0000118400238022EFF3108372B682F31188BC
:102F100083F3108806F0C2FAE4B284F3118810BD7E
:102F20000A46002100F008B80A46002100F04EB819
:102F30000A46002100F056B8214B2DE9F743074619
:102F4000894690461D68EFF3118600238022EFF337
:102F5000108372B682F3118883F3108800F046FC68
:102F6000044688B1D8F80420164B9A4224D801AA06
:102F70004146484600F032FB28B9019C002C0ADC8F
:102F80006FF0730400E04442F6B286F311882046E5
:102F900003B0BDE8F0833C35FFF764FC21460346EF
:102FA000094A284600F092FA3846FEF7ABFD04467F
:102FB0002846FFF78DFCE7E76FF01504E4E700BF54
:102FC000B8110024FFC99A3BFF2F020870B50446D0
:102FD0000D461646324629462046FFF7ADFF031D33
:102FE000F8D070BD10B5FFF7A7FF041E05DA6442E4
:102FF000FEF7D8FA04604FF0FF34204610BD10B53C
:10300000EFF3118400238022EFF3108372B682F372
:10301000118883F31088FFF7CBFE28B1037F052BBF
:1030200002D1742100F025F8E4B284F3118810BDB8
:1030300070B50446EFF3118500238022EFF310836F
:1030400072B682F3118883F31088037F052B09D1B0
:10305000866D3146FEF742FF338801331BB2338061
:103060000023A3652046EDB2FEF762FF85F31188C9
:1030700070BDF8B504460E46EFF31185002380229B
:10308000EFF3108372B682F3118883F31088037F05
:10309000052B0DD1876D3946FEF720FF3B88204672
:1030A00001331BB23B8000232687A36506F0F6F9A7
:1030B000EDB285F31188F8BD012908B50AD00229BF
:1030C0000DD079B9827842F001028270FEF7AAFE33
:1030D000002008BD827822F001028270F8E76FF0CC
:1030E0008500F6E76FF01500F3E710B5FFF7E4FF92
:1030F000041E05DA6442FEF755FA04604FF0FF340F
:10310000204610BDF8B50024284B294E6020C3E9A5
:103110000044284BC3E90044274BC3E90044274B34
:10312000C6E90044C3E9004407F09EFD054648B1E6
:1031300000F160072C7528461835314608F044F92F
:10314000AF42F7D1602007F08FFD044658B100F17F
:1031500060050227174E277520461834314608F0BF
:1031600033F9AC42F7D1402007F07EFD044658B158
:1031700000F140050027104E2773204610343146D9
:1031800008F022F9A542F7D1402007F06DFD044672
:1031900058B100F140050227084E2773204610342D
:1031A000314608F011F9AC42F7D1F8BD941900246A
:1031B0008C190024841900247C190024741900241B
:1031C000002337B582680193EFF311858021EFF377
:1031D000108372B681F3118883F31088546B2CB975
:1031E000EDB285F31188019803B030BD217901A8B3
:1031F00008F0B9F92468F2E738B50D46044640B145
:10320000FEF7F8FBE46A14B1237CAB4203D1FEF76E
:1032100001FC204638BD2468F5E7FFEC124B10B5E1
:103220001B6843B1114808F003F9E0B91048BDE844
:10323000104008F0FDB8EFF3118400238022EFF373
:10324000108372B682F3118883F310880748E4B2C2
:1032500008F0EEF884F3118828B9182007F004FD6F
:1032600008B10123037510BDC41000248C1900247B
:103270008419002410B5037D83B9EFF311848022F3
:10328000EFF3108372B682F3118883F310880E492E
:1032900008F09AF8E4B284F3118810BD022B0CD127
:1032A000EFF3118400238022EFF3108372B682F3D0
:1032B000118883F310880549EAE7012BEDD1BDE8B9
:1032C000104007F0C9BC00BF8C19002484190024E9
:1032D00038B5044600F16405284608F0A9F850B94D
:1032E00004F16C05284608F0A3F838B94FF0FF3216
:1032F000C4E9172038BDFFF7BDFFEDE7FFF7BAFFC0
:10330000F0E738B5044600F12C05284608F090F89F
:1033100028B93434204608F08BF818B938BD00F0CD
:103320008DFAF2E7FEF79CFEF4E770470F4B70B59D
:103330001D68AC68FEF75EFBE37A5A0706D42846A0
:1033400000F032FABDE87040FEF764BB626900230A
:103350000AB11360636104F10C06E372A3891B04D4
:10336000EDD53046FEF71EFCF8E700BFB81100248B
:1033700008B5064B1B689B8E03F00303012B02D19B
:103380000020FEF719F90120FEF73CF8B8110024DF
:1033900008B580683C3008F002F90028D4BF00204E
:1033A000012008BD0023094A10B512F8334002EB92
:1033B000C301844204D14878C04300F0010010BD2D
:1033C00001330B2BF1D10120F9E700BF7C7B1708FB
:1033D00038B580684AB10023194A12F8335002EB1D
:1033E000C304A94214D16468B4B9EFF31184002373
:1033F0008022EFF3108372B682F3118883F3108872
:103400003C30E4B208F0BBF884F31188002414E0E7
:1034100001330B2BE1D1E8E7EFF311850023802284
:10342000EFF3108372B682F3118883F310883C3077
:10343000EDB208F098F885F31188204638BD00BF3A
:103440007C7B17082DE9F04386680024104D4FF06F
:1034500002093C36A04685B0304608F09CF86B68FF
:1034600073B12F7801A90022CDF80C903846CDE930
:103470000138012300F0F8F93946304608F073F8B6
:10348000013408350B2CEAD1002005B0BDE8F083EB
:103490007C7B170838B505464C2007F0F5FB044641
:1034A00030B10122002108F02CF80020AC6238BDB8
:1034B0006FF00B00FBE710B5846A2046FEF706FBB1
:1034C0002046BDE8104007F0C7BBFFEC2DE9F041F6
:1034D0000C4616469846054600284ED0002A4CD089
:1034E00000294ADBEFF3118700238022EFF31083DA
:1034F00072B682F3118883F3108843680BB1FFF72B
:10350000E7F91F4901346E600E68C5F80C801EB9DA
:10351000284607F059FF24E03046324600239168E0
:103520005B1801D5116831B9A3420CDC116829B9C7
:10353000E41A1349ECE710460A46F0E788680344AA
:1035400010460A46F0E791689642A3EB0103A4EB0C
:103550000304A1EB040191600AD10949284607F050
:103560003DFFAC60FFB287F311880020BDE8F08119
:10357000034A294607F038FFF3E76FF01500F5E737
:103580009C19002438B50D4C236843B19A68002576
:10359000013A9A60236813B19B68002B00DD38BDA7
:1035A000204607F045FF23681BB19A6881680A44EA
:1035B0009A6043684560C0689847EBE79C1900240F
:1035C00002680B689A4204D306D840684B68C01A58
:1035D00070474FF0FF307047012070477FB50E46AF
:1035E0006946154600F0F2F9044608BB69463046C4
:1035F000FFF7E6FF002805DA4FF0FF332B60204687
:1036000004B070BD019B7468009AE41A3368002C02
:10361000A3EB02030394029304DA064A013B22441B
:1036200002930392294602A807F044FF0446E6E706
:103630001624E4E700CA9A3B38B5036C04466BB91C
:103640000023236438BD07F007FB236C5859043569
:103650000028F8D1184607F0FFFAF1E70025F4E753
:1036600070B5046C84B1002054F8203063B14A1E58
:10367000013B12F8016F13F8015FAE42F9D00EB9A9
:103680003D2D03D00130EFE76FF0010070BD70B544
:10369000036C05460C4653F8210007F0DDFAA10043
:1036A0002A6C0B1DD05842F824000134286CC658EF
:1036B000002EF4D1012C03D107F0CEFA2E6470BD98
:1036C000083107F0D9FA0646F8E70023024601213F
:1036D00010B5044618460DF031F8002322460621A5
:1036E00001200DF02BF800232246062102200DF0C8
:1036F00025F8002010BDFFEC0F4B10B51B680446E9
:10370000B3F93620002A0ADD1A7C037C9A4206D2DD
:103710000A4900F029F80123002023770AE006492E
:10372000204600F021F802230028F5D0032222775A
:103730002268137710BD00BFB8110024AC1100241B
:1037400038B5436804465BB90368032201251A773C
:103750002046044907F09CFE00232846237738BD05
:103760000025F5E7B811002410B50B68027C5BB1A9
:103770001C7C944206D25A68C0E900328AB958606B
:10378000086007E01B68F2E74A68036022B94360FB
:10379000C1E90000012010BD4260106048600020B7
:1037A000F9E710605860FAE738B50446EFF3118581
:1037B00000238022EFF3108372B682F3118883F323
:1037C0001088037F043B032B0BD800F077F9042308
:1037D00007212046238700F05DF9EDB285F31188BB
:1037E00038BD072105F018FDF7E7FFEC38B5124B9F
:1037F0001D68E8B1EFF3118400228021EFF31082FD
:1038000072B681F3118882F31088028812B2002AFE
:103810000BDD0288013A12B20280FEF731FB002074
:10382000A865E4B284F3118838BD6FF00A00F8E7A8
:103830006FF01500F8E700BFB811002410B5EFF3E2
:10384000118400238022EFF3108372B682F3118873
:1038500083F310880349E4B207F0B6FD84F31188BE
:1038600010BD00BF941900242DE9F04F1746554AAA
:103870001F2885B0D2F800A005460C46DAF808905B
:1038800004D96FF0150005B0BDE8F08FD9B929460D
:103890004846FFF7B1FC0646FFB994B12768012FEF
:1038A00032D13A4629465046FFF792FD07468FBB74
:1038B0003EB1304609F12C0107F0A4FD3046FFF778
:1038C000BDFF0020DFE7002BE1D10B68012BDED02C
:1038D000FFF768FD0028DAD1D3E729465046FFF705
:1038E00057FD30B100230122C7E900230223BB604A
:1038F000D3E72EB173683B60B3687B60F368F6E78B
:10390000C7E90066BE60C8E7002229465046FFF7B7
:103910005FFDCCE7E6B9EFF3118B4FF0800A00238F
:10392000EFF3108372B68AF3118883F31088264868
:103930005FFA8BFB07F07CFD06468BF31188DFF8FE
:1039400088B05EB109F12C013046357407F03CFDBA
:1039500077606368B360A368F360B2E7502007F054
:1039600083F90646C0B1EFF31183EFF3108872B606
:103970008AF3118888F3108800F1500230465946C6
:103980001436CDE9022307F01FFD029A039B9642ED
:10399000F4D1DBB283F31188EFF31183019A029320
:1039A000EFF3108272B68AF3118882F310885846BA
:1039B000019207F03DFD029B0646DBB283F31188BE
:1039C000BFE700BFB811002494190024431E012B47
:1039D00037B50D460CD8084600F046F80446002CD2
:1039E00036DA6442FDF7DEFD04604FF0FF342FE06D
:1039F000002830D1684600F037F804460028EED1A0
:103A0000EFF3118300228021EFF3108272B681F36D
:103A1000118882F310881149DBB2009A086849685E
:103A200002440092019A0A44019283F311880C4ADD
:103A3000019B934208DD0B48009A93FBF0F10A4486
:103A400000FB113300920193009B2B60019B6B6084
:103A5000204603B030BD6FF01504C2E7A41900245E
:103A6000FFC99A3B00CA9A3B38B50025074B04466C
:103A70004FF47A7218682946002313F0CBFE044BEA
:103A8000206028465343636038BD00BFAC19002452
:103A900040420F0038B50C46074B054653F831102D
:103AA00003EBC4031B79DB0703D5FFF75DFE2C771F
:103AB00038BD07F0D7FCFAE7307B1708054B027FCB
:103AC00010B553F83210044607F0E2FC00232377C8
:103AD00010BD00BF307B170830B58DB00023054600
:103AE000694601A8009305F041F9041E05DB01A811
:103AF00009F0CAFA009B28606B6020460DB030BD0B
:103B000073B50346124CC0B122460068596803C21F
:103B10006846104EFFF7A8FF2368009A00206168EE
:103B20009B1A019A891A23600A46002A03F1FF357D
:103B300007DB50B9616002B070BD2046FFF7CCFFD3
:103B4000E6E732442B460120EFE7C4E90032F2E712
:103B5000A419002400CA9A3B08B504F0A5FF05F09B
:103B60000DF80020BDE80840FFF7CABF024A1368FD
:103B700001331360704700BFAC19002400F01AB87D
:103B800038B50D4604462F21284609F0B2F800B199
:103B9000451C284607F00DFB031E08DB07F01CFB45
:103BA000C368236083682362436823770023184631
:103BB00038BDFFEC014800F003B800BF3800002416
:103BC00010B5044648B1FDF715FF054B1A68226091
:103BD0001C60FDF71FFF002010BD6FF01500FBE714
:103BE000B019002437B504460D46002001A912F093
:103BF00029FB019B642B05D0642301A900200193BC
:103C000012F0EEFA00F012F82946204600F02CF8E7
:103C1000044612F0BDFA0449224600F51A7008F075
:103C2000BAFD012003B030BD6139160808B500F0B7
:103C300007F800214FF60170BDE8084009F06DBE9D
:103C4000002307B5054A00930123054905480CF0F8
:103C500027FFC01703B05DF804FB00BF88391608C2
:103C60008F3916089439160870B5054601200E469E
:103C700000F0EEF8044670B100F0BCF9204600F008
:103C8000C1F9334601212A46204600F085FC636ACB
:103C90000146204698476FF00B0070BD00F5297073
:103CA000704770B504460E461546B2B1D0F894324E
:103CB0003BB1D0F8980208F07DFCD4F8940208F0EB
:103CC00079FCD4F890322B60D4F88C326B60D4F845
:103CD0009832AB60D4F89432EB600023C4F88C6265
:103CE000C4F8943270BD38B50446D0F8945212F03E
:103CF0004FFA00F59C70854209D112F049FA00F59F
:103D00009C7008F057FC0123C4F88C3238BDD4F8FD
:103D1000940268B108F04EFCD4F8940208F0B6FAA8
:103D20004FF0FF33C4E9A3330023C4E9A533EDE723
:103D3000D4F88C020028F3DB0128F1D00BF00DFD44
:103D4000EEE738B50D460446FFF7CDFF2B68C4F803
:103D500090326B68C4F88C32AB68C4F89832EB6868
:103D6000C4F8943238BDFFEC10B5D0F89432044654
:103D70000BB1002010BD0949D0F88C0208F04AFAB6
:103D8000C4F8940230B1D4F88C32C4F89802C4F864
:103D90009032EEE74FF0FF30ECE700BFB24016087C
:103DA0000EB417B50446FFF7DFFF58B906AA059908
:103DB000D4F89802019208F0FBFC03B0BDE8104073
:103DC00003B070474FF0FF30F7E70EB417B5044665
:103DD000FFF7CAFF58B906AA0599D4F894020192D0
:103DE00008F0E6FC03B0BDE8104003B070474FF0A8
:103DF000FF30F7E770B505460C461646FFF7B4FFEF
:103E000068B92046D5F894323246012108F04FFBBC
:103E10000446D5F8940208F0CDFB204670BD4FF063
:103E2000FF34FAE710B50446FFF75DFFD4F89C02B3
:103E300008B106F011FF2046BDE8104006F00CBFA7
:103E40000C4608B5FFF7EEFF2046FDF7DBFAFFEC66
:103E500038B505464FF4497006F016FF044638B3EE
:103E6000144B154A0360154BC2618360144B154A0D
:103E7000C360154B02624361144B80F888520361A2
:103E8000134B8361134B4362022380F82B32C0F83B
:103E9000903212F07DF9012300F51A70C4F88C32CB
:103EA000C4F8980212F074F900F59C70C4F89402FA
:103EB000204638BDD93E0208A33C0208253E020830
:103EC000F53D0208433D0208CB3D0208A13D020832
:103ED0009D3C0208413E020808B590F88802FFF7B1
:103EE000B7FF08BD2DE9F74F0D461146044600F017
:103EF000BBF80646F8B1A369204698470746002854
:103F000068D036493046D4F8308208F09AF9C4F8BF
:103F10003002B0B92769FDF745FB006808F0A4FE40
:103F20002F4B2A462F4900902046B847304600F0D4
:103F3000BFF8C4F830824FF0FF35284603B0BDE823
:103F4000F08F4FF0FF35DFF8A890DFF898A012F05F
:103F50001FF900F59C7008F02DFBD4F8300208F032
:103F60001EFA0023C4F834029842A4F838320CDA5E
:103F7000D4F810B0FDF716FB006808F075FE1A4B78
:103F800000904A4651462046D847D4F83022802136
:103F9000384608F02CFA98B194F82B329A0704D4DA
:103FA00063693A461149204698473946204601F050
:103FB000E5FD05460028CAD094F82B32DB07C6D4AD
:103FC000D4F8300208F062F9C4F83082304600F0CC
:103FD0006FF8B2E74FF0FF35F8E700BFF73E16087D
:103FE0009E391608357C1708A4391608348C160833
:103FF000AA391608014A0249FFF774BFAF391608FB
:10400000BE39160838B50446FDF7F4FC084B01220A
:104010001D781A70FDF7FEFC45B9064A2046064990
:10402000FFF760FF022384F82B3238BD0020FCE745
:10403000B4190024C63916083CCF160808B5024941
:1040400043699847002008BD8C61170808B50448EB
:1040500011F028FF034B002808BF184608BD00BF19
:10406000DD7B1708D47B170870B506460C4609B1EE
:104070000B7823B90C48BDE8704008F0E7BD2F2B42
:1040800001D10846F7E7FFF7E1FF0849054620465A
:1040900008F084FE08B92846EDE722462946304656
:1040A000BDE8704000F066BCD47B1708D313170836
:1040B00008B106F0D1BD704701292DE9F34106464C
:1040C00017464EDD55682949284608F067FE044624
:1040D000002847D02649284608F060FE044650BB19
:1040E000244811F0DFFE244B002808BF184608F0D2
:1040F000ADFD804609F0BAF8054670B13F683569F4
:10410000FDF750FA006808F0AFFD1C4B00903A46EE
:104110001B493046A8474FF0FF35B8F1000F02D0D9
:10412000404606F099FD14B12046FFF7C1FF28462E
:1041300002B0BDE8F0811349284608F02FFE04467E
:1041400038B9FFF783FF08F081FD804607F0DEF8FD
:10415000D0E729463046FFF787FF4FF000080446B6
:10416000C8E70024A0460448C4E700BFD6391608B3
:10417000D33E1608D67B1708D47B1708D839160803
:10418000357C1708E9B716082DE9F04F012387B0F1
:10419000074690464FF0000A5F4C02910193224679
:1041A0004146029809F01CF8431C10D109F025F88B
:1041B000D0F800904FF05C0B08EB8908029B994502
:1041C0001FDB019B002B40F0A18000200DE0652843
:1041D0000ED06E280FD0452810D03B693846D8F84D
:1041E00000204E4998474FF0FF3007B0BDE8F08FF0
:1041F0004FF0010AD3E700230193D0E74FF0000A04
:10420000CDE708F0FAFF03684B4503D07B693846D9
:1042100043499847BAF1000F63D0D8F800502C46B4
:104220002B780BB923705CE05C2B04D02E4604F88D
:10423000013B751CF4E76B786E1C0D2B0AD80D2B17
:104240000ED8DFE803F04A0D0D0D0D0D0D57590D79
:104250005D615B5F5C2B35D0782B08D0302B16D09E
:10426000234603F802BB6A7862701C46E1E7033517
:104270000023049616F8012F05931046039206F0CA
:10428000CCFF059BDDE90321A0B90E461AE00435F9
:104290000021737832460136303BD8B2082803D962
:1042A000164604F8011BC4E7AE4203EBC101F0D18E
:1042B0003246F5E7A2F130011B01092905D80B446C
:1042C000AE42D6D104F8013BB3E71046039306F0A3
:1042D000B2FF039B57380344F2E7002384F800B091
:1042E00063707B69384658F8042B09F101090D49C0
:1042F000984763E70723E5E70823E3E70C23E1E7B3
:104300000A23DFE70D23DDE70B23DBE77B69384674
:104310000549984759E700BFDE391608FB7C1708A6
:1043200006411608348C16086624170838B504466A
:104330004569FFF78BFE034902462046A847002047
:1043400038BD00BF8C6117082DE9FF474E4B16465C
:104350000DF10C0801291A8804469B780D46ADF82A
:104360000C2088F802300DD10022484900F0D4FB1F
:10437000054663692046ED1745499847284604B02D
:10438000BDE8F087022901D0042968D17768384652
:1043900008F02BFD01280FD836682569FDF702F9D2
:1043A000006808F061FC3B4B32463B4900902046D8
:1043B000A8476FF01505E1E797F80090B9F12D0FC8
:1043C0000ED0B9F12B0F0BD036682569FDF7EAF84E
:1043D000006808F049FC2F4B324630490090E6E770
:1043E0004FF0010A17F8011F11F0DF0F22D102234D
:1043F000033D012D46D801339D0056F8230000F0FF
:104400009BFA0746043D705911F04CFD48BB7159A9
:104410003A46204600F022FB051EAFDA68422769C3
:10442000366808F021FC1E4B009032461D4920469C
:10443000B847A3E7404608F0A7FC0028C4D0A0EB8B
:10444000080394F82B22B9F12B0F0AFA03F30ABFE1
:10445000134322EA0303DBB284F82B32C2E70123C1
:10446000C6E7705901223946FEF730FB051E85DA92
:1044700027693668FDF796F8006808F0F5FB0A4BE7
:104480000090D2E7002579E7551917083D4002084A
:10449000662417086E1617082F7D1708FB7C17086F
:1044A000E2391608357C1708FC391608F7B551684B
:1044B0000446154600F00CFB002825DA831C23D0A7
:1044C0002F684042266908F0CFFB104B3A46009017
:1044D00020460F49B0474FF0FF366868FEF764FB8F
:1044E00000280EDA2D682669FDF75CF8006808F0F0
:1044F000BBFB084B00902A4605492046B0474FF0C9
:10450000FF36304603B0F0BD0026E6E7ED39160869
:10451000357C1708FA391608032973B50546144681
:1045200017D1916801226068FEF7D0FA002819DAE5
:104530002E692468FDF736F8006808F095FB124BE9
:104540000090224611492846B0474FF0FF3002B094
:1045500070BD516800F076FA0D4B002814BF01467B
:104560001946DFE76168284600F0B2FA002809DA48
:10457000831C07D040422E69246808F075FB054B68
:104580000090DEE70020E2E7FA391608357C1708CC
:10459000E2E41608ED391608F7B5044617461D463D
:1045A00041B1D0F89412374808F0C6F8D4F8940214
:1045B00008F000F8012F29DC334F04F52976D4F8F0
:1045C0009412384608F0B8F8D4F8940207F0F2FFD5
:1045D00011F0DEFD054611F0DBFD802100F59C7336
:1045E00005F10802304600F0B0FA013040D1D4F8AD
:1045F0009842FCF7D7FF006808F036FB234B009089
:104600002046234A234908F0C6F80AE06E6822498A
:10461000304608F0C3FB30B9636920462A681F4959
:104620009847002013E01E49304608F0B7FB80B9D8
:10463000022F06D0A968204603B0BDE8F04001F083
:104640009DBA23692A68174920469847012003B07C
:10465000F0BD337829682D2B03D10A46236912490E
:10466000F2E73246204603B0BDE8F040FFF73ABC1F
:104670003146204601F082FAD4F8940207F09AFFFE
:104680009DE700BF737D17086D7D1708313A160846
:104690003A3A1608357C1708033A1608063A1608FF
:1046A0002E3A16082F7D1708567D17082DE9F74F6B
:1046B00004460D461046012116460BF0EBFB071E83
:1046C0001DDA05223F49304608F003FB28B9276967
:1046D00033462A463C492046B8472669FCF762FF24
:1046E000006808F0C1FA394B00904FF0FF392A46B4
:1046F00037492046B047484603B0BDE8F08F4FF435
:10470000007006F0B1FA064658B938460BF025F8A5
:104710002669FCF747FF006808F0A6FA2D4B0090C9
:10472000E3E74FF00009DFF8B4A021E008F09CFABD
:10473000294B00902A4626492046C0472CE02DD020
:104740004FF00008E368ABEB080206EB08012046D7
:104750009847002832DAFCF725FF0068D4F810806B
:10476000042822D12A4651462046C0474FF0FF393F
:104770004FF40072314638460BF0C6FBB0F1000B27
:10478000DDDAFCF70FFF0068D4F810800428CDD1E3
:104790002A4612492046C0474FF0FF3938460AF0F2
:1047A000DCFF304606F058FAA5E708F05DFA0C4B3E
:1047B00000902A4606492046C047D7E78044C345B3
:1047C000C0DCD5E7463A16084C3A16089F39160859
:1047D000357C17087D3A160847841608E47B1708CD
:1047E0005DC216082DE9F74F05468846104601219F
:1047F0001F460BF04FFB061E11DA2C694FF0FF3AF3
:10480000FCF7D0FE006808F02FFA1D4B00904246DE
:104810001C492846A047504603B0BDE8F08F0C9BCA
:104820000024B94603F1FF3B3C705A4649463046E6
:104830000BF06AFBB0F1000A16DAFCF7B3FE03686E
:10484000042B19D02C69FCF7ADFE006808F00CFAB7
:104850000D4B009042460B492846A0474FF0FF3AC7
:1048600030460AF07AFFD6E7FAD054444FF00003FE
:10487000D144ABEB0A0B3B550C9B002BD5D1EDE79C
:104880009F391608357C1708478416082DE9F3412F
:10489000044610460F461546984606F0D2FC0646DA
:1048A000E8B905221749284608F013FA28B92669FD
:1048B0002B463A4614492046B0472569FCF772FE5C
:1048C000006808F0D1F9009020464FF0FF340F4BFC
:1048D0003A460F49A847204602B0BDE8F08130466D
:1048E00006F0DDFC024658B1089B29462046C04729
:1048F0000028F4DA4FF0FF34304606F0BDFCEAE75A
:104900000446F9E7463A16084C3A1608843A16085F
:10491000357C170810B5044608F067FA0021231803
:104920001A1B013A002A03DD13F8012C2F2A00D0AC
:1049300010BD03F8011DF3E7F8B5044620782546BD
:104940002646013468B92846002708F04EFA2C188C
:10495000B44204D014F8010C06F055FC30B92846D6
:10496000F8BD06F050FC0028E8D1ECE704F8017D22
:10497000EEE7FFECF7B50D4604461049164628460B
:1049800004F1280708F00AFA78B933460C4A4FF4C4
:104990000071384606F089FE0023384684F8283135
:1049A00003B0BDE8F04008F051B92B46054A4FF47A
:1049B00000713846009606F078FEEDE77ADA1608C0
:1049C0008E3A16088C3A160870B5D0E9A7450E46FF
:1049D0002544AC4212D2701E611E10F8012F11F84E
:1049E000013F9A42F9D01AB93D2B01D1204670BD42
:1049F000204608F0FAF901300444EAE70024F5E71C
:104A000070B5D0E9A73605460C468B421E4416D831
:104A10008E4214D9084608F0E8F90130631E0444B8
:104A2000321B002A06DCD5F8A0321B1A0020C5F87C
:104A3000A03270BD14F8012B03F8012FF0E74FF0FE
:104A4000FF30F6E708B5FFF7BFFF034618B13D2179
:104A500008F09AF9431C184608BDFFECF8B5D0F8E9
:104A60009C3205460E46174633B1FFF7ADFF0146AF
:104A700010B12846FFF7C4FF304608F0B6F90446E7
:104A8000384608F0B2F90444D5F89C020234B0B1BB
:104A9000D5F8A0321C44214606F0EEF8024610B9C3
:104AA0006FF00B00F8BDD5F8A03218443B4607491B
:104AB000C5E9A724324606F0D4FD0020F2E72046DF
:104AC00006F0D2F80028EBD00246EFE75B39160873
:104AD00010B5044698B1FFF777FF014678B120463C
:104AE000FFF78EFFD4E9A70100290CDC20B106F006
:104AF000B3F80023C4F89C320023C4F8A032FCF7BA
:104B000089FF002010BD06F0B7F810B1C4F89C0270
:104B1000F5E76FF00B00F5E72DE9F041D0E9A74686
:104B200005460F4690462644B44202D30020BDE815
:104B3000F081224641462846B8470028F7D1204652
:104B400008F053F901300444EEE75B68526800F066
:104B50002FB800690BF0C2BC13B504468DF80710DE
:104B600001220DF1070120690BF0B8FC002802DBDF
:104B7000F6D002B010BDFCF715FD0368042BF7E773
:104B800013B5044601220DF10701E0680BF0BCF9F2
:104B9000002809D003DB9DF8070002B010BDFCF728
:104BA00001FD0368042BEDD04FF0FF30F5E7FFEC7B
:104BB00010B586B0074C0492074A01940292074A46
:104BC000059303920A46014601A800F009F806B0D1
:104BD00010BD00BF814B0208594B0208534B02081D
:104BE000012A2DE9F04706460F46914604DC0024D1
:104BF0000C702046BDE8F0870025836803222C490D
:104C000098474FF00008336830469847431C0446E5
:104C10000BD1002DEDDD00232C467B55E9E74FF04D
:104C20000108F0E74546D046EDE7B8F1000F09D09E
:104C30005B28E6D1B8F1020818BF4FF001084FEA2F
:104C40004808E0E71B28EAD012DC0A2812D00D2819
:104C500010D0082817D1002DD5DD73683046082103
:104C6000013D9847B3680322114930469847CAE787
:104C70007F28EFE76C1C0A210023304679553B550D
:104C800073689847B5E7E0B206F0B4FA82460028A8
:104C9000B9D17C5505F101080235736821463046CB
:104CA00098474D45BEDB444607F808A0A1E700BF82
:104CB000E17B170890F83B220346043200EBC20266
:104CC00092F82802800901280CD1002081F001010E
:104CD00083F82A0292F8283261F3000382F828321E
:104CE00000207047022803D1002083F82A02F1E750
:104CF00093F83C221A4492F83D02800901280CD115
:104D0000002083F82A0292F83D32C3F3800041402C
:104D100061F3000382F83D32E2E7484283F82A1249
:104D20007047024610B50023104612F8014B5C2C68
:104D300000D143B18C4202D1002BF4D110BD002C24
:104D4000F1D12046FAE70123EEE70023027802B909
:104D500070475C2A00F101010AD14BB903465A7829
:104D600003F8012B002AFAD1014601230846EDE79A
:104D70000023FBE790F83B32024600EBC30393F8B5
:104D800048329909032902D113F001000CD092F89E
:104D90003C321A4492F83D0283070CD48309022B5B
:104DA00005D0032B04D0012000F001007047C04360
:104DB00000F00100F8E70020F6E770B5056804464A
:104DC00095F8293213B140680AF0C7FCAB68284651
:104DD00004F1080600259847A368AB4204DC20468E
:104DE000BDE8704005F038BF56F8040F013505F0F6
:104DF00033FFF1E72DE9F041804617460C46B9B183
:104E0000084607F0F2FF0646384607F0EEFF411C61
:104E10002046314405F030FF054658B92546D8F8FC
:104E20001030074A4046074998472846BDE8F081B8
:104E30000E46E9E700233946835507F0E9FEF4E71B
:104E4000923A16081D7C170838B500F10C028168EB
:104E50000446006801F09AF805462046FFF7ADFFCA
:104E6000284638BD2DE9F04F89B0894604461546DD
:104E7000129F1E460097116802F042FA002808DBD4
:104E800014BF01210021204609B0BDE8F04FFFF713
:104E900011BF94F82932B3B139464FF4DB72304672
:104EA0000AF0F8FF071E10DA2D682669FCF77AFB76
:104EB000006807F0D9FE554B00902A465449204619
:104EC000B0470121DFE74FF0FF3794F82832002B7D
:104ED00000F08380236820469847804640B15C20DC
:104EE00005F0D2FE064658B9D8F808304046984733
:104EF00094F82932002BE4D038460AF02EFCE0E783
:104F000083464FF0000AC0E900874BF8089FD1455F
:104F10001EDC94F829322BB1D8F81C300022394617
:104F20004046984702A9002011F08CF9C8B12769C2
:104F30002D68FCF737FB006807F096FE354B0090B4
:104F40002A4633492046B8473046FFF736FFB8E7D0
:104F500055F82A000AF1010A07F078FE4BF8040F11
:104F6000D5E7D4F82C32002B0BD0029F4FF0010074
:104F7000A7EB03071EDA06F099FA8742A8BF074697
:104F8000029704A806F0EEF9012104A806F0F8F94A
:104F900002A904A806F0FCF933461F4A04A903A895
:104FA00006F004FA60B127692D6807F05DFE1B4B1F
:104FB0000090C5E706F07CFA8742B8BF0746DFE7F6
:104FC000039811F08DF8029B154920460093039B2E
:104FD00066692A68B047002155E794F8293223B161
:104FE000E36904AA3946204698472A46494620469E
:104FF00000F0CCFF94F8293205461BB1236A04A9BE
:1050000020469847002DE6DA5BE700BF9F39160877
:10501000357C1708943A1608494E0208A23A160839
:10502000B13A1608F8B50025044606462F4623680F
:105030009D4201DB2760F8BD56F8040F013505F0ED
:105040000BFE3760F3E7FFEC2DE9F04F0446BDB0EF
:105050000E46D1F80090A44F0592039399F8008072
:105060004D4609F10109B8F1000F17D04146384605
:1050700007F08AFE0028F1D1B8F13E0F0AD16B7813
:105080003E2B0DBF0235994DC6F80090356008BF24
:10509000974D04E0B8F1230F05D13560002528466F
:1050A0003DB0BDE8F08FB8F1220F039B8E4F8246D2
:1050B00004BF00234D460393A9468E4B08BF1F46ED
:1050C0000346C84619F8011B69BBC6F80080AA460A
:1050D00000268949504607F0ABFD83460AEB0B07D3
:1050E00007F1010897F80090BBF1000F4DD0B9F11E
:1050F000000F33D1002E67D0314652462046FFF7CD
:1051000079FE0546FFF721FE2E46002EC7D0059BEF
:105110001B681D2BC3DC059A02EB8302013356602A
:10512000059A1360BBE718B102785C2A00D193B1ED
:105130005C2903D0602903D18AF0010A00230BE027
:10514000BAF1000FFAD13846FFF7EBFD0028F5D091
:1051500008F801ABB9E701234046B2E70BF1FF3392
:1051600000225344A3EB0B0013F801195C2903D16F
:10517000834282F00102F7D152B10BF1010B5E497B
:10518000781C07F055FD8344A8E7B9F1000FB1D0B2
:10519000B9F1600F40F059814FF00003314652469B
:1051A000204607F8013BFFF725FE494606463846EC
:1051B000FFF7B7FD049058B9504B25691A4650497E
:1051C0002046A8474F4DA0E72846FFF7BEFD66E7FB
:1051D000049B4FF000021A7000230793FDF742FB77
:1051E000494A0346494907A806F052FA002804DB59
:1051F000DDF81C90B9F1000F18D123692046444A0C
:10520000444998474FF000083E4F31463A46204601
:10521000FFF7F0FD0646B8F1000F02D0404605F05A
:105220001BFD049B03F10108C24652E750220021F6
:1052300009A8FCF740F97C2200211DA8FCF73BF9E6
:105240004FF48073B4F828B21DAAA4F8283208A934
:10525000002320460897FFF7F7FE074668B320466D
:10526000FFF788FD40B30DF1240A4FF001080997BC
:1052700000231DAA08A92046FFF7E6FE4AF8040FFE
:1052800020B108F10108B8F1130FF1D13CAB0022B5
:10529000B8F10F0F03EB880343F8CC2C04DD23692E
:1052A0003A461D4920469847262309AA41462046EA
:1052B00000934B46FFF7D6FD07461DA8A4F828B279
:1052C000FFF7B0FE77B32769FCF76CF9006807F0C9
:1052D000CBFC124B009020460D4A1149B847079865
:1052E00005F0BAFC8EE700BFA67D17089C7D170865
:1052F000997D1708993E16089E7D1708D03A160822
:10530000167D1708927D1708BD3A1608C23A16088E
:10531000CF3A16081D7C17088C7C1708D23A16085D
:10532000357C1708DDF81C801DA940460BF022F8DB
:10533000834620B32769FCF735F9006807F094FC31
:105340006F4B009020466F4A6F49B8474FF00008F6
:105350006E4F07980BF08CF800280CDAD4F81090F8
:10536000FCF720F9006807F07FFC694B00902046AD
:10537000644A6549C847079805F06EFC45E7DDF8C3
:105380008C9009F1010005F06FFC074628B92369EC
:1053900020465C4A5F499847D8E7404601210AF019
:1053A00079FDB0F1000833DAD4F81080FCF7FAF890
:1053B000006807F059FC584B00902046514A52496A
:1053C000C047384605F048FCC0E74FF4007240463D
:1053D0000AF09AFD00281ADAFCF7E4F80368D4F81A
:1053E0001090042B07D1474A20464C49C8474046F5
:1053F0000AF0B3F9E5E7FCF7D5F8006807F034FCEC
:10540000474B009020463F4A3F49C847EFE7834457
:10541000D94507EB0B01D8D88A46DFF82091BA4569
:1054200007D01AF8011C48460AF1FF3B07F0ACFC14
:1054300048B90023AAEB070A4046B84607F80A30E5
:105440000AF08BF985E7DA46E9E7B9F1240F7FF432
:10545000EBAE4FF00003B9463146524609F8013B26
:105460002046FFF7C7FC7B7806467B2B32D107F13D
:1054700002097D214846FFF754FC18B92569294BDC
:10548000294A9CE680464FF0000308F8013B039B45
:1054900013B10123039A13602449484607F07EFCA8
:1054A000F0B994F82A12224A224F00290CBF9246E2
:1054B000BA4694F82B329B0705D453464A461E49F8
:1054C00020466769B847314652462046FFF792FCAE
:1054D0000646A9E6484607F088FC09EB0008D6E72F
:1054E00049462046FFF7AEFA82460028E1D14846F9
:1054F00010F0D8FC054B002814BF82469A46D8E726
:10550000D73A1608CF3A1608357C1708927D170847
:10551000DC3A16081D7C17089F391608E47B17082B
:10552000478416088EC71608E33A1608977D1708B1
:10553000957D1708937D1708E63A1608A67D17088B
:105540002DE9F04FB9B004460D465022002105A8C0
:10555000FBF7B1FF7C22002119A8FBF7ACFF002369
:1055600019AA03A92046A4F828320395FFF76CFD79
:105570000546002800F03082A64907F00FFC81465E
:10558000A549284607F00AFCB9F1000F02D000280F
:1055900040F08C80002319AA03A92046FFF754FD90
:1055A000074608B103781BB923692A469B4925E0C1
:1055B00094F83C8204EB080393F83D329B09012BDD
:1055C00014D094F83B6204EBC60393F84832C3F35B
:1055D0008113033303F00303012B07D9D4F83032CE
:1055E00023B1D4F834A2BAF1000F02DA23692A46B3
:1055F00078E0062E1BD923692A4689492046984718
:1056000094F84832002203F03E03A4F83A2243F013
:105610000103C4F84C2284F8483219A8FFF702FDB0
:105620000121204639B0BDE8F04FFFF743BB0136FA
:10563000B9F1000F2046F6B214BF02250125FFF78D
:1056400099FB321D002384F83B6204EBC60604EB91
:10565000C20284F83A3240EA8513B4F8381292F85C
:1056600028023D4623F03E03514400F03E00034330
:1056700082F8283286F84982C6F84C1269492846D1
:1056800007F08CFB0746002840F03181034619AA39
:1056900003A92046FFF7D8FC054618B10378002B74
:1056A00040F08B8023695F4A5C49AAE05E49284646
:1056B00007F074FB034608BB19AA03A92046FFF7AD
:1056C000C3FC94F83B320546043304EBC30393F860
:1056D0002812C1F38112033202F00302012A03D916
:1056E0002369514A514989E741F0C00183F82812E2
:1056F0000028C3D10023C4F82C3259E14C49284674
:1057000007F04CFB0346002848D119AA03A92046FC
:10571000FFF79AFC024610B12369454A46E794F820
:105720003B02031D04EBC30393F828128D09032DDC
:1057300002D023693E4AD5E718B923693C4A3D495E
:105740005CE7C80725D5D3F82C12D4F8300206F050
:1057500006FE00280BDA2569FBF724FF006807F036
:1057600083FA354B00902046314A3449A84701233B
:1057700084F83A3294F83B321A1D013B04EBC20222
:1057800092F8281221F0C00182F8281284F83B32E6
:10579000B0E741F0010183F82812EBE794F83B32BF
:1057A00004EBC30393F84832C3F38113033303F0CC
:1057B0000303012B3FF662AF18E7214907F0EEFA29
:1057C000034668B919AA03A92046FFF73DFC054620
:1057D00000283FF467AF0378002B3FF463AF012745
:1057E00094F83C62A31993F83D329B09012B03D135
:1057F00023690C4A0D4904E0062E23D92369094A7E
:10580000074920469847B4F83C3203F46053A4F8A3
:105810003C3202E7EF3A1608F53A1608FB7C170807
:10582000717C1708093B1608FB3A16084D7C1708CF
:10583000FE3A1608047C1708033B1608357C170847
:10584000A64D170820460136FFF794FA80F00103B1
:10585000F6B25B0084F83C62264443F0400396F8BD
:105860003D2243EA870302F0380223F03803134352
:1058700086F83D320023C4F82C32B349284607F09D
:105880008DFA0346002840F0B2800A2203A9204680
:10589000C4F82C2219AAFFF7D7FB0546002800F010
:1058A0008780AA4907F07AFA0646002840F09F80D0
:1058B000034619AA03A92046FFF7C6FB074600289E
:1058C00000F09580324604A907F02FF8C4F82C02A6
:1058D0001430272805D8049B9F4202D01B78002B48
:1058E0007DD023692046984A9949984795E6994979
:1058F000284607F053FA0346D8B919AA03A9204647
:10590000FFF7A2FB94F83C220546224492F83D3270
:105910009909012902D023698E4A6BE7022161F3BC
:10592000871382F83D320023C4F82C32002DA4D115
:105930003EE08949284607F031FA0346A8B919AA7A
:1059400003A92046FFF780FB94F83C320546234428
:1059500093F83D229109022902D023697E4A49E742
:1059600042F0C00283F83D22DDE77C49284607F07B
:1059700015FA034620BB19AA03A92046FFF764FBCA
:1059800010B12369754A8FE694F83C32E21892F818
:105990003D227F2A02D82369704A2BE71BB923696D
:1059A0006F4A70492DE7013BC4F82C0284F83C3261
:1059B000002519A8FFF736FB284639B0BDE8F08F5F
:1059C00094F83C32234493F83D329B09012B7FF439
:1059D00051AF23692A460DE7C4F82C02E8E719AA5B
:1059E00003A92046FFF730FB05460028E0D02046FB
:1059F000FFF7C0F90028DBD001264FF00008DFF8E0
:105A00007891059504AB19AA03A92046CDF810801A
:105A1000FFF71AFB38AB07464FEA860A03EB86030B
:105A200043F8CC0C00286ED0049BE3B105AB9A443C
:105A30005AF804BB5F461BF8011BA1B1484607F0AA
:105A4000A3F90028F6D0013607F8018BBB4617F8FA
:105A5000011B21B1484607F097F90028F6D1132E13
:105A6000CAF800B0E4D10136122ECBDD771E38AB78
:105A70003D4903EB870353F8CC0C07F08FF918B9B5
:105A800001233E4684F82832022E58DDA6F1020991
:105A900038AB364903EB890353F8CC7C384607F022
:105AA0007DF9A8BB012394F82982204684F8293285
:105AB00038AB03EB860656F8D01C4E46FEF7D4FAF8
:105AC0004FF02609074638AB00220F2E03EB860362
:105AD00043F8CC2C04DD23692A4625492046984703
:105AE0003B4605AA31462046CDF80090FFF7BAF9AB
:105AF000054627B13846FEF7DBFA84F8298219A853
:105B0000FFF790FA58E7012EB0DC80468146DAE7CD
:105B10001849384607F042F988B9012394F82982D8
:105B2000204684F8293238AB03EB860656F8D01CA1
:105B30004E46FEF799FA4FF016090746C3E74FF0B5
:105B40000008C1464746BEE7193B16081E3B16082B
:105B5000FB7C17080C3B1608113B1608163B160871
:105B6000093B1608047C1708213B16089C7D170882
:105B70008C7C1708997D1708A67D17082DE9F0473A
:105B8000002305460E460C4688461F4F80F83A32E1
:105B900095F83AA2BAF1000F01D000202EE0A31B25
:105BA00039462046A5F8383207F042F8235C22181F
:105BB0001BB10A2B01D0232B05D141462846BDE855
:105BC000F047FFF7BDBC3B2B02F1010909D141466B
:105BD000284682F800A0FFF7B3FC78B94C46C846C7
:105BE000D6E722214846FFF79CF848B9074B2846DC
:105BF0002C691A460649A0474FF0FF30BDE8F087F0
:105C0000441CC146EBE700BFA17D1708993E16086A
:105C1000167D170890F83B32043300EBC30393F86A
:105C200028229209032A09D193F8292280F83C22DC
:105C300093F8282222F0010283F8282200207047DE
:105C400008B503490369126898474FF0FF3008BD53
:105C5000C27C1708002070474FF0FF30704708B52E
:105C60000021436A9847FFEC10B4CB680A68446986
:105C700023B1A44604495DF8044B60472346034919
:105C80005DF8044B184700BF233B160884611708D2
:105C900070B504460D460D4E306830B923692A466A
:105CA00020460B49BDE870401847294607F076F8B2
:105CB00050B963692A46074920469847314620462D
:105CC000BDE87040FFF7D0BF1036E5E7AC7D1708A0
:105CD000C27C17082C3B160801292DE9F74F044612
:105CE0000F46164640F3F1809349506807F056F886
:105CF000054600285FD1022F06D00222012356F864
:105D00002250002B00F0DE80636920468B499847C3
:105D100063698B492046984763698A4920469847BA
:105D200063698949204698476369884920469847AE
:105D300063698749204698476369864920469847A2
:105D40006369834920469847636983492046984799
:105D500063697C4920469847636980492046984793
:105D600063697F4920469847636979492046984787
:105D700063697C4920469847636972492046984781
:105D80006369794920469847636975492046984771
:105D900063696F492046984763697249204698476E
:105DA000002D00F0C38029462046FFF771FF002038
:105DB00003B0BDE8F08F01220023A0E7294610358B
:105DC0002046FFF751FF2B68002BF7D100273E46F6
:105DD0003D46384605F000FA002854D1002DE6D0A3
:105DE0000236013D4FF000086369502E5F4920469E
:105DF00096BF50270127B7FBF6F73D449847B5FB00
:105E0000F7F54545D3D0C1464FF0000A63692046F7
:105E100057499847484605F0DFF9834640B1DBF81B
:105E20000C30002B3AD10AF1010AA9445745F1D1AF
:105E3000636920464F4908F101089847E1E7B946F0
:105E40004FF0000B4FEA09134B4920465AF8032044
:105E5000636901929847019A104606F0C6FF03460F
:105E60009D42626908D80BF1010BC1445E4557D0D1
:105E7000B9F1240FE6D953E04049204601939047F9
:105E8000019B0133ECE7C36833B10068013506F0CC
:105E9000ACFF864238BF064601379AE7DBF80020A0
:105EA0002046636934499847DBF8000006F09DFFFF
:105EB00083465E45B7D96369204630490BF1010B33
:105EC0009847F6E7002D7FF46EAF00262C49204658
:105ED000DFF8B4A03546FFF7DBFE636920462549AD
:105EE00098475AF82600043606F07FFF854238BFEF
:105EF0000546942EF5D102350027502D96BF502629
:105F00000126B6FBF5F606F12408B8FBF6F8B8450D
:105F10003FF45CAF6369204615499847242F8ED91A
:105F200063692046134901379847F0E763692046C3
:105F30001449154D984746E7363B1608393B160875
:105F40004D3B1608883B16088C3B1608983B1608F4
:105F5000A03B1608B93B1608C13B1608C83B1608FB
:105F6000D73B1608DD3B1608E63B1608FA3B160839
:105F70000541160866241708348C160806411608D1
:105F8000F53B16080A3C1608AC7D17082DE9F041D0
:105F900004460E461746D2F80080124D286808B90C
:105FA000114B17E0414606F0F9FEC8B92B7AB3420F
:105FB00008DD236942460D49204698474FF0FF30DF
:105FC000BDE8F0816B7AB34203DA2369424608499F
:105FD000F2E76B683A4631462046BDE8F041184783
:105FE0001035DBE7AC7D1708415C02082F7D1708F0
:105FF0008C7C170810B50749044606F0CFFE38B16F
:106000000549204606F0CAFEB0FA80F0400910BDEE
:106010000120FCE7D3131708E9B716082DE9F04370
:106020009D0795B00446884616461F4670D0E2B1DB
:106030000132FEF79FFC814605A90AF09BF905464F
:10604000484604F009FEB5B12569FBF7ABFA0068D4
:1060500006F00AFE434B00902046434A4349A847B6
:106060004FF0FF3015B0BDE8F08305A940460AF0B7
:1060700081F90546E7E7B90743D53D4B02AD1868FE
:1060800059681A899B7A03C5AB702A80079D05F46D
:106090007043B3F5C04F4FD162238DF80830EA0545
:1060A00044BF72238DF809302B0644BF77238DF847
:1060B0000A30680644BF78238DF80B30A90644BF28
:1060C00072238DF80C30EA0644BF77238DF80D302B
:1060D0002B0744BF78238DF80E306807204644BF55
:1060E00072238DF80F30A907224944BF77238DF81A
:1060F0001030EA0702AA44BF78238DF81130636993
:106100009847FB0704D5636920460B9A1A499847BC
:10611000636916B3771C174920463A469847337887
:106120006569042B17D13846FFF764FF98B9134906
:106130002046A847002095E7B3F5005F01D163230F
:10614000ABE7B3F5804F01D16423A6E7B3F5004F69
:10615000A5D03F23A1E70A49EAE74246094920467C
:106160009847E7E7D73A160884551608357C17088C
:10617000CA3E1608B76E1608C23E1608C73E160875
:10618000662417088B6117082DE9F04F91B005467A
:1061900001A90AF0FDF8041E4EDB039B284603F418
:1061A0007043B3F5804F03D00AF062F9044643E030
:1061B00005F047F80746002842D0284606F015FEAD
:1061C000064630B1431EEA5C2F2A02D100221E4649
:1061D000EA54DFF87480DFF87490DFF874A0384672
:1061E00005F05DF8834650B9384605F045F8041EC1
:1061F00022DB284605F806B009F0E4FFD6E70BF1EC
:10620000010B4146584606F0C9FD0028E7D0494633
:10621000584606F0C3FD0028E1D05B465246C6F55D
:106220008071A81905F041FA2846FFF7ADFF041E5A
:10623000D5DA384605F020F8204611B0BDE8F08FD9
:106240004FF0FF34F8E700BFD3131708E9B716087B
:106250008E3A1608F7B51F46137805460E46042BEE
:1062600026D1541C2046FFF7C5FE08BB2246314606
:106270002846FEF77FFB064602466B690D49284615
:1062800098470D4B32460D4928460097FEF7FEFA17
:10629000044638B90A4B3246084928460097FEF7AB
:1062A000F5FA0446304604F0D7FC204603B0F0BDB2
:1062B0000024FAE7D53E16081D600208845516082A
:1062C000556202082DE9F047054689461646002426
:1062D0004FF00108DFF844A0C84500DA14B12046A9
:1062E000BDE8F08756F828102846FDF7BDFE0746A2
:1062F00048B94FF0FF342B69326851462846984719
:1063000008F10108E8E7024631682846FEF7CEF9B1
:1063100004463846FDF7CCFEF2E700BF1D7C1708A7
:106320001346024A1968FEF7C1B900BFDA3E1608E3
:106330002DE9F04F95B0516804461546FDF794FEDF
:10634000814650B94FF0FF3623692A6820466A49D2
:106350009847304615B0BDE8F08F012109F09AFD4D
:10636000031E029312DA2D682669FBF71BF90068F9
:1063700006F07AFC614B00902A4661492046B047FE
:106380004FF0FF364846FDF793FEE2E7A968204646
:10639000FDF76AFE074650B94FF0FF3623692A68B9
:1063A000204655499847029809F0D7F9EAE705A928
:1063B00009F0E0FF064600283CD1079B03F4704338
:1063C000B3F5804F2CD13846FEF7A4FA686804F084
:1063D00079FF394602462046FEF7CCFA804640B99E
:1063E000236920462A68444998473846FDF760FEED
:1063F000D9E738464FF0260A4746FDF759FE494689
:10640000384606F0CBFCC0B9236920462A683D49CE
:106410009847B8F1000FE8D0404604F01DFCC2E7F1
:10642000B3F5004F14BF4FF0020A4FF0260A4FF0A9
:106430000008E4E74FF0260AF9E74FF4DB72514613
:10644000384609F027FD031E039328DA2D68D4F897
:1064500010A0FBF7A7F8006806F006FC274B009099
:106460002A4627492046D047D3E72D68FBF79AF8FC
:10647000006806F0F9FB244B00902A46204920468C
:10648000D84723E05A46514603980AF027F80028D7
:1064900022DBABEB000B8244BBF1000FF2DC04F11A
:1064A000280A4FF400720298514609F02DFDB0F110
:1064B000000B0CD0E6DAFBF775F80368D4F810B0DF
:1064C000042BD2D12A6820461049D847B3460398F6
:1064D0005E4609F042F99CE7FBF764F80368D4F8DC
:1064E00010B0042BEED02D68FBF75CF8006806F0C6
:1064F000BBFB074B0090C0E71D7C17089F391608AF
:10650000357C1708567D170847841608E47B170862
:106510005DC216082DE9F04F4FF0000993B0054613
:106520000E4690464F46DFF858A1DFF858B1524664
:106530004146304606F054FE421C044612D1B9F1E1
:10654000000F0BD106F059FE03680133B34221DA84
:106550002B69D8F80020424928469847204613B0B6
:10656000BDE8F08F6C2C0CD0732C10D0522C0BD0BB
:106570002B695946D8F8002028464FF00109984762
:10658000D5E747F00307D2E747F00407CFE747F026
:106590000107CCE706F031FE0368B3420CDBFDF7E0
:1065A00055FD01462846FDF75FFD064650B92B69AB
:1065B000D8F800202B49CFE706F01FFE036858F8F3
:1065C0002310EFE706F011FC00223044831B013B4F
:1065D000002B03DD10F8013C2F2B17D003A9304608
:1065E00009F0C8FE002814DAD8F800802F69FAF7FD
:1065F000D9FF006806F038FB1B4B009042461B4950
:106600002846B8473046FDF753FDA7E700F8012DAF
:10661000DCE7059B03F47043B3F5804F07D03B469E
:10662000002231462846FFF7F9FC0446EAE76B6989
:1066300032460F49284698470E4B32460E492846A7
:106640000097FEF723F904460028DBD17B07D9D554
:106650000A4B3246084928460097FEF717F9E4E747
:106660008C7C17081D7C1708D73A1608357C17084C
:10667000D53E16081D6002088455160855620208AA
:10668000E53E1608FB7C17082DE9F34706460D4644
:1066900014460027DFF8B48042462146284606F01B
:1066A0009FFDB0F1FF3F82463ED106F0A6FD036894
:1066B000AB4235DA06F0A1FD0368304654F82310EA
:1066C000FDF7D2FC054658B31D484FF02F084FF098
:1066D0000009002F18BF28462F2106F055FB04465D
:1066E00008B180F8009040F2FF11284609F09CFAAA
:1066F000B0F1000A1DDAFAF755FF0368112B00D13B
:10670000BFB93469FAF74EFF006806F0ADFA0D4BD9
:1067100000902A460C493046A0472846FDF7C8FCA1
:10672000504602B0BDE8F087BAF1700F08BF0127EC
:10673000B2E7002CF1D0204600F8018BCCE700BF77
:10674000E2E416085E3D1608357C1708DB411608A2
:106750002DE9F04FDFF830C18BB004460F461646E6
:1067600002AD4FF00008DFF82491DFF824A1DFF834
:106770000CB1BCE80F000FC59CE80F0085E80F00C6
:106780004A463146384606F02BFD431C05461CD1CF
:10679000B8F1000F15D106F030FD7B1E02689A4259
:1067A00042D106F02AFD0368204656F82310FDF773
:1067B0005BFC0746002841D1236932682B492046FB
:1067C000984728460BB0BDE8F08F462D07D0722DB4
:1067D0001FD03A2D236924D03268514614E006F0C8
:1067E00008FD006806F09DF8C0B28DF80900002889
:1067F000C6D00C38C0B2142803D81D4BC340DA07EA
:10680000BED4236932681B4920464FF001089847DF
:10681000B6E706F0EEFC006806F083F8ADF8180065
:10682000AEE732685946EFE706F0E7FC03683268E6
:10683000BB422369B4BF10491049C0E702A901F067
:1068400013F9051E0DDA3668D4F81080FAF7AAFE9F
:10685000006806F009FA0A4B0090324609492046C2
:10686000C0473846FDF724FCABE700BF1D7C170886
:1068700011001000DE7C17088C7C17082F7D17088C
:10688000703D1608357C17080C801708E93E16087D
:10689000FB7C17082DE9F743516804461546FDF7C0
:1068A000E3FB074650B94FF0FF3623692A682046BC
:1068B00017499847304603B0BDE8F083A9682046E1
:1068C000FDF7D2FB804650B94FF0FF3623692A68A6
:1068D00020460F4998473846FDF7EAFBEAE70146AC
:1068E000384609F01FFB061E0DDA2D68D4F810900B
:1068F000FAF758FE006806F0B7F9064B00902A46F2
:1069000005492046C8474046FDF7D2FBE3E700BFF4
:106910001D7C1708EF3E1608357C17082DE9F0415D
:106920005568C2B006461B492846174606F036FA97
:10693000044600B9BD6829463046FDF795FB05467B
:1069400020B304BB01464FF4807202A806F039FA66
:1069500002A8FFF719FC002804460DDA3F68D6F8B4
:106960001080FAF71FFE006806F07EF90A4B0090CF
:106970003A460A493046C0472846FDF799FB20466B
:1069800042B0BDE8F08109F073FDE4E74FF0FF3459
:10699000F5E700BFF63E1608DC3A1608357C170806
:1069A0002DE9F341516806461746FDF75DFB0546A4
:1069B000C0B109F007FC041E0DDA3F68D6F810805C
:1069C000FAF7F0FD006806F04FF9084B00903A46E0
:1069D00007493046C0472846FDF76AFB204602B00B
:1069E000BDE8F0814FF0FF34F8E700BF4B3E1608DA
:1069F000357C1708D2E90012FDF774BA2DE9F04F83
:106A000013788DB00446042B089140F0C0811146E4
:106A100002F1280011F8013F2BB1303B092B00F2A5
:106A2000B6818142F6D10023571CAF490BA80B93C6
:106A30003B46089A04F02CFE002802DB0B9A002A41
:106A40004FD12569FAF7AEFD006806F00DF9A74BA6
:106A500000902046A64AA749A847A74EB046B3468D
:106A6000B24607960696CDE9046663693A46A3499D
:106A7000204698476369049A2046A0499847069B98
:106A800042469F49CDF80CA02046CDE901B3059BB5
:106A90000093079B6569A8476369324699490025B9
:106AA000204698473B46089A0BA897490B9504F057
:106AB000EFFDA84203DB0B9A002A40F0A280256973
:106AC000FAF770FD006806F0CFF8884B009020467A
:106AD000874A8849A847002384F8283000252E4695
:106AE000C0E04FF4007104F1280920464B460091A4
:106AF0007F49FDF777FE05460B9804F0ADF8002DB1
:106B0000ABDB7D4EB046B346B24607960696CDE95E
:106B1000046609F101010D4611F8012B0A2A00F063
:106B20003B81002AF7D1154605227849484606F0F0
:106B3000D0F840B909F10C00FDF7FEFE0590002DDC
:106B400093D0A946E5E706227149484606F0C1F808
:106B500028B909F10C00FDF7EFFE0490EFE70622DB
:106B60006C49484606F0B5F888B9099009F10C005F
:106B7000FDF7E2FE2C21069006F006F90028DED093
:106B8000099A00F8012BFDF7D7FE8246D7E70622C7
:106B90006149484606F09DF828B909F10C00FDF757
:106BA000CBFE8346CBE709225C49484606F091F8C4
:106BB00070B909F10C00FDF7BFFE80460246114690
:106BC00001320B78303B092BF9D900230B70B6E763
:106BD0000A225349484606F07CF828B909F1120008
:106BE000FDF7AAFE0790AAE708224E49484606F09C
:106BF00070F80028A3D109F10C00FDF79DFE0646B0
:106C00009DE74FF4007104F1280A20465346009195
:106C10003749FDF7E7FD06460B9804F01DF8002EF6
:106C2000FFF65CAF2E46A946DFF80CB10AF1010170
:106C3000884611F8012B0A2A00F0AB80002AF7D110
:106C400090460A223849504606F043F8024600288A
:106C500074D101460AF10C0005F0A1FE0646B8F118
:106C6000000F3ED163693246304920469847636938
:106C70002A462E492046984736B1002D6DD04FF454
:106C80007A736B43B3FBF6F60A23B6F5487F656962
:106C9000204634BF20212121B6FBF3F2009103FBF3
:106CA00012632349A8470023089A0BA80B933B467D
:106CB000204904F0EDFC002802DB0B9A002A4ED19B
:106CC0002569FAF76FFC006805F0CEFF074B0090CE
:106CD0002046074A0749A8474FF0FF300DB0BDE8EE
:106CE000F08FC246A2E700BFF93E1608063F16081D
:106CF00052711708357C1708E2E416080F3F160892
:106D0000143F1608313F1608373F160875801708DC
:106D10006E8017086780170860801708568017086C
:106D20004B8017084280170837801708433F160822
:106D30004A3F1608583F16082C8017080A22594661
:106D4000504605F0C6FF0246002888D101460AF1E8
:106D50000C0005F024FE054681E72E4694E74FF42B
:106D6000007304F128060E49204600933346FDF7D0
:106D700039FD05460B9803F06FFF002DACDB304664
:106D80006569FDF7D9FD074902462046A84700205E
:106D9000A4E708F8019B54E7002205F8012BC3E69D
:106DA000527117088C61170873B516460446002205
:106DB00001A9706805F0B9FD054628B1019B72680C
:106DC0009A4201D01B7843B12369204632680649B4
:106DD00098474FF0FF3002B070BD02466369034927
:106DE00020469847A847F6E7FB7C1708663F160839
:106DF00030B51F4D044685B0436929461D4A984762
:106E0000636929461C4A204698471C4B1C4A204669
:106E100003931C4B1C4902931C4B01931C4B009386
:106E20001C4B6569A8471C4D636920461B4A1C49D9
:106E30009847636929461B4A204698476369294653
:106E4000194A204698476369184A204618499847C6
:106E50006369184A2046184998470023174A204674
:106E600000931749174BFDF711FD05B030BD00BF6A
:106E70000F3F1608723F1608763F1608873F160820
:106E8000833F1608FBD11608143F16088D3F1608DD
:106E9000FA8B16087C3F1608993F1608913F160892
:106EA000313F1608CA58170884B016089E3F1608C6
:106EB000A53F1608AA3F16088C611708463A16081F
:106EC00052711708FD69020803297FB5054614466B
:106ED00018D1506803782D2B0ED14378303B092B05
:106EE0000AD8002203A9013005F01FFD0646A0685C
:106EF0000378303B092B0DD92B69284622681849A5
:106F0000984729E00229F7D150680378303B092BD4
:106F1000F2D80C2603A9002205F007FD31460FF038
:106F200093FAD8B1FAF73EFB03682E69032B0CD015
:106F3000162BE1D02468FAF735FB006805F094FEC3
:106F4000084B22460849009004E0A36807490093D3
:106F5000074B22682846B0474FF0FF3004B070BDA1
:106F6000FB7C1708353D1608357C1708A97C1708E7
:106F7000B5C3160873B515460646002201A9686810
:106F800005F0D3FC28B1019B6A689A4201D01C78B5
:106F900044B1336930462A68044998474FF0FF30BE
:106FA00002B070BD06F02EF92046F9E7FB7C170809
:106FB00073B515460646002201A9686805F0B5FCC0
:106FC00028B1019B6A689A4201D01C7844B13369A8
:106FD00030462A68044998474FF0FF3002B070BD30
:106FE00006F02CF92046F9E7FB7C17081346024A05
:106FF0001968FDF75BBB00BFB23F1608F0B587B05C
:1070000004460120164602A9FCF7E0FC002811DA2C
:1070100036682569FAF7C6FA006805F025FE214BA7
:107020000090324620492046A8474FF0FF352846B9
:1070300007B0F0BD71682046B4F82872FEF79EFDD7
:10704000051E14DB04A90120FCF7C0FC051E11DAA3
:1070500036682569FAF7A6FA006805F005FE114BB7
:107060000090324610492046A8474FF0FF35A4F85B
:107070002872DCE705980399029B8142049A6669AD
:10708000A2EB0302C2BF094B1B1802F1FF322046DC
:10709000C8BF0593059B5B1A0549B3FBF1F305498E
:1070A000B047E4E7C03F1608357C170800CA9A3B92
:1070B000A0860100CE3F16082DE9F0474FF00008EA
:1070C000A4B00446894616464746DFF82CA252462D
:1070D0003146484606F084F8431C054640F08F8050
:1070E00006F08BF803684B45C0F2EC803668002F41
:1070F00000F09C802C22002110A8FAF7DCF903AAEA
:107100007149384605F001FE8146002800F085806F
:10711000DFF8E8A10027032249465AF8040B05F0DE
:10712000BDFD20B101370C2FF5D14FF0FF3714977B
:10713000013772D003AA6449002005F0E6FD00285B
:107140006BD00A22002105F0F0FB431E1E2B64D8F1
:10715000139003AA5D49002005F0D7FD00285CD0FC
:107160000A22002105F0E1FB172856D8129003AA45
:107170005649002005F0C9FD00284ED00A22002102
:1071800005F0D3FB3B2848D8119003AA4F490020B3
:1071900005F0BBFD002840D00A22002105F0C5FB08
:1071A0003D283AD8109003AA4749002005F0ADFDCC
:1071B000002832D00A22002105F0B7FBA0F26C7043
:1071C000C8282AD8159010A8B8F1000F22D005F0D1
:1071D0005BFF0027059005A9384606970EF01CFEB8
:1071E000B84265DA2769FAF7DDF9006805F03CFD79
:1071F000374B0090324637492046B84712E0732D8E
:1072000003D105F0F6FF076861E7752D52D14FF005
:1072100001085CE705F04DFFDBE7236932462E49A4
:1072200020469847284624B0BDE8F08703A9384691
:10723000FCF7CCFB002808DA2769FAF7B3F90068F5
:1072400005F012FD254B0090D4E705A903A8B8F17D
:10725000000F0BD005F030FFA0B92769FAF7A2F9AB
:10726000006805F001FD1E4B0090C3E705F0B6FF76
:1072700040B92769FAF796F9006805F0F5FC194B53
:107280000090B7E705AB184A502110A805F0F2FDB1
:10729000002808DA2769FAF785F9006805F0E4FCA8
:1072A000124B0090A6E7636910AA1149204698473F
:1072B0000025B7E708492369204632684FF0FF35BB
:1072C0009847AFE70B49F6E70E2C1708E23F160880
:1072D000E63F1608357C1708FB7C1708C03F1608E8
:1072E000F43F1608FD3F1608094016081F4016080F
:1072F0008C6117088C7C1708DE3F16087C80170805
:107300002DE9FF4114460E461F460546FAF772FB6B
:1073100021460A9B3A46304600F048FB041E06DA36
:10732000FAF778FB4FF0FF3004B0BDE8F08195F834
:107330002832002B3BD195F8887203934FB10EF0A1
:1073400027FF22464FF48C71D0F83C0108F012FC64
:1073500007462046042203A90FF010F8041E1FDA86
:10736000FAF720F900680A281FD0D5F8108005F038
:107370007BFC164B3246009028461549C04795F8CD
:10738000883243B13FB90EF003FF40F21911D0F833
:107390003C0108F0EFFBFAF73DFB44EAE470C3E779
:1073A000039C003C18BF0124E9E70024E7E703A998
:1073B0000EF048FF039B32460649009328462346B9
:1073C0006F69B847FAF726FB0020ADE7584016086A
:1073D000357C1708B13A1608012938B504461568F6
:1073E0000BDD0749506805F0D9FC30B9054A29463C
:1073F0002046BDE83840FDF759B9034AF7E700BF1A
:10740000033A1608604016086F40160801292DE956
:10741000F04F044685B08846164634DC4E4A316843
:1074200005B0BDE8F04FFDF741B96F2F1FD0742FA5
:1074300005D03A2F23691FD0326859461EE005F067
:10744000D8FED0F800A0454A3146404605F0C8FEB7
:10745000431C0746E9D1B9F1000F40D105F0CDFE3C
:107460000368434518DB236932683D4935E005F080
:10747000C0FE03680393E6E73268294620464FF0D2
:1074800001099847DFE74FF00009DFF8E4B0344D19
:10749000CA46CDF80C90D6E705F0AFFE036856F863
:1074A000235005F0AAFE03680133036005F0A5FE32
:1074B0000368434517DA05F0A0FE036856F823B0C9
:1074C00005F09BFE03680133036005F096FE036838
:1074D00043450ADA236932682249204698473846EC
:1074E00005B0BDE8F08FAB464D46BAF1000FBAD0FB
:1074F00035B129462046FCF7B7FD05460028EED0F9
:1075000059462046FCF7B0FD8046C8B1039B0146B2
:10751000524628460093002309F0C2FA071E0DDAEE
:107520003668D4F81090FAF73DF8006805F09CFB37
:107530000D4B009032460D492046C84715B907E06B
:10754000002DCCD02846FCF7B3FDB8F1000FC6D013
:107550004046FCF7ADFDC2E77F4016088E40160896
:107560002F7D17088C7C170888401608357C170873
:10757000FB7C17082DE9F341516806461746FCF7D6
:1075800073FD0546C8B1002109F002FB041E0DDAA7
:107590003F68D6F81080FAF705F8006805F064FB3C
:1075A000074B00903A4607493046C0472846FCF74B
:1075B0007FFD204602B0BDE8F0814FF0FF34F8E7D0
:1075C000A03E1608357C17082DE9F3470446884687
:1075D00091460126DFF8BCA0464503DB002002B03F
:1075E000BDE8F08759F8262013785C2B43D15378F7
:1075F0006E3B0A2B20D8DFE803F0331F1F1F381F14
:107600003B1F1F1F0600971C00211022384605F063
:10761000C6F90A210546384605F001FC06280DDDAD
:107620002B0E1649EAB220460193C5F30743009397
:10763000C5F307236769B8470136CDE7022807DDA0
:107640006769C5F30723EAB20D492046B847F3E757
:107650000028F1DD6369EAB20A4920469847EBE762
:107660006369094920469847E6E763690749F9E7EE
:1076700063690749F6E763695146EEE794401608E7
:1076800098401608C45F1708662417089D4016081E
:10769000E1E41608348C16082DE9F04F804691B0CD
:1076A0000D461446DFF8B8B226689649304605F014
:1076B00075FB78B9012D40F31C81221D691E4046DF
:1076C000FFF7EAFFB0FA80F676097642304611B04D
:1076D000BDE8F08F33782D2B40F09280012D40F3E0
:1076E00008818949304605F059FB6768D0B93B7875
:1076F00003B34FF0020900264D45E7DD54F829A0F9
:107700004FEA89078149504605F048FB002840F0C0
:10771000E780002E40F0F38009F101030437ED1AF1
:107720003C44C1E77A49304605F038FB38B93B782C
:10773000002BDED04FF002094FF0FF36DCE7394670
:107740004046FCF791FC06460028F3D001A908F05A
:1077500011FE07463046FCF7ABFC002FEAD1266845
:107760006C49304605F01AFB30B9039B03F47043B3
:10777000B3F5C04FDED1BCE76749304605F00EFBDC
:1077800028B9039B03F47043B3F5005FF2E7634944
:10779000304605F003FB28B9039B03F47043B3F5AF
:1077A000804FE7E75E49304605F0F8FA0028A0D0A0
:1077B0005C49304605F0F2FA28B9039B03F47043A4
:1077C000B3F5004FD6E75849304605F0E7FA20B93F
:1077D000039B13F4927F8CD1ACE75449304605F0FB
:1077E000DDFA18B9079B002B83DCA3E7504930462C
:1077F00005F0D4FA00287CD1039B13F0920FEAE73E
:10780000022D76DD67684B49384605F0C7FA20B18E
:107810005946384605F0C2FA38B9A168304605F035
:10782000BDFA68B94FF0030965E74349384605F0EA
:10783000B5FA40B9A168304605F0B0FA0028F1D198
:107840004FF0030978E7002201A9304605F06DF8F2
:10785000236807461B78002B4BD0019B1A78002A1F
:1078600047D101A9A06805F060F8A36806461B7817
:10787000002B3ED0019B1B78002B3AD1D4F804900A
:107880002E49484605F08AFA10B9B742D8D1C9E75F
:107890002B49484605F082FA10B9B742C2DACFE761
:1078A0002849484605F07AFA10B9B742BADCC7E76A
:1078B0002549484605F072FA10B9B742B2DDBFE774
:1078C0002249484605F06AFA10B9B742AADBB7E781
:1078D0001F49484605F062FA58B9B742A2D1AFE74E
:1078E0001C49504605F05AFA18B9002E7FF414AF1F
:1078F000ECE6D8F810304046174A184998474FF040
:10790000FF36E3E6A64D17089F401608D24016083A
:10791000A2401608A54016082E3A16081E3B160867
:10792000A8401608AB401608F63E1608AE401608EA
:10793000B1401608B8401608B7401608BA401608F5
:10794000BE401608C2401608C6401608CA401608AF
:10795000CE401608D540160842801608567D1708F6
:10796000B440160804320139FFF796BE01F1804396
:10797000013B70B504460E4652F8230015460949EE
:1079800005F00CFA30B92A1DB11E2046BDE8704042
:10799000FFF782BE236920462A68034998474FF0C3
:1079A000FF3070BD68E91608567D17082DE9F041D3
:1079B00088B00E461746984603F0FBFB002806DA0F
:1079C0000224F9F7EFFD04604FF0FF3434E003F0D8
:1079D00003FC05460028F3D004A803F01BFE044670
:1079E0000028EED102A803F011FE04460028E8D1D9
:1079F0006B6803A904A8039303F02CFE044658BB4C
:107A0000A96804A803F02AFE044628BB042104A8A0
:107A100003F01DFE0446F8B997B92868E968FEB975
:107A2000002302AACDE9006304AB0EF05DFE041E44
:107A300018DB02A803F0DFFD204608B0BDE8F081A6
:107A40004FF4D2733A46012102A80093434603F053
:107A5000AFFD04460028E0D002A803F0CCFDB0E75B
:107A60000436DDE76442F7E730B599B004460D46C9
:107A70002822002103A8F9F71EFD01A90020FBF729
:107A8000A5FF00B30023069303216B7820468DF8F1
:107A9000153008F0FFF90028039038DAF9F782FD75
:107AA000046864420A9820B107992BF17FF90023FA
:107AB0000A93002C75DA6442F9F774FD04604FF004
:107AC000FF3019B030BD0DA901A805F0F5FA002866
:107AD000D8D012994F29D5DD109A50390D9B02F05C
:107AE0001F020F98C3F3440342EA41221199013166
:107AF000490101F4F0710A430E99490101F4FC6156
:107B000041EAC0210B439BB243EA0243BBE70DAA03
:107B100040F20C5108F02EF8041E1DDB9DF83430A5
:107B20001BB39DF8363003B3EA690E9B22B19A422B
:107B300003D96FF015040FE0EB61BDF93C30B3F5EC
:107B4000006F079314D00BDCB3F5007F25D0B3F59D
:107B5000806F24D04FF0FF34039807F0FEFDA1E7BB
:107B6000B3F5805FF6D10C2303E06FF01204F3E766
:107B70000B2303A928468DF8133000F015F8041ED6
:107B8000EADB07982BF110F90A900028E4D003A94A
:107B9000284600F0B7FA0446DEE70923E9E70A239E
:107BA000E7E700208DE7FFEC2DE9F04F038A95B061
:107BB00005460C4613B94FF4007303822C220021B2
:107BC00008A8F9F778FC6B8A002B7FD0012B00F016
:107BD000828000930293637A202B0ED023692A8A35
:107BE000013B029903EB4213E279D3402372DBB2EB
:107BF000EA69521AD31A0C930893AB78FF2B0393BC
:107C00000AD1EB69B3F5006F68D3B3F5805F6BD22F
:107C10000123AB7007230393089B4FF000080593E3
:107C200003EB43034746CDF8048006930C9B049373
:107C30000233079394F809A0BAF1000F02D0BAF109
:107C40000C0F62D195F802B04FF0010C22690321AC
:107C50000BF101030BF102002E789A400CFA00F0B0
:107C60000CFA03F34FF0000C11FB06221844069B9C
:107C70001844531E4CF1FF31C018634641F1000116
:107C80000FF0C8FD814600283AD0059B42F6D2721B
:107C900000FB1636E379013326FA0BF600FA03F3FC
:107CA000934206F1020296BF03214FF47F63B3FBB8
:107CB000F1F39A4226D801230193BAF1000F28D09C
:107CC000002E00F09B800020034662E00123029317
:107CD000202300937FE702930223FAE7002398E72B
:107CE000022396E7032394E7B3F5005FF8D3B3F5D7
:107CF000804FF7D3B3F5004F2CBF0523042388E74B
:107D00000646D8E70026B146D5E7BAF1100F75D17F
:107D1000002695F802B022692F78BBF1000F29D117
:107D200007EB5202079810184FF0000343F10001CF
:107D3000013861F100010FF06DFD002800F0DB80DB
:107D4000E2794FF6F071049B013A07FB103700FA15
:107D500002F227FA0BF38A4228BF0A46991C8A428C
:107D6000C0F0C780B3F57F6F00F2BE804FF001080E
:107D70004746A5E70BF1FF330BF101009A400123C1
:107D800003FA00F0049B3A441844CCE74FF0010892
:107D90004746B8F1000F00D00E9307B10D90019B3C
:107DA0000BB1CDF82490BDF80830BAF1000F1DD00A
:107DB000BAF1100F1DD110220D9862720E9AA261B5
:107DC00060616B82EB2323719023A3714B4B636241
:107DD00081236381637A202B6BD03C2363715B2307
:107DE00084F82030637A00206B705FE00E9AB24214
:107DF000E1D80C220998A6616272E1E7BAF1200F7E
:107E0000AE784AD1009AEB6995F800B09B1A01222E
:107E100002FA06FA2269A3EB0A0AB6B90BEB920240
:107E200031460AF1030010184FF0000341F1000140
:107E3000013861F100010FF0EDFCC8B92023637235
:107E4000129BA361BDF80030BAE7012E05D10BEB00
:107E5000520200210AF10600E5E7B11E701C4FF046
:107E6000010C8A4000210CFA00F05A441844DAE769
:107E7000E2790BFB10AA2249023A2AFA06F300FA29
:107E800002F28A4228BF0A46D91C8A4205D34FF61D
:107E9000F372934201D91293D0E70136039BF6B2F5
:107EA0009E42AE707FF6C6AE6FF0160015B0BDE80C
:107EB000F08F58236371772384F820300123AA7848
:107EC000934000222372E9896B8A01292A8201D911
:107ED0008B4287D8012BEA8184D9013B9BB2062BC8
:107EE00088BF0623EB817DE7002E7FF44FAF0E9312
:107EF00054E74FF001080127E2E600BFAC80170805
:107F0000F0FFFF0F38B50C4605460A690021E0690D
:107F1000F9F7D1FAE369A28860491A80A2799A70C8
:107F2000E069033004F045FFE3692269DA722369EE
:107F3000E2691B0A13730123A978E2698B4053732A
:107F4000E3696A8ADA81E3692A781A74E3692A8A1A
:107F50005A742B8AE2691B0A9374EB69E269B3F5E0
:107F6000803F3FBFD374AB8BE2691B0A2CBF136207
:107F70001375F822E3695A753F22E3691A83FF22D9
:107F8000E3695A83E3696A69DA616B78E269202BF5
:107F9000616905F1030340D0D1822921E26982F8A9
:107FA0002610E269A96982F82710AA69E169120A14
:107FB00081F82820E269698B82F82910E269E97E5C
:107FC00082F82A10E269D5F80310C2F82B1059681C
:107FD000C2F82F101989A2F833109B7A82F8353035
:107FE0006B780C2BE3690CBF2D492E490A68C3F846
:107FF00036204A68C3F83A20E06962893E30616AF7
:10800000F9F7EEF8E36994F8202083F84120E3695A
:108010004AF65522A3F8FE2138BD51620221E269D9
:10802000D1620121E2691186E269E989518629213B
:10803000E26982F84210E269A96982F84310AA69EC
:10804000E169120A81F84420E269698B82F84510DF
:10805000E269E97E82F84610E269D5F80310C2F8B9
:1080600047105968C2F84B101989A2F84F100E49F1
:108070009B7A82F85130E2690B68C2F852304B6843
:10808000C2F85630E0696289616A5A30F9F7A8F897
:10809000E36994F8202083F85D20B8E7D8401608FB
:1080A000E1401608EA401608F340160838B5151ED8
:1080B0000C4620DBC369AB421DD9CB790022206876
:1080C0009D40294607F0A3FD431C04D1F9F76AFA45
:1080D0000068404238BD854210D12269E1692068BC
:1080E00008F0FCF90028F1DB2369834214BF6FF02C
:1080F0003C000020EEE76FF01C00EBE76FF015008E
:10810000E8E7FFEC2DE9F84F0C4606460127FFF79C
:10811000F9FE002221463046FFF7C8FF22690546D6
:108120000021E069F9F7C7F9738A9F420CDA002D44
:1081300002DA2846BDE8F88F3A4621463046013734
:10814000FFF7B4FF0546EFE7002DF2DB7378202B35
:1081500013D0B6F812A04FF000094FF0F80B3378A7
:10816000994579DB62694FF00008B6F81290F71C68
:10817000DFF864A102FB0399A2E0F38923BB226923
:108180000021E069F9F797F9E369514A2146304641
:108190001A6002F1FF52E36902F500522032C3F87F
:1081A000E421D4E90632013BC2F8E8310222E36956
:1081B000C3F8EC21474AE369C3F8FC210122FFF729
:1081C00075FF051EB5DBC4E721463046FFF79AFE72
:1081D000F28921463046FFF769FF051EA9DBCEE78D
:1081E00022690021E069F9F766F907BB226939467F
:1081F000E069F9F760F97278E3690C2A10D0102A67
:1082000027D0C3F800806FF07F42C3F80480E36991
:1082100083F808B0E369A3F8092083F80B8003E032
:108220006FF07F421A809A70E36983F800B02A46A3
:1082300021463046FFF73AFF051EFFF67AAF0137B9
:1082400063690AEB0705BB42CAD809F10109AA46CE
:1082500085E7C3F80080E7E700274FF0FF38EFE736
:1082600022690021E069F9F726F9B8F1000F1DD164
:108270000B225146384604F070FD40B13A68E3697C
:108280001A607A685A603A891A81BA7A9A72E369EE
:108290000822DA72E369E268DA81E369E268DA8285
:1082A000E369E2891A82E369E2891A832A46214650
:1082B0003046FFF7FBFE051EFFF63BAF08F1010855
:1082C000237A08EB09059845CADB002531E700BF92
:1082D00052526141000055AAFC401608044B1B682D
:1082E0000360C3F1105303F500230B60704700BF18
:1082F0007036160808B54FF490214FF0405002F048
:10830000A3FC0748C0F1605101F5803102F09CFCEC
:108310004FF400314FF00050BDE8084002F094BC2B
:108320000000003810B5D0F88C4001F4D873A0F8E4
:108330007410226822F4D87213432360D0F88C2082
:10834000936861F30003936010BD10B5EFF31184DF
:1083500000238022EFF3108372B682F3118883F337
:108360001088FFF7DFFFE4B284F3118810BD10B569
:10837000EFF3118400238022EFF3108372B682F3AF
:10838000118883F3108849B1D0F88C201368926863
:1083900003F4D87302F0010213430B800021E4B20E
:1083A000FFF7C0FF84F3118810BDFFECF0B5036E3A
:1083B000EFF3118000228021EFF3108272B681F377
:1083C000118882F31088D3F88C20156825F00101FC
:1083D00005F001041160D3F88060D3F8887072084A
:1083E00002EB4702B2FBF6F2642A41D9013225F4CE
:1083F0000041520821F00101D3F88C502960D3F8D4
:108400008C50EA60264A0A4093F87A10012939D143
:1084100042F4C06293F87B50092D02D0082D36D16A
:10842000A9B342F48052D3F88C100A60D3F88C6060
:1084300093F87C107568494225F4405501F40051C9
:1084400029437160D3F88C5093F87E60A96821F4B9
:10845000407126B1D3F89C600EB141F40071A9605F
:108460002243D3F88C30C0B21A6080F31188F0BD7B
:10847000C2F3420522F00F0241F400411204120C33
:108480002A43B9E7022908BF42F48062C2E7B3F881
:108490007A10B1F5E06F08BF42F08052C3E700BF29
:1084A000FEE9FFEF036ED3F88C20506AB3F8762014
:1084B00040EA0242C0B20A600022A3F87620704768
:1084C00010B5006EEFF3118400238022EFF31083C8
:1084D00072B682F3118883F31088B0F8743039B122
:1084E00043F02001E4B2FFF730FF84F3118810BDA0
:1084F00023F4907121F00101F4E7036ED3F88C307E
:10850000D869C0F340107047036ED3F88C3099627D
:10851000704710B5006EEFF3118400238022EFF353
:10852000108372B682F3118883F31088B0F8743028
:1085300041B143EA020189B2E4B2FFF706FF84F3D6
:10854000118810BD23F08001F5E7036ED3F88C305D
:10855000D869C0F3C010704708B5036E114693F890
:108560007D2022B1D3F8980008B1F8F711FB002064
:1085700008BDF8B50346B1F5887F10469B685D6974
:108580002C6E00F0288110DCB1F5817F00F0CC80EA
:1085900040F20F13994200F0FC8040F2011399421F
:1085A00000F09F806FF018007FE040F23313994293
:1085B00053D040F23513994278D0B1F5987FF1D17C
:1085C000EFF3118600238022EFF3108372B682F35B
:1085D000118883F31088D4F88C3010F0010F1F68D5
:1085E00027F001021A60D4F88C30D4F890209D68EE
:1085F0002AD000F0060180F0080045F00805A1F13E
:10860000020CA1F1040EC0F3C000DCF1000343EB47
:108610000C03DEF100014FEA034341EB0E0143EA94
:10862000402322F4403043EA414320F400701843D1
:10863000F8F7C2FAD4F88C309D60D4F88C301F6003
:10864000F6B286F311882FE022F4403025F00805B9
:1086500020F40070F8F7B0FAECE7EFF31182002392
:108660008021EFF3108372B681F3118883F31088B1
:10867000D4F88C30C607196821F001051D60D4F8C4
:108680008C506B684CBF43F4803323F480338007F5
:108690004CBF43F4003323F400336B60D2B2D4F800
:1086A0008C30196082F311880020F8BDEFF311823D
:1086B00000238021EFF3108372B681F3118883F3D6
:1086C0001088D4F88C300128196821F001051D604C
:1086D000D4F88C506B680CBF43F4004323F4004380
:1086E000DBE7002A00F0918094F87A20D2B1511E85
:1086F0004A424A4151024FF4807294F87C3094F817
:108700007E509B0143EA45730B43134394F87D204D
:1087100043EAC27343F030038360D4F8801004F05E
:108720008BFBC1E71146E8E7002A6ED0936803F09F
:108730003002302A69D19A0003D5D4F89C20002A4F
:1087400063D0002B03DAD4F89820002A5DD013F40C
:1087500080721CD013F4007F0CBF0223012384F825
:108760007A308368C3F3801384F87C308368C3F362
:10877000407384F87E308368DB0F84F87D3004F02A
:1087800077FBC4F880002846FFF710FE8CE71346FD
:10879000E5E7EFF3118600238022EFF3108372B632
:1087A00082F3118883F31088B4F8743028460021CE
:1087B0006FEA43436FEA5343A4F87430FFF7A9FE0E
:1087C000D4F8900020F4402020F4807040F4802001
:1087D000F8F7F2F934E7EFF3118600238022EFF384
:1087E000108372B682F3118883F31088D4F8900056
:1087F000F8F7E2F9B4F8743001212846C3F30E0308
:10880000A4F87430FFF785FE1AE76FF015004CE707
:1088100010B5046E94F88400F8F72CFB002294F84D
:1088200084001146BDE81040F8F7F8BF38B5056E72
:1088300006492A4695F88400F8F7F0FF044618B96F
:1088400095F88400F8F72AFB204638BD51880208C5
:1088500010B51446D2F88C20D3699BB29806A4F8C0
:10886000763013D5B4F8741089060FD5204605F07C
:1088700069FEB4F876301A0606D5B4F874301B06D3
:1088800002D5204605F028FE002010BD13F00E0F83
:10889000EFD00E231362ECE7036E0A461E49D3F8AD
:1088A0008C308B4220D00CD8A1F540518B421FD088
:1088B00001F580618B421FD0A1F500618B421FD072
:1088C000704716498B421FD001F580618B421ED044
:1088D000A1F518418B421DD111484FF000410AB15A
:1088E0000A460021F7F782BF0D484FF08041F6E7B6
:1088F0000B484FF48021F2E709484FF40021EEE7DE
:1089000007484FF40031EAE706481021E7E7054839
:108910002021E4E7704700BF0078004000100140CC
:10892000E8440258F044025870B50026046E05462B
:108930003146204684F87860FFF719FD3146284615
:10894000FFF7AAFFD4F88C20136823F00D031360FF
:10895000D4F89000F8F718FAD4F89400F8F714FA5D
:10896000D4F89C0008B1F8F70FFAD4F8980018B1C1
:10897000BDE87040F8F708BA70BDFFEC38B5046E7A
:10898000002201210546D4F88C301A60FFF784FFDD
:10899000D4F89000F8F710F9D4F89400F8F70CF92F
:1089A000D4F89C0008B1F8F707F9D4F8980028B17A
:1089B00020F4402040F48020F8F7FEF8D4F88C1022
:1089C000284694F87C304A685B4222F47D5203F4D6
:1089D000005313434B60D4F88C20104B11680B40AC
:1089E0001360D4F88C2094F87910936823F4E06332
:1089F00023F0010343EA41639360FFF7D7FCD4F807
:108A00008C200020136843F0005343F00D031360E3
:108A10000123A4F8740084F8783038BD03BEFF3316
:108A20007FB50D490D4805F091FB0D4968460D4D88
:108A300004F0BFF900231C4655F8041B39B15E1C35
:108A4000303368468DF8093005F080FB3346013439
:108A5000082CF1D104B070BD88010024084116082B
:108A6000154116083081170813B504460DF10601AB
:108A70000948FFF77CFC0A2C02D10D20F7F7E2FD34
:108A8000E0B2F7F7DFFDBDF806100348FFF75DFC25
:108A9000204602B010BD00BF8801002408B50DF0CB
:108AA0007FFC002008BDFFEC10B5084B4FF0E02420
:108AB0000022074963610F20A261F8F7AFFE072388
:108AC0000F202361BDE81040F8F7E8B9FF52070016
:108AD0009D8A02080C4A82B0D36813F0400302D08A
:108AE000002002B070478021D1600193019BB3F553
:108AF000803F02D36FF07300F3E7D3685B06EFD4D7
:108B0000019B0133F1E700BF004000580023092812
:108B100002DC40EA0310704701330A38F7E7FFEC44
:108B200008B50120F7F7D6FD024BCA225A6253223C
:108B30005A6208BD0040005813B5FFF7F1FF0E4B15
:108B4000DA6822F02002DA6000220192019AB2F57E
:108B5000003F09D36FF07304FF2200205A62F7F739
:108B6000B9FD204602B010BDDA68920602D4019A1F
:108B70000132EAE70024EFE7004000583D4B0120B6
:108B80002DE9F0413C4E5F6DF7F7A4FDB7424AD0A6
:108B90003A4B9F4247D04FF4803200213848F7F7D4
:108BA00025FE00224FF480313548F7F71FFE4FF4C1
:108BB000407233481146F7F719FE4FF40042002186
:108BC0002F48F7F713FE0025FFF7B6FF044610B154
:108BD00001350A2DF8D1B7421AD0284B9F4217D041
:108BE000FFF79EFFFFF776FF044650B9214B9A68C6
:108BF00022F040029A60234A1A61DA6822F0800269
:108C0000DA601C4FFF2300207B62F7F763FD7E656F
:108C10000020F7F75FFD04B145BB1B4B012200208C
:108C20001A70BDE8F081194BD3F8703403F4407327
:108C3000B3F5407FC7D00F4C4FF48032002110486D
:108C4000D4F800806568F7F7D1FD00224FF4803139
:108C50000B48F7F7CBFD4FF4407209481146F7F780
:108C6000C5FDC4F8008065606665A6E76FF0730017
:108C7000D7E700BF00400058EDFECEFACEFA0DF067
:108C8000704402583F1F7C00454E002400400258AB
:108C90002DE9F84306460D46324F7B683A68BC6AB8
:108CA00039688A42F9D179688B42F6D10A21C2F338
:108CB000021C02F00F0003F00F0943F3003801FB20
:108CC0000C00C2F3023C08EA01083060C2F3032042
:108CD00001FB0C007060C2F30150C2F3034201FBC0
:108CE0000022C3F30340B260C3F3011201FB0299F7
:108CF000C3F303229044C3F30352C3F34233C6F8D1
:108D00000C9001FB020008F1FF3800F16402C6F884
:108D1000108000F5FA6072610722B3FBF2F2C2EB39
:108D2000C2029B1AB36104F099F9011E404618BFB4
:108D3000012104F087F9002348443362F0613A6965
:108D400065B1C2F30E02A3B20749D31A01324B43F5
:108D5000B3FBF2F342F2107253432B600020BDE8E4
:108D6000F88300BF00400058A0860100FFF790BFC5
:108D70002DE9F84F85690769D0E90089D0E902A695
:108D8000002D4FD06D03ADB2D0F814B0FFF7C8FE80
:108D9000FFF7A0FE044688BB5046FFF7B7FE024629
:108DA00048461204FFF7B2FE42EA00224046FFF7AF
:108DB000ADFE10431D4A00F07F3020F0FE401060F1
:108DC000ABF16400FFF7A2FE0446781CFFF79EFE9D
:108DD00001463046FFF79AFE40EA050343EA0443A2
:108DE00043EA012323F07F4323F0C0035360D36899
:108DF00023F08003D360FFF79FFE04460B4D0C4E1B
:108E00006B6DB34206D00120F7F764FC00206E655D
:108E1000F7F760FCFF2300206B62F7F75BFC20464E
:108E2000BDE8F88F4FF46045AEE700BF0040005842
:108E3000CEFA0DF000B58DB001A904F03DF901A8FE
:108E4000FFF796FF0DB05DF804FBFFECF0B50446AC
:108E50000D46124E89B024F01F0425F01F05104F57
:108E600005F0D2FBA54201D809B0F0BDE369324656
:108E7000394600200793A369069363690593236924
:108E80000493E3680393A3680293636801932368E0
:108E900000932346F8F768FB2034E3E7A081170826
:108EA000204116082DE9F8430D4614461E4602EBF4
:108EB00003081B4903461B4A074600209DF82090E3
:108EC000F8F752FB2B46174A00201749F8F74CFBDE
:108ED0002346144A00201549F8F746FB3346114A49
:108EE00000201349F8F740FBAC4207D8A84505D944
:108EF00041462846BDE8F843FFF7A8BF3B46094A6C
:108F00000C490020F8F730FBB9F1000F06D03146CC
:108F1000204600F005FB4146081AEBE7BDE8F88360
:108F20005C411608AE8117086B4116087E41160891
:108F300091411608A44116082DE9F04399B0044662
:108F40004022002108AF3846F8F7B5FA204600F075
:108F50001FFBE56C2DB1A8B34FF47A735843B0FBF7
:108F6000F5F5A38E03F00303012B2DD1D4F8AC301B
:108F70004021204A384602F098FB2046E66894F8E3
:108F800010808C3454F8409C00F002FB0A22B5F5A6
:108F9000487F079734BF20232123CDF80080B5FBFD
:108FA000F2F102FB1152CDE90534CDE90312CDE90E
:108FB00001903346104A11490020F8F7D5FA19B04C
:108FC000BDE8F0830546CCE7A3680026DFF83090C3
:108FD0009B6AD3F8088058F8043F002BCDD03F2E71
:108FE000CBD8C6F14001B8194A4602F05EFB0644F0
:108FF000F1E700BFD941160884811708DD41160842
:10900000B76E16082DE9F04784B0704D06468846C5
:1090100004AF05F0F9FA2B68002B00F0C2806C4B0E
:109020001B6800206B4A8C336B49CDE900833346C3
:10903000F8F79AFA2B68002B00F0B580644ABA461C
:10904000D2F80090C9F88830D9F88840E36E226FD2
:10905000616FA06F0092614ACDE901106049002064
:10906000F8F782FAA368E2682169606900925B4AB6
:10907000CDE901105B490020F8F776FAA369E269AF
:10908000216A606A0092554ACDE9011056490020D4
:10909000F8F76AFAE36F2268D4F88010D4F88400F5
:1090A00000924E4ACDE9011050490020F8F75CFAD1
:1090B000D4F888306268EFF314810020CDE90021F4
:1090C000464A4B49F8F750FAA36A444A00204949F6
:1090D000F8F74AFA2B68484A5146003B474818BF00
:1090E000012300934FF44073FFF7DCFE2B680BB1B4
:1090F000D3F800A00123514641480093D9F84C30E1
:10910000D9F85420FFF7CEFE00F04CFA8146002833
:1091100052D04FF47A744FF440734443B4FBF3F4E9
:1091200038490020384AF8F71FFA0A23B4F5487F77
:109130004FF00000B4FBF3F234BF2021212103FBE8
:109140001243CDE90092CDE902312F4A4FF440732A
:109150002E49F8F709FA00212D480DF0A1F805F085
:1091600053FA2B6838464BB3194B196832464346BD
:1091700029F1CAFC05F048FA286818B9254B1B6884
:109180001B68EBB9002029F1DFFBEFF3118300230B
:109190008022EFF3108372B682F3118883F3108874
:1091A000FEE71C4B3CE71B4BBA46D3F80090D9F8BE
:1091B000880000F049F947E70446B1E7154BD4E7CA
:1091C000BD46BDE8F04729F1BFBB00BFC410002475
:1091D000B4110024CE81170813421608BD81170868
:1091E0004642160874421608A2421608D0421608D3
:1091F000FE4216082D431608C00D002444431608ED
:10920000484316084D4316089281170888431608EC
:10921000398F0208B81100242DE9F041074688462D
:10922000164E3568FAF78CFA414604463846FAF786
:1092300031FC134B1B681BB10CF07EFF0443E4B2FE
:1092400074B1104C28460DF0A6F8236853B1C5F848
:109250008830356828460DF0A0F8D5F888302360AE
:10926000BDE8F081346820460DF097F8D4F88810F6
:1092700005F18800BDE8F04100F007B9B8110024FD
:10928000AC110024C410002438B5036D0C4605460B
:1092900011469BB9204601F0E7FC2865286DB0B166
:1092A0000119686521F00701091AE96400F050F915
:1092B000AB8E002043F48053AB8638BDC36CA34211
:1092C000ECD000F073F82B6D002BE7D1E2E74FF004
:1092D000FF30F2E70B4C08B52368EFF3118300234E
:1092E0008022EFF3108372B682F3118883F3108823
:1092F0000DF04EF9246820460DF04FF8D4F88800A0
:1093000000F002F8B81100240146012000B500DF8A
:109310005DF804FB08B5094AC0230949013B42F83E
:10932000041BFBD1FEF7E6FF064B0BB128F126FE2E
:10933000FFF776FBBDE8084001F02EBBC00D00240E
:10934000EFBEADDE7D1F150838B504464518207800
:1093500008B1AC4200D138BD0134FFF785FBF6E718
:1093600070B5104D2C680CF0E7FE70B10E4E204623
:109370000DF011F833684BB1C4F888302C682046E2
:109380000DF00BF8D4F88830336070BD2D68284696
:109390000DF003F8D5F8881004F18800BDE870409E
:1093A00000F073B8B8110024C410002410B50446AE
:1093B000006D20B1A38EDB0401D501F04DFCA38E1E
:1093C00023F48053A3860023C4E91433E36410BD5F
:1093D0002DE9F041037F04460D46023B012B1FD8C7
:1093E000F1B1164F3E68FAF7ABF980462574204676
:1093F000FAF782F9804513D0114B1B680BB10CF0C2
:109400009BFE104C30460CF0C6FF236853B13D68FC
:10941000C6F8883028460CF0C0FFD5F888302360A5
:10942000BDE8F0813C6820460CF0B7FFD4F8881006
:1094300006F18800BDE8F04100F027B8B81100241B
:10944000AC110024C41000240146002000B500DF48
:109450005DF804FB38B5CD1D036D044625F0070506
:109460007BB1C36CAB420ED9436D2A46002118462E
:10947000F8F721F8626D03462A446265E26C521BDC
:10948000E264184638BD0023FBE703460A46022083
:10949000194600B500DF5DF804FBFFEC70B5064629
:1094A000114D2C68FAF70AFB3046FAF725F970B12E
:1094B0000E4E20460CF06FFF33684BB1C4F8883075
:1094C0002C6820460CF069FFD4F88830336070BDFA
:1094D0002D6828460CF061FFD5F8881004F188004B
:1094E000BDE87040FFF7D1BFB8110024C4100024BC
:1094F00070B5036D06460D46144623B1818E01F00A
:109500000301FFF753FF2C44284624F00704611B96
:10951000C6E91455F16400F01BF8002070BDFFECA3
:109520000246084669B1D31D1044084A23F00703D8
:1095300020F00700C01A80081968914200D108B9CC
:109540008000704704330138F6E700BFEFBEADDEA0
:10955000C21D80B522F0070282B0134600AF79B970
:10956000391DB94228BF394621F00701091A21F0F7
:1095700003011144054A8B4204D10837BD4680BD22
:109580000144F1E743F8042BF5E700BFEFBEADDE81
:10959000C16C406DFFF7C4BF10B5C46CFFF7F8FF96
:1095A000201A10BD09480A4A20F0070300F2F920EA
:1095B00020F00700C01A80081968914200D108B94C
:1095C0008000704704330138F6E700BFC70D002460
:1095D000EFBEADDE08B5FFF7E5FFC0F5407008BD92
:1095E0007047FFEC38B50025C1680446C0F88050CC
:1095F000C0F88450C0F8885061B91C4B186840F21C
:10960000EE23A0F2EE20E364C4E91400BDE8384084
:10961000FFF79EBFC36CD422406D2946D43B18444B
:10962000C4F88800F7F747FF636DE16CD4F8882031
:109630000B4413606369D4F8882023F00103C2F857
:1096400084304FF08072D4F88830C3F888206FF0EF
:109650001602D4F888309A62F022D4F88830C3F821
:10966000CC50D4F888305A6038BD00BF7036160828
:1096700010B5D0F8802004460B46FAB91F4A12688C
:1096800082421CD11E4C216811B9BDE81040184718
:10969000A1F1D400C2E92031D4222060F7F7A0FD67
:1096A000236803F1D4021A60164A2368C3F88420A1
:1096B00080225A604FF08072C3F8882010BDC0F835
:1096C0008010D422D0F88810C0F88410A1F1D40002
:1096D000C4F88800F7F784FDD4F8883003F1D40289
:1096E0001A60084AD4F88830C3F884208022D4F85D
:1096F00088305A60D4F88830DCE700BFB811002405
:10970000C41000240997020838B50E4B1C68F023DA
:10971000D4F8845083F3118862B6D4F880302046A0
:109720009847EFF3118300238022EFF3108372B682
:1097300082F3118883F3108800232846C4F8803010
:10974000FFF7E2FDB811002438B50A460169044666
:1097500029B14B69036103B9436100234B61637E07
:10976000207EC3F3C00520B9E068007C60F3C3032A
:109770006376CB6820464A819847637E65F3C303CE
:10978000637638BD37B50446C0680A4680B10368C1
:10979000B4F85E10009121469D6804F11D03A847AE
:1097A000002803DA237C43F00103237403B030BDA7
:1097B0006FF00400F6E7FFECF0B5047E3CB313460F
:1097C0006401144FE5592E0415D4AE03124E48BF60
:1097D00045F080652E40334343EA814301F04F0159
:1097E00043F0805343F40043E351437EC28023F0AF
:1097F0004F0319434176027E0123084900201032AD
:10980000D1F81C4893402343C1F81C38F0BD2146D1
:109810002346D5E7000B084000F8F3FF000008409E
:10982000F0B590F818C0144E4FEA4C17BC592504F7
:1098300017D4A303114D42EA814301F04F0148BF01
:1098400044F0806425402B4343EA8C5343F080531B
:1098500043F40043BB51437EC28023F04F031943BE
:109860004176007E0123064A83400020D2F81C186E
:109870000B43C2F81C38F0BD0009084000F833FC67
:1098800000000840437E8A88DB06C97801F00301A6
:1098900001D5FFF7C5BFFFF78FBFFFEC417E027E0A
:1098A000CB064FEA42124CBF084B094B89071344C1
:1098B0001A6822F4001248BF42F080521A60437EB8
:1098C00023F0080343760020704700BF00090840DA
:1098D000000B084001F07F03F0B5EFF31184002185
:1098E0008025EFF3108172B685F3118881F310881B
:1098F0008718FD7C93B1062B0ED801219940294091
:1099000039B18E074FF001031AD49C460133072B5F
:1099100006D1E4B284F31188002010E02946EFE775
:109920000CFA03F63142F1D025EA0605E4B2FD74E3
:1099300084F311881C214B4322B160331844F0BDDD
:109940000226F1E703F59273F8E710B5C0B1B9B19B
:10995000EFF3118200238024EFF3108372B684F3B7
:10996000118883F310884B7E097EC3F300131844DB
:1099700001238B40C17C0B43C374D3B283F31188A2
:1099800010BDFFEC024BD3F80808C0F30D20704760
:1099900000000840037C61F341030374002070471A
:1099A000EFF3118200238020EFF3108372B680F36F
:1099B000118883F310880848D0F8043841B123F0A7
:1099C0000203C0F80438D3B283F311880020704733
:1099D00043F00203F5E700BF00000840084601F02D
:1099E0003BB910B5182001F03FF9044618B1182210
:1099F0000021F7F760FD204610BDFFEC70B5EFF3D6
:109A0000118600238022EFF3108372B682F311884F
:109A100083F31088037CDA0611D50B4CD4F8083890
:109A2000DB070CD5D4F80458052045F0010325F0D8
:109A30000105C4F8043801F0E1F8C4F80458F6B29E
:109A400086F31188002070BD0000084070B54B7E81
:109A500005460C465B070CD422695AB9237E1A4886
:109A60005B01195841F000611950637E62F3820373
:109A7000637670BDD18819B92046FFF765FEEBE724
:109A8000E388124E5A1E1144227EB1FBF3F15201BB
:109A90004B43905900F06040034343EAC1430A49F5
:109AA0009351237E5B015A5842F004425A50637E20
:109AB00043F004036376237E002BDAD16B7C06220D
:109AC00062F307136B74D4E7000B0840100B0840D7
:109AD0001023054A1361054B1169C90601D5013BE5
:109AE000FAD10320F6F798BE00000840400D0300AD
:109AF00040F02000054A064B10611169890601D526
:109B0000013BFAD10320F6F787BE00BF00000840F2
:109B1000400D030038B5036904460D4643B1437E4A
:109B2000DB0606D5007E8001FFF7E2FF23691BB943
:109B300038BDFFF7CDFFF9E729462046FFF704FEC1
:109B4000F4E710B5EFF3118400238022EFF31083C4
:109B500072B682F3118883F310886FF06D01E4B25E
:109B6000FFF7D8FF84F31188002010BD70B5437E45
:109B70000446DE063CD5037E3D495B015B581D046F
:109B800034D5EFF3118500238022EFF3108372B6F2
:109B900082F3118883F31088027E5201535823F414
:109BA000004343F090435350324A037E590102EB85
:109BB000431318688007FCD58B58EDB243F00203BD
:109BC0008B50207E8001FFF793FF207E2A490122DF
:109BD000D1F81C388240204623EA0203C1F81C3821
:109BE0006FF06D01FFF796FF85F31188002070BDBF
:109BF000EFF3118600238022EFF3108372B682F315
:109C0000118883F310881C4DD5F8043843F4007391
:109C1000C5F80438D5F804381B07FBD5227E0A2086
:109C20001649F6B25201535823F4004343F09043CF
:109C30005350F6F7F1FD237E114A02215B012046C5
:109C400099500122D5F8043843F48063C5F80438EC
:109C5000217ED5F81C3810318A406FF06D0123EA5F
:109C60000203C5F81C38FFF755FF86F31188BDE7DE
:109C7000000908400809084000000840000B08409F
:109C8000080B0840002882B006DD00230349043396
:109C90000A6898420192FADC02B07047001008404E
:109CA00030B503460B4C1A1D1B1A994200DC30BD1F
:109CB0002368C3F3072502F8043C02F8035CC3F3EE
:109CC0000745C3F3076302F8025C02F8013C134640
:109CD000E9E700BF00100840F0B5057E1F4F6D0199
:109CE000EB5903F0004392B3C688541E3444B4FBCE
:109CF000F6F4467E134306F0030643EAC443012EFE
:109D0000174E08BF43EA4473EB51457E047E05F0CD
:109D100003056401012DA35908D1124DD5F8085847
:109D2000ED0554BF43F0805343F0005323F08043CC
:109D3000033243F004439210A351037E00201B031F
:109D400003F1804303F50123824202DCF0BD0124CC
:109D5000CFE751F8204001301C60F5E710090840BA
:109D60000009084000000840F8B50D6907460C4698
:109D70005DB90B7E30495B015A5842F000625A507F
:109D8000637E65F382036376F8BDEB881BB94B7E77
:109D900043F040034B762A89EB889A4208D3617ED0
:109DA000480605D420460021BDE8F840FFF7CCBCAA
:109DB0009B1A627E002B22F04002627602DDE6886A
:109DC0009E4212DD1E46217E1C4B4A01D358F21CD6
:109DD0009BB2B3EBA20F11DA194A0123D2F834086F
:109DE0008B400343C2F83438CEE7ECD12A79D2074E
:109DF000E8D5627E42F040026276E3E72B89324684
:109E0000296820461944FFF767FF637E43F0040387
:109E10006376237E23B97B7C052262F307137B7470
:109E20002B891E44EB88B6B2B3422E81ACD8637E38
:109E30005906A9D4B6E700BF000908401809084030
:109E400000000840184A38B50346C0688A60EFF33E
:109E5000118400228025EFF3108272B685F31188F9
:109E600082F310885A7E12F0080219D11D694A61E6
:109E70004DB95A7EC3E90411510708D50020E4B258
:109E800084F3118838BD5A6951615961F6E7194662
:109E9000D30602D5FFF768FFF0E7FFF7D7FDEDE740
:109EA0006FF00F00EBE700BF000089FF054B064A8B
:109EB000C3F8102BD3F8002B42F00442C3F8002B58
:109EC000704700BF000008401800086010B5044645
:109ED0006030FFF701FF0422637C62F307136374B1
:109EE000BDE81040FFF7E2BF00221146FFF7EEBFCA
:109EF000344A00202DE9F047D2F80438324C23F0E0
:109F00000103C2F80438FFF7F3FDE06818B10368F5
:109F10002146DB689847FE232C4E2D4F00254FF03D
:109F2000FF0A4FF01C09E374237509FB054830460E
:109F3000C7F800A06FF06D01C7F800A20135FFF768
:109F4000E9FD98F8793006F1C4006FF06D0123F057
:109F50004C0320371C3688F87930FFF7DBFD98F882
:109F60003D31072D23F04C0388F83D31DDD1154BF1
:109F70004FF0FF3200211548C3F818284FF00112A6
:109F8000C3F81C280B22C3F81428C3F81028D3F8F0
:109F9000002822F4FE62C3F800284022238A23F41A
:109FA000706323F00403238202232372FFF738FC3B
:109FB000402200210748FFF7FFFBBDE8F047FFF70D
:109FC00075BF00BF00000840484E0024A84E002482
:109FD000080908406C4F002438B5124D0446D5F8E6
:109FE000043843F40073C5F80438D5F804381B0767
:109FF000FBD5227E0A200C495201535843F080437E
:10A0000043F400135350F6F707FCD5F8043800204A
:10A0100043F48063C5F80438637E43F00803637635
:10A0200038BD00BF00000840000B0840427E0346D8
:10A03000D20601D4FFF7D0BF027E06485201115864
:10A0400041F40011115000205A7E42F008025A7665
:10A05000704700BF0009084010B5EFF311840023DA
:10A060008022EFF3108372B682F3118883F3108895
:10A0700029B1FFF713FCE4B284F3118810BDFFF798
:10A08000D5FFF8E7F8B5437C044603F0F003202B36
:10A0900040F0AC8000F592756FF046012846FFF75E
:10A0A00039FD6FF0460104F16000FFF733FD94F8CD
:10A0B0003D31A77D23F00803B4F81760E07D84F8F4
:10A0C0003D3194F87930B4F8191023F00803B4F84E
:10A0D0001B2084F87930238A23F001031B051B0D14
:10A0E00043F440532382637D13F0600F05D004F1E5
:10A0F00015012046FFF746FB5BE00C2F26D80FF238
:10A10000080C5CF827F000BF3DA10208F5A1020889
:10A110004DA102084DA202084DA10208EBA20208BF
:10A1200039A3020839A3020841A302085DA302086B
:10A13000EFA00208EFA00208B3A10208207C4707A5
:10A1400004D5022A02D11F0600D526B1237C43F094
:10A15000010323742DE003F01F03012B47D0022BD2
:10A160000CD0002BF2D10029F0D1C0F30013C0F3C2
:10A170004000A17740EA4300607715E001F07F03DB
:10A18000062BE3D8C3EBC3030A064FF002024FEAE3
:10A1900083034CBF603303F5927323445B7EC3F3A8
:10A1A000C00363770023A37704F11D012046FFF766
:10A1B0008DFE237CDB0716D594F878302846764947
:10A1C0005B015A5842F400125A5094F8793043F027
:10A1D000080384F87930FFF7FFFE237C43F0010386
:10A1E0002374FFF763FE0023A4F85E30F8BD6677A2
:10A1F000A677D9E7207C4707A8D5002AA6D103F087
:10A200001F03022B17D1002E7FF471AF01F07F00E6
:10A2100006283FF66CAFC0EBC0000E064FEA800088
:10A220004CBF603000F592702044FFF737FB2046AA
:10A23000FFF75AFEBDE7002B7FF459AF012E7FF4E4
:10A2400056AF034662F304132374F0E7277C7807C4
:10A250007FF57CAF002A7FF479AF03F01F03022B58
:10A2600012D1002E3DD101F07F00062839D8C0EB75
:10A27000C0000A064FEA80004CBF603000F59270C3
:10A280002044FFF7D3FED2E75BBB012E03D147F09A
:10A2900010072774CBE7022E23D1CBB20BBB090AE0
:10A2A000A37C0139042914D8DFE801F0030B0D0F5A
:10A2B0001100012262F30303A374237C43F0200303
:10A2C000C2E70222F6E70322F4E70422F2E70522BE
:10A2D000F0E723F00F03A374237C43F001032374FE
:10A2E000EBE73B077FF532AF01E7DF067FF42EAFE8
:10A2F0000A437FF42BAF7F2E3FF628AF637C03F039
:10A300000F03022B3FF422AF244AD2F8003823F483
:10A31000FE6343EA0013C2F8003858B902469300BE
:10A3200043EA0223228A22F4706222F004021343D9
:10A3300023827CE70122F2E7DE067FF407AFD6E650
:10A34000207C40077FF502AFDB067FF4FFAE0E43B3
:10A350007FF4FCAE012A7FF4F9AEC8E6207C470703
:10A360007FF5F4AED8067FF4F1AE0A437FF4EEAE8B
:10A3700004F115012046FFF705FA00287FF419AF14
:10A38000228AF6B2064B13401EB143F402732382B5
:10A390000FE743F48073FAE7000908400000084023
:10A3A000F7F0FFFF2DE9F04F85B0DFF8B092D9F854
:10A3B0001440D9F8181041F4403242F4407222405F
:10A3C0000C4022F0E96222F4E02222F47D7222F0B5
:10A3D0000102C9F8142000F09D80270300F19E803F
:10A3E000660313D5DFF87492D9F81838D9F81C2809
:10A3F00013409BB20193002B40F03A81D9F81838F2
:10A40000FF21954A9BB2002B40F02081002C12DAEC
:10A41000924A0121924DD2F80438284623F00103D4
:10A42000C2F8043828F16FFAE86820B103685B6964
:10A430000BB12946984721050AD58949C86818B142
:10A4400003681B6903B198470021854828F15BFA2E
:10A45000E20659D5814B1D6A05F00F09B9F1060FC7
:10A4600052D805F4F012B2F5002F00F0A781B2F532
:10A47000402F00F0B181B2F5802F45D1C5F30A1508
:10A48000002D41D0DFF8D8811C2606FB0986D6F8BE
:10A490003471002F40F07D8196F83CA1BAF1000F95
:10A4A00040F07381D6F830717B7C03F0F003102B01
:10A4B00040F06B81402DAB4607F11D00A8BF4FF067
:10A4C000400B1FFA8BF10191FFF7EAFBA5EB0B00A4
:10A4D000FFF7D8FB96F83D31022238466AF3820333
:10A4E00086F83D317B7C62F307137B740199A7F8F2
:10A4F0005E10FFF7C7FD1C2303FB098898F83D3168
:10A5000023F0040388F83D31564B1C4200F079815A
:10A51000FFF7EEFC002005B0BDE8F08FD9F8186811
:10A52000D9F81C281640360C0ED1D9F81838FF215E
:10A530004D4A1B0C002B3FF453AFDD0701D51068CB
:10A5400011605B082032F5E7DFF820810027A8F5CD
:10A550009275F00740D5444B4FEA471A5AF803105A
:10A56000D9F8142801EA0203D90701931ED5012264
:10A570003D4B4AF803206A7C002F44D102F0F002E0
:10A58000602A13D1D5F834216ABB95F83D2167F3D1
:10A59000820285F83D2195F83D2112F0040105D194
:10A5A000FFF784FC6A7C61F307126A74019B9A07C7
:10A5B00003D502222C4B4AF80320019B1B070BD525
:10A5C0006A7C02F0F002202A02D12548FFF75AFDEA
:10A5D0000822254B4AF80320760807F1010708F105
:10A5E0001C08B6D1FCE639462048FFF7ADF895F8CF
:10A5F0003D211E4967F38202A1F5927085F83D2145
:10A60000FFF724FAC7E702F00F02022ACED1D8F8EA
:10A6100010104FF01C0B41B90BFB075B9BF83D2161
:10A6200061F382028BF83D21C0E70BFB075B4046DC
:10A630000021FFF789F89BF83D214146084822F0A8
:10A6400004028BF83D21FFF701FAAFE7D80700D5E8
:10A6500011605B082032D6E6080908400000084077
:10A66000484E002400108000080B08406C4F002466
:10A67000704F4FF00008A7F1600A019BDA0773D50D
:10A680000121D9F81028D9F834584FEA481B01FAAB
:10A6900008F32B420293684B18BF42F080025BF82C
:10A6A0000360164016F0010303933BD0029B012286
:10A6B00025EA0305604BC9F834584BF803209AF893
:10A6C0001120B8F1000F57D102F0F002502A10D13A
:10A6D0005849A1F16000FFF747FB9AF8792053072A
:10A6E00007D4FFF7E3FB9AF8112068F307128AF802
:10A6F00011209AF81010880614D5504B21F0200133
:10A700009AF81220D3F8040802F00F0E22F00F027C
:10A7100000F0700040EA0E10C3F804088AF8101028
:10A720008AF81220320703D50822434B4BF8032046
:10A73000F30607D539465046FFF716FB10223E4B6D
:10A740004BF8032030060FD5039B4BB9029B3946CB
:10A750003A4A25EA03053A48C2F83458FFF704FBA1
:10A760008022354B4BF80320019B08F101081C3770
:10A770005B08019381D149E602F00F02022AD1D190
:10A7800039462F48FFF7F0FACCE72846FFF77AFA68
:10A79000B1E63889FE883B68361A1844AE42A8BF35
:10A7A0002E461FFA86F84146FFF77AFAA81BFFF7F4
:10A7B00069FA3B899844A7F80880A5E6204A527CAC
:10A7C00002F0F002102A7FF49FAED3F8002B42F083
:10A7D0008062C3F8002B97E61A480821FFF760FA59
:10A7E00090F90010A0F11503C288002906DB2AB1F8
:10A7F0005A7C012161F307125A7485E65A7C0221C2
:10A80000F8E7A3047FF5D1AD0C4BD3F800296FF323
:10A810000A0242F04002C3F80029D3F8042842F4A7
:10A820008072C3F80428DA6822F4705242F4C052ED
:10A83000DA60BAE5A84E0024080908400000084084
:10A84000484E00245D4E002438B50B4CE060214694
:10A8500003681B689847054618B10023E360284643
:10A8600038BD7520F6F71AFB01212046FFF798F84E
:10A8700002232372F3E700BF484E002470B504465C
:10A88000EFF3118580260023EFF3108372B686F371
:10A89000118883F31088FFF72BFBEDB285F3118845
:10A8A0000E4D2046236829465B689847EFF31184D4
:10A8B0000023EFF3108372B686F3118883F31088B8
:10A8C0007520E4B2F6F7D6FA00212846FFF768F8BB
:10A8D0000846E96084F3118870BD00BF484E00242B
:10A8E00070B52B4DE86808B1FFF7C8FFEFF311868C
:10A8F00000238022EFF3108372B682F3118883F372
:10A90000108800212248FFF74BF875200C46297269
:10A91000F6F7B0FA752021462246F6F77FFF1D4B69
:10A92000FF204FF0FF32F6B2C3F80809C3F8080B56
:10A93000C3F82809C3F8280BC3F84809C3F8480B23
:10A94000C3F86809C3F8680BC3F88809C3F8880B13
:10A95000C3F8A809C3F8A80BC3F8C809C3F8C80B03
:10A960004FF48060C3F81048C3F81448C3F8344863
:10A97000C3F81C48C3F81828FFF7BAF8FFF7A8F87F
:10A980006B7C64F303036B7486F3118870BD00BFA6
:10A99000484E002400000840894AF8B5D2F80C3827
:10A9A00023F0007343F08073C2F80C38D2F80C38EF
:10A9B0005901FBD583484027F6F7FEF88248F6F7A1
:10A9C000FBF8824EFFF78CFF814B4FF4F4720021AD
:10A9D0001846F6F770FD7F490246034604464FF0DD
:10A9E0001C0C42F8601B4260FE22C27402750022F9
:10A9F0000CFB02411C335E641C6501F1780591F883
:10AA0000791041F010016970D1B2013283F85C1005
:10AA100061F07F01072A83F84810697821F003016B
:10AA20006970A3F84A70E3D100234021DAB2013300
:10AA3000C0F824611C30072BC0F8144180F8202195
:10AA400080F80C21A0F80E11F0D100226249752087
:10AA5000F6F7E4FE002803DABDE8F840FFF740BF50
:10AA60005E4C80235E4DA360E36843F04003E360E7
:10AA70000320F5F7D1FE2369002B01DB013DF7D15F
:10AA8000236943F001032361554B544C2269D207DB
:10AA900001D5013BFAD103200025F5F7BDFEA36BDC
:10AAA000142043F48033A36300F0A8F82368322015
:10AAB00043F0C0032360E36823F0005343F0804376
:10AAC000E36000F09BF8C4F8005ED4F800384FF45F
:10AAD000806023F4C053C4F80038D4F8003843F041
:10AAE0000303C4F8003840F20123636203F59203C4
:10AAF000A3624933C4F804314933C4F808314933F7
:10AB0000C4F80C314933C4F810314933C4F8143156
:10AB10004933C4F81831FEF7EBFFFEF7D9FF4FF0C9
:10AB2000FF33C4F81058FF21C4F814582D4AC4F854
:10AB30003458C4F818382C4BC4F81C581868203303
:10AB40000028ACBF00204FF0084043F8200C43F829
:10AB5000105C43F8181C9342F0D1244B0022FF20D4
:10AB600023491C682033002CACBF00244FF008445C
:10AB700043F8204C43F8102C43F8180C8B42F0D1CA
:10AB8000164B13489A614FF0FF325A605969194ABF
:10AB900021F07F4121F47C0121F47C4121F0FF016F
:10ABA0000A4300215A61144A9A6181229A60FEF791
:10ABB000F7FEFFF79DF97520BDE8F840F6F76EB98E
:10ABC000004002580BAC08000CAC0800F4811708D8
:10ABD000484E0024D8811708A5A3020800000840A9
:10ABE000400D0300E009084000090840000B084040
:10ABF000E00B08400AFCB0F810380C0082B00022CC
:10AC000009490092009B834201D302B07047019230
:10AC1000019B8B4203D9009B01330093F2E7019B18
:10AC200001330193F4E700BFAD7301000A4601460A
:10AC3000034808B500F06BF8024B186008BD00BF70
:10AC4000BE43160830500024024B0A4601461868DD
:10AC500000F022B830500024024B0146186800F082
:10AC6000DFB800BF30500024024B0146186800F0E6
:10AC700033B900BF30500024024B0A460146186821
:10AC800000F087B930500024024B0146186800F0EC
:10AC900052BA00BF30500024F8B5C56A04460E46CB
:10ACA0001746032D32DC00F067F806F11F00F31998
:10ACB000A26820F00F00012723F00F03A0F110017C
:10ACC0005E1A3244103EA26004EB85020825D16072
:10ACD00040F8105CD1684F60A0F1080140F8086CA2
:10ACE000A3F108064D60D66143F8085C50F8083CB3
:10ACF0002046D2693B435360E36A3B44E36200F081
:10AD000067F82046BDE8F84000F05AB8F8BDF8B53D
:10AD100001F10F03A2F5B87506464FF4B87223F09F
:10AD20000F030D44002118461C46ED1A03F5B877B1
:10AD3000F6F7C1FB034600F1400200F5B071A2F145
:10AD400010009A6310321033D8638A42F7D120463C
:10AD500000F00DF82A4639462046C4E95964FFF749
:10AD60009BFF04F5B2700AF085FC2046F8BD012275
:10AD7000002100F0D4BBFFEC104B37B51C68054632
:10AD80004CB101A900F0E2FB01980028D4BF0020DB
:10AD9000012003B030BDF7F765FD00280CDB284625
:10ADA000F6F7F2FE002801DB0120F2E7F6F7FAFBE6
:10ADB0000368002BF3DCF7E72046EAE7C410002421
:10ADC000024B1B680BB9F6F73BBF7047C410002459
:10ADD00038B5054608680C4600F015F8C21C05EBAE
:10ADE000021205EB0015AB6B23B1196811B1206895
:10ADF000814205D39460C4E9023203B1DC6038BDFE
:10AE00001A469B68F0E7B0F5800F07D203090020CF
:10AE1000012B00D8704701305B08F9E7122070471A
:10AE200070B505460C46A9B1FFF7A6FF98B9EFF338
:10AE3000118300228021EFF3108272B681F3118812
:10AE400082F31088D5F86021DBB22260C5F860413A
:10AE500083F3118870BD54F8043CA4F1080123F079
:10AE6000010344F8043C54F8083CCA185068C6076B
:10AE700013D4CB58D2E902061344B06008B1D668A7
:10AE8000C660126854F8080C104444F8080C5A685C
:10AE900002F0010202435A601A4654F8043CCB1AED
:10AEA0005868C00710D4D3E90210816009B1D8688E
:10AEB000C86054F8081C186808441860516801F00C
:10AEC00001010143516019462846FFF781FF2846DA
:10AED000BDE87040FFF774BFF8B506460F46EFF3C4
:10AEE000118300228021EFF3108272B681F3118862
:10AEF00082F310880022D0F86041DBB2C0F86021F4
:10AF000083F31188002C39D1002F35D007F11705B4
:10AF100025F00F05AF422FD83046FFF72DFFB5F5CE
:10AF2000800F32D22846FFF76EFF06EB0010846BCD
:10AF3000FCB12368AB42A36829D3E26893600BB1EC
:10AF4000E268DA602368581B0F280CD92344611982
:10AF500060514D6025605A6802F00102024330469C
:10AF60005A60FFF735FF6368083443F0010344F883
:10AF7000043C3046FFF724FF2046F8BD25682146F3
:10AF800030462C46FFF74CFFBCE71220CDE71C46AD
:10AF9000CEE72DE9F84F074692460D4621B91146F6
:10AFA000BDE8F84FFFF798BF32B9FFF739FF4FF010
:10AFB000000B5846BDE8F88F02F1170323F00F0B82
:10AFC0005A45F4D8A1F10804FFF7D6FE55F8088CCD
:10AFD000C3450AD804D25A462146384600F0B7F88D
:10AFE0003846AB46FFF7ECFEE3E755F8041C04EBEC
:10AFF000080921F00101D9F80430611ADA0748681C
:10B000004CBF002654F80860C30706EB080354BF82
:10B01000D1F800C04FF0000C63445B4576D3B445D3
:10B02000ABEB080308D29C4555D2A3EB0C03BCF153
:10B03000000F53D1AB4626E09E42FBD29B1BB2468B
:10B04000D1E9022082600AB1C868D0609C45A4EBB7
:10B05000030446D90A683846D21A43440A6023607A
:10B060000A6842F001026260D9F8042002F001028D
:10B070001A43C9F80420FFF7ABFE04F1080BBAF13C
:10B08000000F1BD0534609EB0600D9E9021291606C
:10B0900011B1D9F80C20CA6022689E421A4422607D
:10B0A0002ED9F61AA118A65023684B60436803F006
:10B0B0000103334343603846FFF78AFE3846FFF703
:10B0C0007FFE5D453FF475AFA8F10802294658465A
:10B0D000F6F786F86DE74FF0000AB1E79A46634647
:10B0E000AEE722686368424443F001032260636074
:10B0F000D9F8043003F001031343C9F80430BCE766
:10B10000436803F0010313434360D7E73846FFF772
:10B1100057FE51463846FFF7DFFE834600283FF4CE
:10B1200048AF2946A8F10802F6F75AF829463846EA
:10B13000FFF776FE3DE738B50D46FFF7CDFE044636
:10B1400018B12A460021F6F7B6F9204638BDF0B40A
:10B150000C680B4606460D196968C90719D41859B9
:10B16000D5E902172844B96009B1ED68CD601D68C2
:10B1700099181C59AD1A25449D504A601A604468BC
:10B180009B5804F001041C4344603046F0BCFFF7B8
:10B190001FBE02F110018C4209D39918A41A9C50C9
:10B1A0004A601A609B5843F001036B60EEE7F0BC05
:10B1B000704738B505460024204602F095F818B9C6
:10B1C0006FF00104204638BD294601F0E7FD002854
:10B1D000F8D00134F0E7FFEC044B1B688342C6BF94
:10B1E000034B03EB00100020704700BF4C8E170884
:10B1F000508E17081F2804DDA0F17F0358425841E4
:10B20000704701207047202805D0093804288CBFDA
:10B2100000200120704701207047A0F13003092B66
:10B2200007D920F02000413805288CBF00200120DC
:10B23000704701207047A0F14103192B98BF2030BF
:10B24000704738B505463020FFF70EFD044630B98B
:10B25000F6F7A8F90C2303600024204638BD40F619
:10B260000141284604F016FE002803DA2046FFF7C5
:10B27000F3FCF1E72060F0E738B5044638B9F6F79B
:10B2800091F94FF0FF3509230360284638BD006867
:10B2900004F063FA05462046FFF7DEFCF5E710B53B
:10B2A00028B9F6F77FF909230360002407E0041D9D
:10B2B0002A220068214604F027FE0028F5DD2046FA
:10B2C00010BDFFEC10B50446C0B10378B3B101F076
:10B2D0008CFD0021204410F8012C431E2F2A07D09A
:10B2E0002F21204601F005FD00B1441C204610BD71
:10B2F000001B012804DD18461970ECE7014CF5E746
:10B30000014CF3E7D31317087ADA160810B5044690
:10B3100008B30378FBB101F068FD0021204410F868
:10B32000012C431E2F2A0DD02F21204601F0E1FCD5
:10B3300088B10022A04208D000F8012903782F2B01
:10B34000F8D003E0001B012802DC044C204610BDAD
:10B3500018461970E3E7024CF8E700BF7ADA1608DE
:10B36000D3131708034638B1044A03CA186010689B
:10B3700059609860002070470C207047408E170875
:10B3800020B1012902D1417000207047162070477A
:10B3900020B119B10B680370002070471620704768
:10B3A00008B5034608469847F6F706F907B500932F
:10B3B00013460A46014603480AF0B4FD03B05DF89F
:10B3C00004FB00BFA1B30208002303600B6813B99C
:10B3D0000860486070474B681860FAE70B680360C4
:10B3E00003B9486008607047034608461146126872
:10B3F00012B14A689A4201D1FFF7E6BF1A680260AB
:10B40000186070470B6802468BB180B1834208D147
:10B410001A680A604A689A4209D100234B60704753
:10B420002BB118461B689342FAD100F00BB8704755
:10B430000346006828B102681A6002B95A60002306
:10B44000036070470A680346006852B148B14A6811
:10B4500082424FF0000206BF4B601146016819603E
:10B4600002607047002303604B6843600A6812B9AA
:10B470000860486070471860FBE7002343600B6872
:10B48000036013B9C1E90000704758600860704755
:10B49000D0E9003232B90B6033B94A600023C0E909
:10B4A000003370471360F7E75A60F7E7FF207047F3
:10B4B0000120704738B543680C460568084AD9171B
:10B4C000E5FB02311846074B074AC0184FF000034E
:10B4D00041F100010CF04EF92060002038BD00BFA2
:10B4E00000CA9A3B3F420F0040420F000D461646ED
:10B4F000044608B501F004FF31462846A047F5F799
:10B5000081FF034640B1B2F5004F05D212B202806E
:10B5100000209870586070476FF01500704710B5A4
:10B52000FFF7EFFF041E05DA6442F6F73BF804600C
:10B530004FF0FF34204610BD28B121B10388002010
:10B540001BB20B6070476FF01500704710B5FFF726
:10B55000F3FF041E05DA6442F6F724F804604FF0A6
:10B56000FF34204610BD1F299FBF012203688A4077
:10B5700013439ABF036000206FF0150070471F2926
:10B580009FBF012203688A4093439ABF0360002053
:10B590006FF01500704703460020186070471F29A0
:10B5A0009DBF0068C84000F001006FF015007047B3
:10B5B0002DE9F8430746104689461546984601F09E
:10B5C00014FC06461830FFF75FFB044688B10323DE
:10B5D000721C29460371089BC0E90298036114306C
:10B5E00001F00BFC3846214601F0ACFE0020BDE81E
:10B5F000F8830C20FBE738B50446006808B92060E2
:10B6000038BD0568FFF728FB2846F7E7034600200A
:10B610001860704737B50024054601A9047020461C
:10B620000AF010FEA04204DAF5F7BCFF006803B090
:10B6300030BD019B20466B700AF024FE0028F3DB2E
:10B640004FF40063A8706C602046EB60EFE7017078
:10B65000002070470B68437000207047C1600020D5
:10B6600070470EB430B588B001466FF000420BACA5
:10B6700002A854F8045B01F041FA02A822462946C8
:10B68000019400F04FF808B0BDE8304003B07047B7
:10B690000EB403B503AA52F8041B019200F01DF882
:10B6A00002B05DF804EB03B070470CB40A4600B575
:10B6B00089B071B1014602A801F020FA0BAA0A99DB
:10B6C00002A8019200F02EF809B05DF804EB02B078
:10B6D000704702A801F02AFAF0E7F0B58DB01446E1
:10B6E0000D46074602A8019201F020FA224629469B
:10B6F00002A800F017F8059E01363046FFF7B4FAAD
:10B70000044660B10146324606A801F0F7F9019AF5
:10B71000294606A800F006F83C600DB0F0BD4FF0D9
:10B72000FF30FAE707B5009200220B46114600F001
:10B7300003F803B05DF804FB2DE9F04F8FB0044629
:10B740000025DDF860B01978002900F00084252973
:10B7500007D001330293236820460135D946984724
:10B76000E9E393F801A09A1CBAF1250F0292F2D0F6
:10B7700000273E46B846B8F13F0F48D8BAF12B0F24
:10B780003AD010D8BAF1200F38D0BAF1230F3BD0FD
:10B79000BAF12A0F58D118F4807F5BF8043B4AD0E5
:10B7A00023EAE37707E0BAF12D0F2AD0BAF1300F80
:10B7B00030D148F00108029B13F801AB0293BAF1B3
:10B7C000000FD8D1AAF14503022B00F297800AF1AD
:10B7D000200A48F400585FFA8AFA18F4807F08BFFC
:10B7E0000627BAF1650FF9B240F09E80013148F4A6
:10B7F0008048C9B200229FE048F0020848F00408DF
:10B80000D9E748F00808D6E748F01008D3E7B8F5BC
:10B81000007F24D2AAF13003DBB2092BB8D818F488
:10B82000807F4FF00A020ABF48F0800802FB07370A
:10B8300002FB0636BFE7002BA7BF48F080081E4674
:10B840005E4248F08808B6E7BAF12E0F40F07683E2
:10B8500018F4807F40F07B8348F48078ABE7BAF13E
:10B860007A0F0FD0BAF1740F0CD0BAF16A0F06D16B
:10B8700028F480681FFA88F848F420689BE7BAF13A
:10B880006C0F0BD118F4007F18BF48F4006828F43F
:10B8900080681FFA88F848F400788CE7BAF1680FDE
:10B8A0000BD118F4806F18BF48F4006828F40078B2
:10B8B0001FFA88F848F480687DE7BAF1700F81D1EB
:10B8C00028F420681FFA88F848F400780AF0DF03AB
:10B8D000532B40F0C481D946A24B59F804ABBAF1BE
:10B8E000000F08BF9A4618F4807F504614BF3946AF
:10B8F0004FF0FF3101F093FA07460FE0AAF165031C
:10B90000022B7FF66AAFBAF1630FDFD1D946012768
:10B910000DF1200A59F8043B8DF8203018F0080F7B
:10B9200040F08F81B04686E1BAF1660F7FF462AFD6
:10B930000A4648F400480F210BF1070B0F2908A80D
:10B940002BF0070928BF0F21B9EC020B00F034FBE4
:10B950009DF82430DDF820B003F00902012A38D028
:10B9600018F0020F38D1C8F3800A4FEA4A1A13F0D0
:10B970000C0F3ED0BAF1000F0CBF03230423B342D7
:10B980000CDA18F0080FA6EB030608D13746236837
:10B99000202120469847013FF9D135440026BAF1CD
:10B9A000000F04D0236851462046013598479DF882
:10B9B000243008F400586C4F13F0080F6B4B08BF8D
:10B9C0001F463B469A461AF8011B41B9EF1BFD186A
:10B9D000A9E04FF02D0ACAE74FF02B0AC7E7B8F1EC
:10B9E000000F01D02039C9B223682046984753463A
:10B9F000E8E7C3B2B8F5804F01931AD21A4608A9F6
:10BA000005330B44019919B113F8011D302929D0D0
:10BA10001BF1040F2BDB934529DABBF1000F48F42F
:10BA2000004802DB019B9B4524DA0BF10107019BD7
:10BA3000DF1B0FFA88F3002B0393B6BF2BEAEB73DF
:10BA400005230133BAF1000F00D00133A7B17A1CEE
:10BA50001344B342B4BFF31A002318F0090F1FD1E7
:10BA60001E4614E001990139C9B20191CAE7019B50
:10BA70005F1EDEE70027DCE718F0100F18BF013368
:10BA8000E7E7202120460493013E9047049B22686B
:10BA9000002EF6D11D44BAF1000F05D1B24648E0A0
:10BAA0001E46BAF1000F04D02368514620460135E6
:10BAB000984718F0080FF1D0039B002B58DA2BEAB7
:10BAC000EB7A7B42ABEB0A020493019B0AF1FF3A4B
:10BAD00004999A4236BF08AB3027D31802F101020D
:10BAE00038BF5F796B1C8A450393236826DA18F008
:10BAF000100F06D0BAF1FF3F03D12E212046984700
:10BB0000039DD3450AD19DF82530352B28D805D182
:10BB10009DF8243013F0100F08BF3127013523683A
:10BB2000394620469847374602E2013E30212046FA
:10BB300098472368002EF8D15544BDE73946204682
:10BB400005929847BAF1FF3F059A07D1AB1C2E2109
:10BB500020460592039323689847059A039DB4E70E
:10BB60003127DBE710821708C7431608C3431608BE
:10BB70009DF82510204631291EBF9DF8243023F062
:10BB800010038DF8243023689847002F23683BDD8D
:10BB90002E212046984701220235924601992046DF
:10BBA0002368013551450AF1010A88BF38325FFA2E
:10BBB0008AFA92BF30216A4412F8131C98475745FD
:10BBC0005246EBDA18F4005F236820460CBF65216B
:10BBD00045219847BBF1000F04DB1FD19DF82430AD
:10BBE000DB061BD5CBF1000B2D212368204698479F
:10BBF0003021BBF1090F13DC236820469847043538
:10BC000023680BF130018CE718F0100F01D10135DA
:10BC1000D8E72E21204602359847D3E72B21E4E7C9
:10BC20000131ABF10A0BC9B2E3E708F1FF38236831
:10BC30002021204698474745F7D335444646A5EB93
:10BC400008050AEB070806E0236820461AF8011BDE
:10BC5000984706B1013EC245F6D13D4463E7BAF1CB
:10BC6000640F08F4206302D0BAF1690F7BD1B3F5F9
:10BC7000206F63D10BF1070B2BF0070BD946DBF8D4
:10BC8000041059F8080B28F4805B00292BF0100BE6
:10BC900006DA40424BF4805B61EB41011FFA8BFBFB
:10BCA0001BF4807F04D01FB950EA010300F0CA8062
:10BCB0000DF1200A0A23524600F04EF9A0EB0A00CB
:10BCC0005FFA80F81BF4807FCDF8048000F0BC8020
:10BCD0002BF0010A47451FFA8AFA40F3B88044F274
:10BCE0001002FBB20BEA0202102A03D12BF0110B57
:10BCF0001FFA8BFA1AF0100F00F0B38008F1380227
:10BD00006A4412F8192C302A40F0A3802AF4C04A61
:10BD10002AF0100A1FFA8AFA1AF0080F40F0B280CF
:10BD20001AF0010F06D09E4240F3C680F31A03EBCF
:10BD30000807F3B25B1B5FFA83FB9EE0D94618F459
:10BD4000007F59F8040B4FEAE0719CD118F4806F22
:10BD500099D018F4006F0BBF40F3C03140F3C0110D
:10BD600000B240B28FE7B3F5206F1DD10BF1070B86
:10BD70002BF0070BD946DBF8041059F8080B28F014
:10BD8000060BBAF1580F1FFA8BFB47D0AAF16F03CD
:10BD9000DAB2092A4AD8092B48D8DFE803F051273C
:10BDA000474747471847473818F400710BF1040913
:10BDB000DBF8000001D00021E1E718F48063FAD03D
:10BDC00018F4006301D180B2F5E7C0B2D7E728F0DC
:10BDD00016080A231FFA88FB1BF4807F03D017B9CB
:10BDE00050EA01022ED00DF1200A64E7029B1B7875
:10BDF000562B0AD1029B0133029343681A680792BB
:10BE000001682046FFF78EFC95E04BF0100B1BF00D
:10BE1000100F01D04BF4804B1023DDE718F0100F0A
:10BE200001D04BF4C04B4FF40473D5E72368204690
:10BE300025210235984723685146204698477AE0E5
:10BE40000823C9E7B8463DE74346DA4652E743468A
:10BE500050E71AF4804F01D1013300E00233DBB226
:10BE60005AE741F206021AEA020F3FF455AFF3E730
:10BE7000236820212046013598470BEB0503DBB2F0
:10BE80009E42F5DC9E42CCBFF61A00261AF0100F37
:10BE900014D023683021204698471AF4804F33D0BD
:10BEA0001AF4005F05F1020523680CBF78215821C0
:10BEB00020469847BA4619E047463BE741F2060359
:10BEC0001AEA030FF6D01AF0020F05F101052368F4
:10BED00014BF2B2120211AF4805F18BF2D21E7E722
:10BEE0000AF1FF3A2368302120469847C245F7DC23
:10BEF000A7EB08034745B8BF00231D44B8F1000F66
:10BF000004D1019B1D440EE60135D3E708F1FF3350
:10BF10000EAA204652FA83F25FFA83F8236812F8D9
:10BF2000181C9847EAE7013F2368202120469847DC
:10BF3000002FF8D13544CB46029B04E4BAF17A0FC6
:10BF40003FF4A5ACBAF1740F7FF48FAC9FE42846A0
:10BF50000FB0BDE8F08F00BF2DE9F84313F400796E
:10BF60001C4606460F4618BF23F40074154618BF3A
:10BF70004FF001094FEAE4783046394622464346FD
:10BF80000BF048FC092AB4463B4606460F4609DC3E
:10BF90003032A44505F8012B73EB0803ECD2284698
:10BFA000BDE8F883B9F1000F01D03732F1E757321D
:10BFB000EFE7FFECC2925D7D2DE9F74F10EE904A5E
:10BFC00007460E4614F000441CBFB1EE400B01249E
:10BFD000B5EE400BF1EE10FA11D121EAE172053015
:10BFE000302144F00204F5F766FA0025BB1900225F
:10BFF00030465A713C713D6003B0BDE8F08FB4EE3D
:10C00000400BF1EE10FA02D744F00804EDE79FED83
:10C01000407BB4EE470BF1EE10FA02DD44F004046D
:10C02000E3E79FED3D6BB4EEC60BF1EE10FA14D4CE
:10C030003D4908230F25012031ED027B20EE077BCF
:10C04000B4EEC67BF1EE10FA04DB00FA03FCB0EEAE
:10C05000470B6544013BEFD216E09FED316B33494E
:10C0600008230F25012031ED027B20EE077BB4EE83
:10C07000C67BF1EE10FA05D500FA03FCB0EE470BD3
:10C08000A5EB0C05013BEED232B125EAE573013395
:10C090001A449642A8BF1646254B03EBC60393ED00
:10C0A000007B30EE070B9FED1E7BB4EEC70BF1EE6D
:10C0B00010FA04DBB2EE047B013580EE070B07F1CA
:10C0C000040BDFF87090DFF870A051EC100B0BF050
:10C0D000BBFB6FF0030388460090DB1B0193019BC1
:10C0E0005B449E4282DD4A465346009841460BF02F
:10C0F00091FB3030514600920BF8010F98464846AC
:10C100000A2200230BF086FB81468A46E7E700BF40
:10C11000FFFFFFFFFFFFEF7F00003426F56B0C43AE
:10C120000080E03779C34143E0821708288317086D
:10C13000188217080080C6A47E8D0300411E0020CF
:10C14000034610B511F8012F02B910BD782A08D89E
:10C15000712A0DD8622A4DD01ED82B2A35D0612ADB
:10C160002DD0F5F71FFA162303604FF0FF30ECE7F0
:10C17000723A062AF5D801A454F822F0A7C10208A1
:10C1800063C1020809C2020863C1020863C1020850
:10C19000B3C10208FFC10208652AE2D1002BE0D03A
:10C1A00040F48060CEE7002BDBD140F20110012388
:10C1B000C8E7002BD5D14FF493700223C2E7002BC0
:10C1C000CFD14FF48B700423BCE7022B08D0042B93
:10C1D0000BD0012BC5D100F4A16040F00300B1E702
:10C1E00000F4A16040F02700ACE700F4A16040F04B
:10C1F0001700A7E7002BB4D020F48070A2E7002B33
:10C20000AFD040F008009DE7002BAAD040F480702A
:10C2100098E700BF37B50025044608460195FFF7AB
:10C220008DFF011E0ADB204601AB2A4604F086FA88
:10C23000041E03DA6442F5F7B5F90460019803B00F
:10C2400030BD73B50024064608460194FFF776FF1B
:10C25000051E19DB30464FF4DB72294603F01AFE47
:10C26000061E0EDB294601AB224604F067FA051EC6
:10C2700007DA6D42304603F070FAF5F793F905607E
:10C280000194019802B070BD2046FBE7F8B5064660
:10C29000002862D0B0F8284114F0020458D00121DF
:10C2A00000F0CCF90446F5F77DF9076809F070FF56
:10C2B0000830864244D009F06BFF00F59C7086423E
:10C2C0003ED009F065FF00F51A70864238D009F0BB
:10C2D0005FFF054600F0D1FA0022D5F89803034627
:10C2E0006BB1B342196835D183420CBFC5F89813BE
:10C2F0001160D5F89C13994201D1C5F89C232846BA
:10C3000000F0C3FA7068002807DB03F026FA054640
:10C310001CB9F5F747F92C46076806F10800F5F750
:10C32000E3FB002801DAF5F73DF9B06928B196F88A
:10C330002A311B0701D4FEF78FFC3046FEF78CFC38
:10C3400024B14FF0FF34F5F72DF907602046F8BD12
:10C350001627ABE71A460B46C2E71627F1E700F0AF
:10C3600000B870B504460D46164600F0AFF9002837
:10C3700002DA4FF0FF3070BD204600F0D2F90028FD
:10C38000F7DB002332462946606884F82B3103F03E
:10C390003EFC01304FF0FF3018BF0020EBE700F00B
:10C3A00000B870B5044630B9F5F7FCF8092303600E
:10C3B0004FF0FF3070BD01220021406803F027FCE0
:10C3C000431C0646F4D0204600F072FAA369256AA1
:10C3D0005BB1626A934208D0521B94F82B31D51896
:10C3E000204600F085FA701BE4E75D1BF8E70029A2
:10C3F0004FF0000307B506DB0093012300F015F8AA
:10C4000003B05DF804FB1846FAE738B5044659B1A5
:10C4100044F60105204600F0A2FF431C0E2BF9D87C
:10C4200025FA03F3DB07F5D538BD2DE9F0470546BE
:10C430000F4699469DF82080164642B138B15368A0
:10C44000002B04DB39B941461046FFF7DEFF00251B
:10C450002846BDE8F08701294FF0000405D104709B
:10C4600041463046FFF7D1FFF2E700F1FF3A304690
:10C4700000F075FF0A2801D00D280AD1B9F1000F8C
:10C4800002D00A232B55013400232B55E0E71C462C
:10C49000EDE7431C02D1002CF6D1D8E7631C02342F
:10C4A0000AF8010FA742F2D80022EA54D8E710B5E3
:10C4B0000C4611461A46614300F006F80028CCBF2E
:10C4C000B0FBF4F0002010BD2DE9F04106460F4608
:10C4D000154642B9F5F766F84FF0FF3409230360BB
:10C4E0002046BDE8F081B2F828319B070CD4F5F75F
:10C4F00059F8092303604FF0FF3495F82A3143F0CF
:10C50000020385F82A31EBE793693BB90A460146F5
:10C51000686803F0E3FF041EE2DAECE7104600F07F
:10C52000C7F9284600F0D2F8002807DA4FF0FF34A8
:10C53000284600F0DDF9002CD2DADEE7D5E9074025
:10C54000241AB4F5807F01D1FF2F23D8BC42314695
:10C5500028BF3C462246A7EB0408F4F741FE2B6AAD
:10C56000EA692344344493422B620CD2B8F1FF0FA2
:10C5700013D942462146686803F0B0FF0028D5DB96
:10C580000444A41BD4E70021284600F057F80028F3
:10C59000ECDACBE73446B846EBE7B8F1000FF0D061
:10C5A00021464246286AF419F4F71AFE2B6A4344DE
:10C5B0002B62E6E710B568B909F0EAFD00F010F863
:10C5C000002804460ADA6442F4F7ECFF04604FF0F6
:10C5D000FF3010BD012100F031F8F1E70020F8E74D
:10C5E00070B5044640B300F048F9012104F1080099
:10C5F000002600F023F8012104F59C7000F01EF8DD
:10C60000012104F51A7000F019F8D4F8985325B9EF
:10C61000204600F03AF9304670BDB5F828319B0746
:10C6200003D430462D680646F1E70121284600F084
:10C6300005F80028F5DAF5E70646ECE7F8B54368B3
:10C6400005460F46002B3EDBB0F828319B073AD554
:10C6500000F02EF9AC69FCB12E6AB44207D128462D
:10C6600000F046F92C6AAB69E41A2046F8BD6B6A03
:10C670009C4226D1361B32462146686803F02EFFC5
:10C6800000280DDA95F82A3143F0020385F82A31A3
:10C69000F4F788FF04686442284600F029F9E4E7CB
:10C6A0000444361A0FB1002EE5DCAB6926442B6238
:10C6B000B442D4D02B6A5A1C2A6214F8012B1A7087
:10C6C000F6E70024E8E76FF00804CEE710B504466B
:10C6D00030B9F4F767FF092303604FF0FF3010BD56
:10C6E0008369E3B100F0E4F8606AA269904213D074
:10C6F000236A94F82B111B1A2046C4E90822002251
:10C70000591A84F82B210122FFF729FE002803DAA9
:10C71000204600F0EDF8E0E7204600F0E9F80020C0
:10C72000DDE7826932B1B0F828319B0702D50121DB
:10C73000FFF784BF0020704770B591F82A31054695
:10C740000C465B071BD5064616F8013B0BB9401B90
:10C7500007E022460121FFF7B7FE002802DC4FF078
:10C76000FF3070BD16F8013C0A2B01D03046EAE7D5
:10C7700001212046FFF762FF0028F7DAEFE700F01B
:10C7800034FB0028EDD0014622462846FFF79CFEE8
:10C7900040EAE070E5E70EB403B503AA52F8041BC3
:10C7A000019200F005F802B05DF804EB03B07047A9
:10C7B00070B586B0044616460D46014601A800F045
:10C7C000DBF9204600F074F82946324601A8FEF74E
:10C7D000A9FF0546204600F08BF8284606B070BD3C
:10C7E00008B5F5F781F9002803DABDE80840F4F749
:10C7F000D9BE08BD38B50122044600215430FEF7E9
:10C800008EFE4FF0FF35002304F15C002566C4E97D
:10C81000FB3300F03CF804F5C670C4F8905100F00A
:10C8200036F804F52F70C4F8C052BDE8384000F067
:10C830002EB838B504465430F5F756F90023C4F83D
:10C84000F033D4F8EC536DB904F16400FFF7C8FF7E
:10C8500004F5CA70FFF7C4FF04F53170BDE8384035
:10C86000FFF7BEBF284650F8083BC4F8EC33FFF78B
:10C87000B7FF2846FEF7F0F9E3E710B50446204677
:10C88000F5F782F90028FADB10BDF5F7D9B908B53C
:10C8900000214FF0FF330122083081818360FEF7D1
:10C8A0003EFE002803DABDE80840F4F77BBE08BD71
:10C8B00070B5044609F0C4FE05462369984203D1C9
:10C8C000A38A0133A38270BD04F108063046F5F750
:10C8D0005BF9031E07DAF4F765FE0368042BF5D055
:10C8E0008C2BF3D05B42002BEDD101232561E9E7CE
:10C8F00010B5044609F0A4FEA38A012B0ED1002333
:10C9000004F10800A3824FF0FF332361F5F798F993
:10C91000002805DABDE81040F4F744BE013BA382CD
:10C9200010BD0A22002100F000B873B50C4616466F
:10C93000019090B301A800F05FF9019B1D782D2DA7
:10C9400001D02B2D12D1013301933246214601989B
:10C9500000F025F82D2D0FD1B0F1004F08D9F4F7D4
:10C9600021FE222303604FF0004003E00025ECE7A6
:10C97000F9D0404254B910E0002805DAF4F712FE6D
:10C98000222303606FF000403CB135B1236813F8F7
:10C99000012CAA4201D1013B236002B070BD2DE9F8
:10C9A000F04385B00E4615460446019000284FD04E
:10C9B00001A800F021F9019B1F782D2F01D02B2F0A
:10C9C00019D101330193284601A900F045F8051E4D
:10C9D00013DAF4F7E7FD00241623036076B33FB1C2
:10C9E000019B13F8012CBA4204BF03F1FF330193FA
:10C9F000019B336022E00027E5E74FF0FF38002479
:10CA0000B8FBF5F805FB08F96FEA0909019B03AAD1
:10CA10002946187800F0CAF858B1444503D8039B5A
:10CA200010D199450EDAF4F7BDFD4FF0FF34222303
:10CA300003602D2FD2D16442002ED1D1204605B003
:10CA4000BDE8F08304FB0534019B01330193DDE76E
:10CA50000029CDD10C46F1E770B502460D460C68B1
:10CA6000A8B92378302B24D16378661C03F0DF0348
:10CA7000582B04D11021A07800F098F820B9344642
:10CA8000082210462C6070BD02341022F9E71028ED
:10CA900009D12378302BF4D1637803F0DF03582BCE
:10CAA000EFD10234EDE7831E182BEAD94FF0FF30A7
:10CAB000E9E70A22E5E738B5C36805464469E41AA0
:10CAC000944228BF1446002C0ADD0069224618440F
:10CAD000F4F786FBEB682A6900212344EB60D1540C
:10CAE000204638BD07B501228DF807100DF107016A
:10CAF000FFF7E1FF03B05DF804FBFFEC064B013AE2
:10CB00000360064B42614360054B83600023C0E92C
:10CB100003310B70704700BFE5CA0208B7CA0208AC
:10CB200045CB0208C3680133C3607047034B036001
:10CB3000034B83600023C360704700BF25CB02080E
:10CB400045CB02080020704701210069FFF776BD40
:10CB500038B504460D462169284600F010FC013026
:10CB600003D0E3680133E36038BDF4F71BFD0368CD
:10CB7000042BF0D0F8E7FFEC094B03608B6963B13D
:10CB8000B1F82831074A13F4807F074B08BF1346DA
:10CB900083600023C0E903317047024BF8E700BF10
:10CBA00051CB020845CB020849CB02080A290ADC0E
:10CBB0002F281EDD2F3181421BDBA0F13003012025
:10CBC00002B113607047242913DCA0F13003092B54
:10CBD000F3D9602805DD563181420ADBA0F1570305
:10CBE000EDE7402805DD3631814202DBA0F1370355
:10CBF000E5E700231846E3E770B5044605682E46CE
:10CC000001353078FEF7FFFA0028F8D1266070BDB4
:10CC100038B505460C4600F0E8F8611E2B1811F8EF
:10CC2000012F12B928461A7038BD03F8012BF6E718
:10CC300070B506460D460024315D19B1284600F056
:10CC4000A3F808B1204670BD0134F5E738B50546B4
:10CC500000F0CBF80130FEF707F8044610B1294682
:10CC600000F0A7F8204638BD30B57E210024094ADF
:10CC700063185B1012F83350854204DA5C1C8C4256
:10CC8000F6DD054805E001DD591EF8E702EBC302B9
:10CC9000506830BD28831708CB4316082DE9F041B2
:10CCA00005464E1E8718BD4202D10020BDE8F08126
:10CCB00095F80080404600F01DFB044616F8010F71
:10CCC00000F018FB201AF1D1B8F1000FEED00135B9
:10CCD000E9E7431E0A4410B5914201D1002007E064
:10CCE00013F8014F11F8010B201A01D1002CF3D1D8
:10CCF00010BD0346002010B51C4613F8012B8A42D4
:10CD000008BF2046002AF7D110BD2DE9F041884622
:10CD100016460446C0B1254629782C460135D1B1C6
:10CD2000404600F031F80028F6D129782F46013529
:10CD300039B1404600F028F80028F6D000233B70B7
:10CD40002F462EB1376003E012B11468002CE2D1F7
:10CD50002046BDE8F0810C46FAE7024401399042D2
:10CD600006D1002070474FF0FF300CE001200AE0B0
:10CD700010B5047811F8013F9C42F4D3F6D8013085
:10CD80009042F6D1002010BD03461A7818460133B0
:10CD90008A4202D0002AF8D110467047421E10B5D0
:10CDA00012F8014F11F8013BE01A01D1002CF7D124
:10CDB00010BD421E11F8013B02F8013F002BF9D1D2
:10CDC00070470B4610B562B913F8012B002AFBD14E
:10CDD00004E013F8014B00F8014B14B9581A01385C
:10CDE00010BD013AF5D10270EEE703461A46013351
:10CDF00011780029FAD1101A704710B50244044680
:10CE00000139904205D011F8013F00F8013B002B99
:10CE1000F7D1121A0021F4F74EFB204610BD02464E
:10CE2000014410B58A42134603D01C780132002C0D
:10CE3000F8D1181A10BDFFEC30B50C4B0025D3E922
:10CE400000428A4208D0A14206D0013508331F2D86
:10CE5000F5D10C464FF480528368C46123F48053AB
:10CE600023F00F0313438360002030BD2087170891
:10CE7000C06970472DE9F74304460F461E460D462C
:10CE80001078002840F0BA80002D00F3BC8003B079
:10CE9000BDE8F083252804D00132013D04F8010BE0
:10CEA000EEE7537802F10208252B27D0413BDAB296
:10CEB000382A00F2A180382B00F29E80DFE803F0D0
:10CEC0002D373C9C9C9C9C47499C9C9C6E9C9C80C8
:10CED0009C9C909C9C9C9C9C979C9C9C9C9C9C9CA3
:10CEE00021329C42449C9C329C5062646B1D9C701D
:10CEF0009C9C84929C9C9C9C94000A2301202370FF
:10CF00005AE0B369062B77DC404A52F82330404A96
:10CF100029462046FEF7C9FB4EE0B369062B6BDCC1
:10CF20003C4AF2E733690B2B66DC3B4AEDE7336999
:10CF30000B2B61DC394AE8E77269642392FBF3F357
:10CF4000374AE5E7F368FBE7F368364AE0E7B3689A
:10CF5000F6E7B3680C2293FBF2F102FB1133EFE723
:10CF6000D6F81090B9F10B0F46DC706900F076F836
:10CF7000011E484618BF012100F064F8F3682A4AF0
:10CF80000344C5E7B368E0E7B3680C2293FBF2F112
:10CF900002FB1133D9E733690133D1E77368CFE777
:10CFA000B168224B224A0B29C8BF13462046184AB3
:10CFB0002946FEF77AFB022004442D1A42465FE719
:10CFC000B1681C4B1C4AEEE7304600F072F80023B3
:10CFD00000902946194A20460193FEF766FBEBE7CD
:10CFE0003368ADE7092389E773696422B3E773699E
:10CFF000134A03F26C738BE70020DDE7002D3FF747
:10D0000049AF002043E72070781B40E79488170859
:10D01000348C160878881708488817081888170865
:10D020004D4F16080B591708524F16084A4F16084D
:10D03000EA881608CBA01608647A1708574F160816
:10D040005B4F16080346044A012B32F8100001DD3D
:10D0500001B10130704700BFB08817084FF4C871A4
:10D06000034690FBF1F201FB12025AB1642290FBDD
:10D07000F2F002FB103030B113F0030F0CBF0120AF
:10D08000002070470120704710B504464069D4E97C
:10D09000032100F26C7000F020FAA36818223C21F2
:10D0A00002FB00326368206801FB023301FB0300CE
:10D0B00010BDFFF7E9BFFFEC2DE9F04F454B4FF4F2
:10D0C0006162066885B00C4640F26D17B6FBF3F559
:10D0D00003FB1563B3FBF2FB02FB1B333C22B3FBE8
:10D0E000F2FA02FB1A3301933B4BB6FBF3F640F224
:10D0F000B55303FB1655B60006F2B270FFF7AEFF4C
:10D1000000280BBF4FF000094FF001093B464FF4D8
:10D11000B7739D4247D206F2B273002700930B23E8
:10D1200007EB0308494603934FEA680808F1010238
:10D1300010460292FFF786FF8542DDE9022344D2C2
:10D1400049464046FFF77EFF854240D208F1FF3353
:10D150009F42E5DB0135494638464636FFF772FF08
:10D16000019B2D1A009A2360791C2846C4F804A05C
:10D17000C4E90476C4E902B500F0CAF9A0610098D8
:10D180002669FFF76BFF011E304618BF0121FFF72C
:10D1900059FF28440023E0612046A362C4E9083314
:10D1A00005B0BDE8F08F06F2B370ED1A06F1010884
:10D1B000FFF754FF002846460BBF4FF000094FF021
:10D1C00001093B464FF4B773A3E71746C0E747464C
:10D1D000C0E700BF80510100801F8607FFF76CBFCA
:10D1E000002307B5CDE9003300F02AFA03B05DF85B
:10D1F00004FB08B500F0D9FA08BD08B500F0D5FA6F
:10D20000083008BD1FB5044610B9002004B010BD99
:10D210000021009002AB6A460846019109F06CF9C2
:10D220000028F2DA02988442F0D9034B039A9A421A
:10D23000C8BF0130EAE700BFFF64CD1D07B578B174
:10D24000094AB0FBF2F302FB13006A4600934FF465
:10D250007A735843002301901946184609F04CF997
:10D2600003B05DF804FB00BF40420F0030B591B041
:10D27000054601A903F07EF8041E0BDB039B03F4B3
:10D280007043B3F5804F08D0F4F78CF91423036092
:10D290004FF0FF34204611B030BD2846002100F089
:10D2A0008CF805460028F3D0F4F7A4FB0B4808F0EF
:10D2B000F9FD0B4B0122002814BF0146194609480D
:10D2C000F5F704FC012229460448F5F7FFFB044664
:10D2D0002846FDF7C1FCF4F79DFBDBE73A50160842
:10D2E0007ADA16083750160808B5FDF775FF00B151
:10D2F000006808BDA0F16103192B98BF2038704762
:10D300002DE9F0410A4D2B6843B90A4C0A4E0B4FE8
:10D31000DFF82C80B44203D101232B60BDE8F081FB
:10D3200054F8043BBB42F5D34345F3D29847F1E7A9
:10D330003450002478111C089C121C0800000208BC
:10D3400078111C080368002223B932B11160002350
:10D350000B6070471A461B68F6E70160F7E707B5F0
:10D36000024601210DF1070000F05AFA0028CCBF57
:10D370009DF807004FF0FF3003B05DF804FB37B5B0
:10D380000A468DF8070004460D460DF107000121FD
:10D39000FFF79AF800280BDD0A2C0BD195F82A31FB
:10D3A0005B0707D501212846FFF748F9002801DA75
:10D3B0004FF0FF34204603B030BD2DE9F04F0D464D
:10D3C00091B0064638B9F4F7EDF816230360002053
:10D3D00011B0BDE8F08F04781CB9F4F7E3F802232C
:10D3E000F4E749B94FF48070FDF73EFC804630BB4E
:10D3F000F4F7D8F80C23E9E74FF000082F2C0BD0F6
:10D400004FF48071284600F0D5F9002840D0284616
:10D41000FFF7EBFC012814D82C464FF02F0B4FF0F0
:10D42000000A33782F2B0ED083B9A542284602BFBD
:10D430002C462F2304F8013B00232370C8E7054640
:10D44000DCE72C18E9E7771C3E46EAE73746B946A1
:10D4500017F8012F2F2A01D0002AF8D12E2B0DD139
:10D46000BB1B012BF0D072782E2A07D1022B05D1DD
:10D47000A542E9D014F8013D2F2BFAE7631B0133D5
:10D480003B449B1BFF2B07DDF4F78CF85B23036009
:10D490004046FDF7E1FB9AE709F102092046BA1B75
:10D4A0003146A9EB060900F801BBF3F799FE01A983
:10D4B0004C44284684F800A002F06AFF0130E7D00F
:10D4C0003B782F2BC0D1039B03F47043B3F5804FFF
:10D4D000BAD0F4F767F81423D9E770B50E461446AE
:10D4E0000546FFF7BBFD011E304604F1FF3418BFAF
:10D4F0000121FFF7A7FDA5F2B27340F26D1202FB06
:10D5000003446FF4F6631D4404EBA504204470BD8E
:10D510000229DCBF02F1FF320C31002A02EB0003CA
:10D520001046A1F10201B8BFD01CC1EB411103EBC1
:10D53000A0036FF0630092FBF0F003444FF4C87057
:10D5400092FBF0F213440C22072091FBF2F10B4402
:10D5500093FBF0F0C0EBC000181A70472DE9F043C0
:10D56000002A68D0D0F810900027D2F800E01646C4
:10D57000BEF1000F03D199F80030C3602DE04C4696
:10D5800014F8018B1EF801CBB8F13D0F14BF4546CE
:10D590000025B5EB0C0C1DD1002DF1D1B8F13D0FDC
:10D5A00002F1100218BF0024002D42D1BCB18268E4
:10D5B000056101328260726872B1013A012A3AD87B
:10D5C0000460D6E902200AB11060002003B11F6098
:10D5D000BDE8F0836546E1E705603F20F8E7726843
:10D5E000012A13D0022A05D02ABB826804610132C5
:10D5F0008260E6E78268013251F8224014B1247853
:10D600002D2C03D1002101610160F1E78268002423
:10D61000551C51F8251021B191F800C0BCF12D0F17
:10D6200003D1046104608560D7E7023204610160C0
:10D63000DEE7013799E7002303754FF0FF30C7E7B6
:10D640002DE9F84F0A9E8146884617469A469DF86E
:10D650002CB000F0AAF80446C0B1B8F1000F1FD0FA
:10D660008368002B01DD037D3BB9002201233F21AC
:10D67000226022612375C4E9023125695DB12B78EE
:10D6800033B13A2B1ED10135E36025613F250BE014
:10D69000A3680133A360A3684B4508DB0023236123
:10D6A00000234FF0FF3523752846BDE8F88F58F862
:10D6B000231021610029F3D00B782D2BF0D10131FB
:10D6C0002161DAE71BF0010F6CD02D2B10D1013551
:10D6D00033465246414625612046FFF73FFF3F282B
:10D6E0000546E1D1A3680133A36000232361DBE792
:10D6F0001BF0020F3FD03346524641462046FFF70B
:10D700002DFF3F280546CFD1236913B15B78002B4D
:10D7100031D0A3680133A36000232361B6E7C4E9D5
:10D720000337A3680133A360B0E743783A2B03D0F3
:10D73000013626610578B7E7A36877785A1C2FB1C0
:10D7400001360023A26026602361F3E758F8221017
:10D7500039B10E782D2E04D0023321602761A360E9
:10D76000E8E70023236123600378C4E90223837878
:10D770003A2B99D1DEE723691B78002FCFD03D7873
:10D7800026693A2D96F800900CBF01373F2549468F
:10D790003846FFF7F9FA0028C7D10136C4F80C90D3
:10D7A000266173E7002FEAD17AE708B5F3F7E9FEBF
:10D7B000203008BD70B50D46044638B159B9F3F7AD
:10D7C000F1FE162300240360204670BD40F20113D1
:10D7D000002908BF1D46104808F064FB0F4B0028C5
:10D7E00014BF06461E463046FFF7FFFA0130A84236
:10D7F00003D9F3F7D7FE2223E4E744B92846FDF71F
:10D8000033FA044618B9F3F7CDFE0C23DAE73146B4
:10D810002046FFF7CEFAD7E73A5016087ADA16080C
:10D82000F8B506460F461446F2B1B2F82831DB07C8
:10D830001AD53D461046FFF73BF894F82B3103B15B
:10D84000ADB9A369002B60D02046FEF76AFF00281F
:10D850002EDAAF425CD194F82A31204643F002031D
:10D8600084F82A31FFF744F84FF0FF301CE0013B09
:10D87000013DDBB284F82B31234493F82C3106F8B8
:10D88000013BDAE75A1C013D22621B7806F8013B96
:10D8900018D194F82A3103F0FE030025204684F8BD
:10D8A0002A31FFF725F8781BF8BD31D006442D1A30
:10D8B00045B9EEE702F028FB002815DB28D0636AA3
:10D8C00003446362D4E908329342DBD3A169E2697D
:10D8D0006068521A9542C4E90811EBD92A463146CC
:10D8E00002F012FB0028E0DABD42B4D094F82A31ED
:10D8F00043F00103D2E72A463146606802F004FB98
:10D900000028F1DB04D006442D1A002DF3D1C0E726
:10D9100094F82A31002DBED0E8E7034603F17F4397
:10D9200003F1FF1313B508460B2B37D8DFE803F0DC
:10D9300006363612363636153636281F24F15EFF87
:10D94000002804461DDA6442F3F72CFE04604FF011
:10D95000FF3416E024F1F8FFF2E711B300220B893F
:10D9600000924A680078C96800F0C0F8E8E70B78D0
:10D97000012B16D14B78012B06D0022B09D083B98D
:10D980000024204602B010BD4968807801F096FB63
:10D99000D6E74B68186801F00BFCF1E76FF018044C
:10D9A000D1E76FF01504CEE708B500F039FEBDE809
:10D9B000084000F013B8002070471046704708B5C3
:10D9C0004AB14B688A6803F0050313438B6013B1B7
:10D9D0000869F4F7E7F8002008BDFFEC00234FF4D6
:10D9E000DB720249024802F013BF00BFCC8817085F
:10D9F0003E501608426900209379013393717047B5
:10DA000061B14369012200200A80DA7902F0010243
:10DA10008A701A684A609B880B8170476FF0150006
:10DA2000704740F20153994205D122B14369002069
:10DA30009B68136070476FF01800704710B5446919
:10DA4000E37943F00403E371A3792BB9A068FDF7F0
:10DA500003F92046FDF700F9002010BD38B51C463B
:10DA600043691546DA79D2070FD51A68AA420FD949
:10DA7000281982420CD398889B6800FB04F200FBB3
:10DA80000530F3F7ADFB204638BD6FF00C00FBE727
:10DA90006FF01A00F8E770B506461C4615460846B2
:10DAA00073691A68AA420CD929198A4209D399883C
:10DAB0009B6801FB04F201FB0531F3F791FB204663
:10DAC00070BD6FF01500FBE710B54469A379013B09
:10DAD000DBB2A37143B9E3795B0705D5A068FDF715
:10DAE000BBF82046FDF7B8F8002010BD2DE9FF4136
:10DAF00005460C200E4690461F46FDF7C5F8044625
:10DB0000E8B19DF8283010210E4A03F00303C0F855
:10DB100000808780C3712B4686606846FDF7C5FD8F
:10DB2000234600220849684602F0A1FE051E02DADB
:10DB30002046FDF791F8284604B0BDE8F0816FF06B
:10DB40000B05F8E748501608EC88170870B504462E
:10DB50000D46E36D2046DB6A98470028F9D0E36D57
:10DB6000294620465B6ABDE8704018472DE9F74F0B
:10DB7000858F0446B0F9403088462DB24FF08009B9
:10DB800001920135AB42D8BF0025E28F12B2AA4202
:10DB90000AD0A38F2DB2626C00201BB202F8038062
:10DBA000A58703B0BDE8F08F019B002B30D0EFF3C9
:10DBB000118AEFF3108772B689F3118887F3108802
:10DBC000E28F12B2AA421ED1E27802F0FF0BE2B954
:10DBD0000121E26D20466170926A904704F11C00B9
:10DBE000F3F790FFE26D06465946926A2046904749
:10DBF0005FFA8AFA8AF31188E27862B9002EC4DAF1
:10DC00006FF00300CDE70026F2E76FF07F06EFE745
:10DC10006FF00A00C5E76FF07F00C2E72DE9F74F0C
:10DC2000836881460E4601925C6904F148073846D4
:10DC3000F3F768FF051E2FDB00254FF0800B019BDB
:10DC40009D4204D2E3785BB30DB96FF07F05E36DBD
:10DC5000012120469B699847B4F85020B4F852300F
:10DC600012B21BB29A42B4F95420C0F29E80B4F8AA
:10DC70005010B4F8523009B21BB2C91A0A2392FBF1
:10DC8000F3F2914205D8E36D1B6A13B100222046DE
:10DC900098473846F3F786FF284603B0BDE8F08F73
:10DCA000B4F85230B4F8502019B212B28A421FD0E0
:10DCB000A26D0133525C1BB2B4F954109942D8BF23
:10DCC0000023A4F85230A36813F4E07F05D00A2A99
:10DCD00007D113F0400F18BF0D22013506F8012BB4
:10DCE000ADE70D2AF9D113F4807F18BF0A22F4E7BB
:10DCF000002DACDCD9F80830002B50D0D9F800103A
:10DD000011F040014ED1EFF3118AEFF3108872B693
:10DD10008BF3118888F31088E26D20465FFA8AFA47
:10DD200092699047B4F85010B4F8522009B212B278
:10DD300091422CD1E26D0121204692699047B4F8BE
:10DD40005010B4F8522009B212B2914202D08AF3B4
:10DD5000118874E7E278BAB9012204F12400A270B4
:10DD6000F3F7D0FE8AF31188002803DBE378002B59
:10DD70003FF465AF002D7FF46AAFE378002B7FF4AA
:10DD800064AF6FF0030562E76FF07F00EAE78AF3A4
:10DD90001188E36D012120469B6998474FE76FF09A
:10DDA000500554E76FF00A0551E7B4F85230B4F863
:10DDB00050101BB2D31A03FA81F15FE72DE9F0414D
:10DDC00083685E6906F114052846F3F79BFE041E7E
:10DDD00023DBF378002B36D13378013313F0FF07C0
:10DDE00034D0012F2DD1EFF3118800238022EFF3DF
:10DDF000108372B682F3118883F3108833795FFA47
:10DE000088F86BB9F36D30461B689847041E07DA33
:10DE100088F311882846F3F7C5FE2046BDE8F08157
:10DE2000F36D30469B689847041EF36D03DA5B6818
:10DE300030469847ECE79B6901213046984788F3C4
:10DE400011883770E6E76FF07F04E3E76FF017049F
:10DE5000E0E7F7B50E4600F1600700F1700557F8EE
:10DE6000044F8CB16368A26843F018033340134336
:10DE7000A3604BB101A92069FDF75EFB019B002B5C
:10DE800002DC2069F3F78EFEAF42E8D103B0F0BDAB
:10DE90002DE9F84383680E4615465C6904F12C08A9
:10DEA0004046F3F72FFE071E4ADB002D52D004F147
:10DEB0006002002352F8045F002D37D104EB830287
:10DEC000193304F1340904EB830356664846736141
:10DED000F3F752FEA38FB4F940201BB201339A42EC
:10DEE000D8BF0023E28F12B29A422CD1484604F1E7
:10DEF0004809F3F757FE4846F3F73EFEB4F85020C2
:10DF0000B4F85230484612B21BB29A421EBF736830
:10DF100003F001031D43F3F745FEE378BBB145F081
:10DF2000180529462046FFF794FF06E00133042B2D
:10DF3000C0D100236FF00F0773614046F3F732FE44
:10DF40003846BDE8F883756805F00405CEE7002D76
:10DF5000F3D0E6E77369002BEFD01D607561ECE745
:10DF60002DE9F047836880460F4616465D69464BAB
:10DF70001B6823B1EB78ABB16FF07F0425E0F3F7BA
:10DF800077FD0028F6D105F1340A5046F3F7BAFDC3
:10DF9000041E1ADBEB7803F0FF018BB35046F3F756
:10DFA00001FEE9E7EFF3118400238022EFF31083F1
:10DFB00072B682F3118883F3108807EB0608B84520
:10DFC00006D1E4B284F3118834462046BDE8F087D8
:10DFD000EB6817F8011BD80703D50D2905D11A07DF
:10DFE00005D42846FFF7B2FDE9E70A29F9D113F075
:10DFF000240F03D00D212846FFF7A8FD0A21F0E7E2
:10E00000D8F80030B146284683F04008EB6DC8F3DD
:10E0100080189B6A9847B9F1000F01D1344623E07C
:10E02000EB6817F8011BD80703D50D290AD11A0789
:10E030000AD442462846FFF799FD041E10DB09F179
:10E04000FF39E8E70A29F4D113F0240F01D10A219E
:10E05000EFE742460D212846FFF788FD041EF6DA59
:10E06000B14501D2A6EB0904AA8FEB8F12B21BB205
:10E070009A4204D0EB6D012128469B6A984750468E
:10E08000F3F790FDA1E700BFC41000242DE9F0478D
:10E0900000F1340804460E464046F3F733FD051EF2
:10E0A0001DDBEFF3118700238022EFF3108372B69C
:10E0B00082F3118883F31088E37803F0FF0553B3EC
:10E0C000A38F6FF07F05E387FFB287F311881E4FA0
:10E0D000002DD7F800902CDA4046F3F763FD284670
:10E0E000BDE8F087E36D0121204684F801A09B6A1A
:10E0F00098474846F3F706FDE36D054600219B6A05
:10E1000020469847002DDFDBA28FE38F12B21BB2AF
:10E110009A42E7D1D8E74FF0010A04F11C09F3E76E
:10E120004FF47A7008F01EFA3B68A3EB0903B34280
:10E1300006D2E36D20461B6B98470028F0D0CBE752
:10E140006FF07305CBE700BFAC1900242DE9F04157
:10E150000B7905460C462BB10B6943F001030B61AB
:10E160000523CB600122002104F1340004F11C07D7
:10E17000FDF7C7F90122002104F14800FDF7C1F9BC
:10E180000122002104F11400FDF7BBF900223846FA
:10E1900004F124061146FDF7B4F900223046114679
:10E1A000FDF7AFF90122002104F12C00FDF7A9F9D8
:10E1B00000213846F4F780FF00213046F4F77CFF59
:10E1C000234628464FF4DB720249BDE8F04102F0D5
:10E1D0001FBB00BF0889170810B504460121FFF7CF
:10E1E00038FEA3783BB1002304F12400A370BDE8FE
:10E1F0001040F3F7D7BC10BD10B504460421FFF75B
:10E2000028FE63783BB1002304F11C006370BDE875
:10E210001040F3F7C7BC10BD70B583680E461546B5
:10E220005C69E36D1B695BBB40F207339E422ED0F5
:10E23000B6F5427F1CDAB6F58A7F00F08E8040F298
:10E2400015139E4200F0AD806FF0180040F20113EC
:10E250009E4200F0B280B6F5817F37D1002D00F0EC
:10E26000B4802B68A3606B68E360EB6823612CE0EB
:10E2700037D040F209339E424FD06FF0180025E0AE
:10E28000984710F1190FCFD00028DFD01EE0EFF330
:10E29000118100238022EFF3108372B682F311887C
:10E2A00083F31088B4F85220B4F8503012B21BB285
:10E2B0009A420CDCB4F85030B4F852201BB212B2BF
:10E2C0009B1ACAB282F311882B60002070BDB4F88B
:10E2D0005220B4F8500012B2B4F9543000B2121AFD
:10E2E000EEE7EFF3118100238022EFF3108372B683
:10E2F00082F3118883F31088E28FA38F12B21BB2CE
:10E300009A4203DCA38FE28F1BB2D8E7E28FA08F83
:10E3100012B2B4F9403000B2E1E7EFF3118100230B
:10E320008022EFF3108372B682F3118883F3108892
:10E33000A28FE38F12B21BB29A4206DAE38FA28F4A
:10E340001BB212B29B1A013BBBE7A28FE08F12B245
:10E35000B4F9403000B2121AF4E7EFF3118600234B
:10E360008022EFF3108372B682F3118883F3108852
:10E3700035F0020209D1B4F85030A4F85230E36D00
:10E380001B6A13B1114620469847013D012D04D860
:10E39000A38F2046E387FFF72FFFF6B286F311889D
:10E3A00093E742F210712046FFF770FE00288CD0F0
:10E3B00010F1190F3FF461AF88E735B1A3682B6006
:10E3C000E3686B602369EB607FE76FF015007DE722
:10E3D00070B504460D46EFF3118600238022EFF35B
:10E3E000108372B682F3118883F3108881F00103E1
:10E3F000C37089B91821FFF72CFD637823B104F1AC
:10E400001C006570F3F7CEFBA3782BB1002304F159
:10E410002400A370F3F7C6FBF6B286F3118870BD33
:10E4200010B5044600211C3007F0C6FF002104F19E
:10E43000240007F0C1FF012104F1340007F0BCFF04
:10E44000012104F1480007F0B7FF04F12C0001217D
:10E45000BDE8104007F0B0BF70B5836805465C6941
:10E4600004F114063046F3F787FB2378012B06D915
:10E47000013B23703046F3F795FB002070BD00216F
:10E48000E36D204621709B6998472B685B0604D496
:10E490004FF47A612046FFF7F9FDEFF31185002371
:10E4A0008022EFF3108372B682F3118883F3108811
:10E4B000E36D2046DB68984723791BB9E36D20465E
:10E4C0005B689847EDB285F311882046FFF784FE1C
:10E4D0002046FFF7A5FFCDE770B5002504462E4680
:10E4E000A28FE38F12B21BB29A4211D1A28FE38F97
:10E4F00012B21BB29A4204D1E36D002120469B6AFE
:10E500009847ADB2EDB12046BDE87040FFF774BE4C
:10E51000E36D2046DB6A98470028E7D0E38F20466A
:10E52000616C1BB2E26DC95C526A9047E38FB4F92B
:10E53000402001331BB29A42E38700DCE6870135B5
:10E54000CEE770BD2DE9F341B0F850505A23B0F931
:10E55000546004462DB200270135AE42D8BF0025D5
:10E5600016FB03F6642396FBF3F6E36D2046DB69A6
:10E57000984700283FD0B4F85280B4F85020B4F83F
:10E5800052300FFA88F812B21BB29A4220DBB4F86C
:10E590005010B4F8523009B21BB2C91AB142E36D3F
:10E5A00021D2E36D01A920465B6998474545DCD03F
:10E5B000B4F850300137A26D1BB2D0542BB20135E4
:10E5C000A4F85030B4F95430AB42D8BF0025CCE7A2
:10E5D000B4F85220B4F9543012B2B4F850109B1A67
:10E5E00003FA81F1DAE71B6A002BDAD00122204618
:10E5F00098470028D5D0BFB217B12046FFF7ECFDF1
:10E6000002B0BDE8F081FFEC08B5044B186818B102
:10E6100003689B6803B19847002008BD08000024E8
:10E62000002070477047036E93F87830002B0CBFC2
:10E630006FF07F0000207047704700207047002077
:10E640007047036E93F87900032894BF00200120DF
:10E65000704770B5036805460E469B6898470446A8
:10E6600050B1C6803046FCF7FFFA206028B92B680D
:10E6700021462846DB6898470024204670BD806804
:10E6800090F8783013B10121FFF7A2BE7047002146
:10E690008068FFF79DBE10B5836840F20930814263
:10E6A0005B6900F0B08011DC40F20730814265D038
:10E6B000B1F5427F00F08B8040F20110814229D0F9
:10E6C000B1F5817F51D06FF018000EE040F6025096
:10E6D00081420BD040F60350814214D040F60150E5
:10E6E0008142F0D1C3F88820002010BD002A00F03C
:10E6F000AB80D3F87E101160B3F88210918093F84C
:10E7000084309371F0E7002A00F09E8093F87C300B
:10E710001360E9E7002A00F0978099681160D968D2
:10E7200051601969D16093F88310E1B101F1FF3EA6
:10E73000DEF1000141EB0E0148024FF4807193F8C5
:10E7400082400843A4F1020CDCF1000444EB0C0409
:10E7500040EA841040F0300090601046D3F87E10FC
:10E76000FEF76AFBC0E70846E9E7002A6CD01168AB
:10E7700099605168D960D2681A61B5E7EFF31180EA
:10E7800000218024EFF3108172B684F3118881F3A5
:10E790001088B3F85240B3F8501024B209B28C423A
:10E7A00007DCB3F85010B3F8523009B21BB2CB1AE1
:10E7B00009E0B3F85210B3F8504009B2B3F954303D
:10E7C00024B2091B5B1AC1B281F31188A0E7EFF3F1
:10E7D000118000218024EFF3108172B684F3118838
:10E7E00081F31088DC8F998F24B209B28C4203DC4C
:10E7F000998FDB8F09B2D9E7D98F9C8F09B2B3F912
:10E80000403024B2DDE7EFF3118000218024EFF3E4
:10E81000108172B684F3118881F310889C8FD98F90
:10E8200024B209B28C4206DAD98F9B8F09B21BB28F
:10E83000CB1A013BC7E7998FDC8F09B2B3F940309F
:10E8400024B2091B5B1AF4E76FF015004DE770B5B1
:10E850000D46044658B151B1086808B1FCF7FCF9FF
:10E86000236829462046DB68BDE87040184770BD24
:10E8700010B590F878300446ABB1002180F87810DC
:10E88000FFF7A6FDD4F88C0003685B689847D4F8BE
:10E89000900003685B689847D4F894000368BDE86B
:10E8A00010405B68184710BD70B50C468568EFF3E3
:10E8B000118600238022EFF3108372B682F3118851
:10E8C00083F3108800212846FFF782FD2846FFF7D2
:10E8D000CFFF0023F6B2AB87EB8786F3118823685E
:10E8E0005B6923B120460121BDE87040184770BD27
:10E8F0002DE9F04184680D46002C52D02046FFF7E8
:10E90000B7FF3220FCF77AF9D4F88C1031B12B68BC
:10E9100028465B6898470023C4F88C30D4F89810D8
:10E9200029B16868FFF793FF0023C4F898302646A2
:10E9300004F130074FF00008D6F8081129B1D4F8D7
:10E940009400FFF784FFC6F808810C36BE42F3D16D
:10E95000D4F8941031B12B6828465B68984700239F
:10E96000C4F89430EFF3118600238022EFF3108374
:10E9700072B682F3118883F3108804F1AC08D4F8DE
:10E98000AC7087B9F6B286F31188D4F8901029B12B
:10E990002B6828465B689847C4F890700023A387CB
:10E9A000E387BDE8F0814046FCF742FD416800295D
:10E9B000E5D0D4F89000FFF74AFF94F87930013B96
:10E9C00084F87930DBE7FFEC2DE9F84F84680D46D9
:10E9D000804661674B6840219C606868FFF739FE9C
:10E9E000C4F8980000287ED0404B0122C36028461E
:10E9F0002B6894F8D0101E68032341F08001B047C3
:10EA0000C4F88C0030B96FF0120429464046FFF775
:10EA10006FFF65E0846001222B68284694F8D410CB
:10EA20001E68022341F08001B047C4F8900000281E
:10EA3000E9D0846000222B68284694F8D8101E681C
:10EA40000223B047C4F894000028DCD004F5827695
:10EA500004F59A7A4FF0000B8460B1464021D4F857
:10EA60009400FFF7F6FD706000283CD0A6F808B0CF
:10EA700006610C3656F8082C1D4B5645D360EDD177
:10EA800004F1E4064FF0800A6021D4F89000FFF70B
:10EA9000E0FD706038B30661164A7368DA60EFF320
:10EAA000118BEFF3108772B68AF3118887F3108801
:10EAB00004F1AC013046FCF787FC94F879205FFA4A
:10EAC0008BF3013284F8792083F3118808364E45A0
:10EAD000DAD12B685B6913B10121284698470024DD
:10EAE0002046BDE8F88F6FF00B048EE725E602089C
:10EAF00007EF020871F0020837B5044615460846CC
:10EB00001A466946002300F0AFFB23682A4669468F
:10EB10001B682046984703B030BDFFEC2DE9F0415B
:10EB200090F8783004460E468B4249D0FFF7A0FE9D
:10EB3000002E45D0012E4BD1002204F1BC07D4F8A1
:10EB40008C003B461146FFF7D7FF051E3CDBD4F88F
:10EB50008C30002202219C603B46D4F89000FFF7E5
:10EB6000CBFF051E30DBD4F89030324631469C6036
:10EB70003B46D4F89400FFF7BFFF051E24DBD4F812
:10EB80009430264604F13007DFF84C809C60D6F8BC
:10EB90000811C1F80C80D4F8940003681B699847E9
:10EBA000054688B994F87A300C360133BE4284F8B1
:10EBB0007A30ECD10121204684F87810FFF708FC68
:10EBC00000252846BDE8F0812046FFF751FEF8E712
:10EBD0006FF01505F5E700BF07EF02082DE9F843D0
:10EBE0000F46117884689E4611F060095388D4F866
:10EBF000985092F803809078B2F804C0D6887DD1FE
:10EC00005278063A052A00F2D380DFE802F003D1F9
:10EC1000423A654BB8F1020F26D0B8F1030F2CD061
:10EC2000B8F1010F40F0C4802C6800F019FB00F12E
:10EC30001002234650F8041B904243F8041BF9D1FC
:10EC4000028812201A8086424FF001032946A8BF8D
:10EC500006462B71EE80786803681B699847002888
:10EC600009DA00236B8106E004F1BC01286800F09A
:10EC700030FB0028E7DABDE8F883296800F0B4FA31
:10EC8000F7E7002940F09480D9B22046FFF746FF0D
:10EC9000EFE7802940F08C802B6894F878201A7078
:10ECA0000120D0E7012940F0838094F87820012AE0
:10ECB0007ED1D4F8C020944502D00132944577D15A
:10ECC000002B75D12046FFF7D3FD94F8781020462D
:10ECD000FFF724FF0020B6E7812969D194F8782056
:10ECE000002A65D1D4F8C020944502D00132944561
:10ECF0005BD1002B59D12A681370D1E7B9F1200FED
:10ED000056D15278203A032A52D8DFE802F0140292
:10ED10003242A1294CD1D4F8C0309C4548D1D4F816
:10ED20007E2007202B681A60B4F882209A8094F81D
:10ED300084209A7187E721293AD1072E38D1D4F857
:10ED4000C0309C4534D1BEF1000F0BD0DEF800304E
:10ED5000C4F87E30BEF80430A4F882309EF8063045
:10ED600084F88430D4F88830002BB3D00020984742
:10ED7000B0E721291CD1D4F8C020944518D103F064
:10ED8000030384F87C30D4F88830002BA2D0012013
:10ED9000EDE721290CD1D4F8C0309C4508D1D4F836
:10EDA0008830002B96D00220E1E76FF0200062E768
:10EDB0006FF05E005FE700230B81D0F89400496894
:10EDC000C388CB8003681B691847FFEC2DE9F04727
:10EDD0000446EFF3118800238022EFF3108372B60C
:10EDE00082F3118883F3108800F19C094846F3F7F9
:10EDF0006FFD94F87D30002B59D004F1B40AD4F89B
:10EE0000B4502DB95FFA88F888F31188BDE8F0870F
:10EE10006A6800212B89106817891844B4F95420B6
:10EE2000FF1AB4F850300133BFB29BB29342A8BF6F
:10EE30000023B4F852208EB212B2934212D116B10E
:10EE40002046FFF7C9F9B7422ED85046FCF7F0FA32
:10EE500029462046FFF7AFFFD1E7B4F85220B4F8B7
:10EE600050200DE0B742EAD9B4F85060B4F852200F
:10EE700036B212B29642F0DBB4F85020B4F8522009
:10EE8000B4F8506010F801C00131A26D36B202F83A
:10EE900006C01AB20133A4F850209BB2B4F9542032
:10EEA0009342A8BF0023C4E72B891E442E81D4F8C7
:10EEB000B430002BA6D02346024AC8214846F4F7B6
:10EEC00005FB9FE703EF020810B5006EEFF3118416
:10EED00000238022EFF3108372B682F3118883F34C
:10EEE000108859B190F87D3013B9012380F87D3036
:10EEF000FFF76CFFE4B284F3118810BD80F87D1039
:10EF0000F8E7FFF763BF38B584680869EFF3118548
:10EF100000238022EFF3108372B682F3118883F30B
:10EF20001088B1F90A3013F16E0F0CD08BB9038140
:10EF300004F1B401FCF748FA2046FFF747FFEDB2B1
:10EF400085F3118838BD94F87A30013B84F87A3023
:10EF5000F5E701462046FFF72EFFF0E72DE9F74FD2
:10EF60008346EFF311834FF0800A01930022EFF301
:10EF7000108272B68AF3118882F31088D0F89080DC
:10EF8000B8F80620602A38BF60220092DBF8AC7027
:10EF90007FB37D682868EFF31189EFF3108472B6B0
:10EFA0008AF3118884F310880021BBF83CC08EB22C
:10EFB000BBF83E200FFA8CFC12B2944502D0009BA5
:10EFC000B3421DD8BBF83C10BBF83E2009B212B2C8
:10EFD000914205D1DBF85C2000215846926A9047A7
:10EFE00016B15846FFF708F95FFA89F989F31188D5
:10EFF000EEB99DF8043083F3118803B0BDE8F08FBB
:10F00000BBF83E60DBF8442036B2925D4254BBF858
:10F010003E20BBF94060013212B29642ABF83E206E
:10F0200003DC4FF00003ABF83E300131BDE70BF1DC
:10F03000AC00FCF7FDF99BF8792029464046013ADF
:10F040008BF879200122EE802F612A71D8F80020F8
:10F0500012699047002899D0CBE741B1006E828FAA
:10F06000C38F12B21BB29A4201D0FFF777BF70472D
:10F0700070B50D4684680869EFF31186002380227D
:10F08000EFF3108372B682F3118883F3108804F1D2
:10F09000AC01F6B2FCF798F994F87930013384F8B2
:10F0A000793086F31188B5F90A3023B92046BDE8D6
:10F0B0007040FFF753BF70BD7047FFEC2DE9F04F74
:10F0C0008FB0242280460F4605A80021F2F7F3F9FD
:10F0D00004234FF0020A4FF0010B0693032343F27F
:10F0E0007820CDF810A0CDE9083BCDE90AA3FBF7C5
:10F0F000BBFD044638B96FF00B0507B13C602846EC
:10F100000FB0BDE8F08F43F26C2904AE002104F18A
:10F11000BC054A46F2F7CFF984F87B800FCE0FC5C5
:10F120000FCE0FC596E80300C2231E4A85E80300F0
:10F1300084F87F300823102184F880B084F884306C
:10F140004FF4167384F803B06846A4F8543004F5FD
:10F150009A73A36542F6E063A4F8403004F5637344
:10F160006364114BC4E9173404F5405383F870A26B
:10F17000C3F86C220D4AC3F874424346FCF795FA73
:10F1800021466846FEF7E2FF051E04DA2046002409
:10F19000FBF762FDB1E74C442046FBF755FB054603
:10F1A000ABE700BF5C891708288917085350160879
:10F1B00030B585B085680B4A102195F87B30044640
:10F1C0006846FCF772FA684601F043FB2046FBF7FD
:10F1D00055FB05F19C00F3F77BFB2846FBF73CFD54
:10F1E00005B030BD5350160870B50C4604282BD816
:10F1F000DFE800F01503211D1F00154D2846FDF71F
:10F20000F4FD0023A21C1946834202F1020214DB22
:10F210004000032302306370C0B2207006E0032375
:10F2200004204B70092308708B70C87070BD094DA5
:10F23000E4E7094DE2E7094DE0E7EE5C013302F84F
:10F24000011C02F8026CDFE76FF01500EEE700BF6B
:10F25000615016082C1917086C50160865501608CE
:10F260000048704774891708012813D002281FD05E
:10F2700068BB07230B7005234B705369487163F01B
:10F280007F038B700323CB7040230B710A238B7198
:10F290000720704707230B7005234B70D3698871D3
:10F2A0008B700223CB7040230B7100234B71EFE76F
:10F2B00007230B7005234B709369C87063F07F03BD
:10F2C0008B7040230B7100234B710123DFE700207B
:10F2D00070472DE9F0410D460446002800F0878074
:10F2E0000021042624274FF003080846FFF7F1FF0A
:10F2F0008023012102224FF0090EA070E371001259
:10F30000FA23A671E0704FF0100CA672052084F865
:10F3100000E0627022716171237284F809E06B6809
:10F3200084F815C04FF0060CE3720023A074E67554
:10F3300084F81AC04FF0070CE07684F81E8023731F
:10F340006173A273E27321746374E7742375A1750A
:10F3500027766276277761776F6884F820C00F443C
:10F3600084F82100E7776F6984F823804FF00A085A
:10F3700067F07F0784F8253084F8268084F82270AF
:10F38000402784F827E084F8247084F828606E68A9
:10F3900084F82A300E4484F82B2084F82C8084F8DA
:10F3A000296084F82D3084F82E3084F82F3084F8CA
:10F3B00030C084F83100EE6984F8332084F832607C
:10F3C00084F8347084F8353084F8361084F837C007
:10F3D00084F83800A86960F07F0084F8390084F868
:10F3E0003A2084F83B7084F83C3084F83D103E208D
:10F3F000BDE8F08100F0BEB9F8B5037A04460E46C8
:10F400008B4223D2CB00FF2B22D88900C068FBF7A8
:10F4100033FC074668B1257A8020FBF735FC47F8B6
:10F42000250070B9013D237AAB4205DD3846FBF774
:10F4300013FC6FF01600F8BD57F82500FBF70CFC25
:10F44000F0E70135AE42E7D8E76026720020F2E728
:10F450006FF01700EFE701220021FCF752B8F8B572
:10F460000446057A013D07D2E068FBF7F5FB20462C
:10F47000BDE8F840F2F72ABBAF007026E368D85920
:10F480003044103E00F0A8FA16F1100FF6D1E368F0
:10F49000D859FBF7E1FBE5E72DE9F74FDDF830A0A0
:10F4A00089461E460192074606F03EFE0546F2F7E3
:10F4B00063FB041E3FDBBAF1000F51462A7AB8BF46
:10F4C0000AF10701C9108A42884609DC0131284641
:10F4D000FFF792FF041E03DA2846F2F763FB2AE0E7
:10F4E000DAF100020AF00704E86802F0070258BFE8
:10F4F000544250F828104FEA880A01EB04118A6838
:10F50000FAB9C1F800902846EA68019B52F80A202F
:10F5100002EB04125360EA6852F80A2002EB04126C
:10F520009760EA6852F80A2002EB041204EBC80460
:10F53000D660F2F737FB204603B0BDE8F08FD8461F
:10F54000D7E701341031082CD9D108F1010B2A7A00
:10F5500000245A45F3DC08F102012846FFF74CFF6E
:10F56000041EB9DBEB680AF1040A019A4FEACB04E6
:10F5700053F80A30C3F80090EB6853F80A305A6029
:10F58000EB6853F80A309F60EB6853F80A30DE608E
:10F59000A2E72DE9F04106460F46F2F7EDFA041E08
:10F5A00002DA2046BDE8F081337ADBB10025F3684A
:10F5B0001B6803EB0508D8F8082082B15B595B058E
:10F5C0000DD401213846FFF717FF041E0ADBFB6844
:10F5D00040461968294400F015FA041E02DB103574
:10F5E000302DE4D13046F2F7DDFADAE7F8B5002342
:10F5F00005460F460B6006F097FD0646F0B1002D5C
:10F600001FDB037AB5EBC30F1BDAF2F7B5FA041E62
:10F6100012DBF368EA1005F00705304653F8223094
:10F6200003EB05153D60AB68002B04BF00256FF0B0
:10F6300008043D60F2F7B6FA2046F8BD6FF00A0400
:10F64000FAE76FF00804F7E72DE9F04106460F46A8
:10F6500006F06AFD0546002E35DB037AB6EBC30FD4
:10F6600031DA002F2FDBF2F787FA041E0FDB2B7A3B
:10F670004FEAE708B7EBC30F0CDB08F1010128469E
:10F68000FFF7BAFE041E05DA2846F2F78BFA204689
:10F69000BDE8F081EB68F01007F0070106F00706FF
:10F6A00053F8282053F8200002EB011100EB06105C
:10F6B00000F0A8F90446284614EA240438BF3C4662
:10F6C000F2F770FAE3E76FF00804E0E710B5FFF730
:10F6D000BBFF041E05DA6442F1F764FF04604FF0DB
:10F6E000FF34204610BDF0B585B0044606F01CFD81
:10F6F0000546F2F741FA002814DB002C0DDB2B7ACB
:10F70000B4EBC30F09DAE210EB6804F0070453F816
:10F71000223003EB04139A6832B92846F2F742FA12
:10F720006FF0080005B0F0BD1A466E4603F11007F1
:10F730001068083252F8041C3446BA4203C4264604
:10F74000F6D1102200211846F1F7B5FE2846F2F74F
:10F7500029FA684600F040F9E4E710B5FFF7C3FF67
:10F76000041E05DA6442F1F71DFF04604FF0FF3418
:10F77000204610BD00F05AB838B50F4C06F060FFB7
:10F780000546A368984204D1A38900200133A381D0
:10F7900038BD2046F2F7F8F9002807DAF1F702FF42
:10F7A00000680428F5D08C28F3D040420028EFD11F
:10F7B0000123A560A381EBE7A804002408B506F0A7
:10F7C0003FFF0A488389012B0CD1002383814FF02E
:10F7D000FF338360F2F734FA002805DABDE8084009
:10F7E000F1F7E0BE013B838108BD00BFA8040024FF
:10F7F00010B503460446184613F8012B2AB9001B1E
:10F800001C30FBF741FA18B910BD2F2AF3D1F6E7E7
:10F8100000F11803013C14F8012F12B900221A70EC
:10F82000F2E72F2AFAD003F8012BF4E708B50348D2
:10F83000FFF7DEFF024B186008BD00BFE2E41608C8
:10F840003850002400232DE9F04116461360027859
:10F8500088B0002A45D08DF81C30CDE9010301A8FD
:10F86000CDE90333CDE9053300F04AF8002835DA55
:10F87000019FDDE90354384600F036F803788046EE
:10F880003846D3B1FFF7B4FF48B96FF00B040698C0
:10F8900008B1FBF7E1F9204608B0BDE8F0813DB1C1
:10F8A0006B68C0E900436860474604460025E2E70C
:10F8B000A368C0E90043A060F6E7FFF799FF0028BE
:10F8C000E3D035B16B68C0E9004368600024306064
:10F8D000DDE7A368C0E90043A060F7E76FF010041C
:10F8E000D5E76FF01504D6E70278034601300AB178
:10F8F0002F2AF9D11846013302782F2AFAD07047FF
:10F90000F8B5036804461B782F2B11D005462E4806
:10F9100006F0C8FA2D4A55F8143B002818BF0246D5
:10F920002B492846FBF7B4FE6369002B46D02360C1
:10F93000284B196823681A782F2A42D100252E46B1
:10F9400041B90A466FF001002261C4E90031C4E9FF
:10F950000265F8BD53B301F117005F1E10F801CF27
:10F9600017F8012FBCF1000F06D182B12F2A0ED05B
:10F970004A680E461146E3E722B12F2A02D0944589
:10F98000F6D3EBD900216FF001000A46DCE71846F8
:10F99000FFF7AAFF0346007858B1CA8902F00F02A8
:10F9A000032A08D08A680D460021E2E71A46194664
:10F9B000C8E71A46C8E71A460020C5E76FF00B00F3
:10F9C000C7E76FF01500C4E73A5016087ADA160850
:10F9D0008C3A16083850002470B5866805467EB10A
:10F9E00034691CB164680CB1A0470446304605F088
:10F9F0005DFF0023C5E90033C5E90233204670BD31
:10FA00003446FBE7F0B50D4685B00646002840D0E9
:10FA10008768002F3DD000293BD0884203D10024C5
:10FA2000204605B0F0BD384605F0F9FE041EF7DBB0
:10FA3000336800937368CDE90137002303933B6972
:10FA4000BBB1FA8902F00F02032A0BD1DB6983B143
:10FA5000694630469847002804460ADA384605F0D9
:10FA600025FFDDE7F26803921B6813B168469847EB
:10FA7000F1E7284604ACFFF7AFFF6B461A4608359E
:10FA800003CAA24245F8080C45F8041C1346F5D1F8
:10FA9000C5E76FF00804C3E7F0B5876885B0044692
:10FAA0000D461668002F55D03B69C3B940F20D339F
:10FAB0009D420DDCB5F5417F0EDBA5F54175092DA5
:10FAC0000AD8DFE805F02A090909090909162226DA
:10FAD00040F20F539D422CD06FF0180007E05B6995
:10FAE000002BE3D03246984710F1190FDED005B055
:10FAF000F0BD236836B1326822B143F040030020E4
:10FB00002360F4E723F04003F9E7236843F48063BC
:10FB1000F5E7236823F48063F1E7FB8903F00F0323
:10FB2000032BD9D03146384605B0BDE8F04005F08A
:10FB300099BE3B69002BCFD05B69002BCCD001AACA
:10FB400040F20C51204698470028D0DBBDF90C301C
:10FB50003380CCE76FF00800C9E70EB403B503AA01
:10FB600052F8041B0192FFF797FF02B05DF804EB17
:10FB700003B070470EB477B507AD01A955F8046B13
:10FB80000095FFF733FD041E06DB2A463146019837
:10FB9000FFF782FF041E05DA6442F1F703FD0460FB
:10FBA0004FF0FF34204603B0BDE8704003B070470B
:10FBB00070B5866804460B4615463EB136692EB1CF
:10FBC00036691EB1B04700280DDA70BD012D05D091
:10FBD000022D0AD025B16FF01500F6E762681344D4
:10FBE000002BF8DB63606068EFE76FF05700ECE72D
:10FBF00037B50C4601A91546FFF7F8FC002804DBD1
:10FC00002A4621460198FFF7D3FF03B030BD10B557
:10FC1000FFF7EEFF041E05DA6442F1F7C3FC04604F
:10FC20004FF0FF34204610BD70B50D4688B0064633
:10FC300007F0B3F9002325EA000501A80196069311
:10FC40008DF81C30CDE90233CDE9043305F0F7FD22
:10FC500000281FDB0298059900900B78002B38D004
:10FC6000C38903F00F03032B35D103699BB3DB6C0E
:10FC70009BB32A469847002804DA4442009805F0CE
:10FC800015FE0CE0009805F011FE0698F0B9002072
:10FC900008B070BDFFF770FD041E0CDA64420698D0
:10FCA00018B1FAF7D9FF00230693F1F77BFC046043
:10FCB0004FF0FF30ECE76A4629463046FFF7C2FDB9
:10FCC0000446FFF77BFD002CDFDAE7E7FAF7C4FF15
:10FCD000DDE71124D2E70624D0E75824CEE7C38914
:10FCE000024613F00F0014D013696BB1CA0701D597
:10FCF0009A6862B111F002000BD0DB68002B0CBFD8
:10FD00006FF00C00002070476FF0050070476FF037
:10FD10000C0070472DE9F04F8BB0054617468A4618
:10FD20000193002977D012F0060F4FF0000803A8C6
:10FD3000039114BF149B4FF4DB79CDF8208018BFDA
:10FD4000D3F800908DF82480CDE90488CDE90688A9
:10FD500005F075FD041E35DB049E4FF0840BF2891F
:10FD600002F00F022BFA02FB1BF0010B12D03046FF
:10FD700005F09CFD089818B1FAF76EFFCDF82080C9
:10FD80003A465146284600F093FD044620460BB003
:10FD9000BDE8F08F39463046FFF7A1FF041E0CDBAB
:10FDA0003B05C5E9007BC5E9026B11D507992846DB
:10FDB00000F088FC0028044612DA00233046AB60CD
:10FDC00005F074FD08980028E0D0FAF745FFDDE75C
:10FDD000F38903F00F03032B0ED133691C681CB9A0
:10FDE000089890B90024D1E7019B3A460799284624
:10FDF00029EA0303A047DDE7012B09D133691B681A
:10FE0000002BEDD028469847D4E7FAF725FFE9E71D
:10FE10006FF00504D1E76FF01504B7E770B504463D
:10FE200086B00D46164607F0B8F8214603462A4626
:10FE300002A80096FFF76EFF041E0CDB0023049857
:10FE40000093059BDDE90212FFF726FB041E02DA90
:10FE500002A8FFF7C1FD204606B070BD0CB41FB567
:10FE600006AB53F8042B039300930023FFF752FFD4
:10FE700005B05DF804EB02B070470EB403B503AAF9
:10FE800052F8041B0192FFF7C9FF02B05DF804EBC2
:10FE900003B070470EB417B505AA52F8041B0192BF
:10FEA000FFF7BCFF041E05DA6442F1F77BFB046038
:10FEB0004FF0FF34204603B0BDE8104003B0704758
:10FEC00010B403688468DB0707D55CB123694BB1C4
:10FED0009B683BB15DF8044B18476FF00C005DF870
:10FEE000044B70476FF00800F9E737B50C4601A9DD
:10FEF0001546FFF77BFB002804DB2A4621460198C4
:10FF0000FFF7DEFF03B030BD10B5FFF7EEFF041EB4
:10FF100005DA6442F1F746FB04604FF0FF342046F7
:10FF200010BDFFEC2DE9F04F8846A1B081460028B6
:10FF300000F040810378002B00F03C81002900F0A4
:10FF400039810B78002B00F0358100264FF0010A33
:10FF5000039003A808968DF824A0CDE90466CDE9A6
:10FF6000066605F06CFC041EC0F29380049DEB89CC
:10FF700003F00F03032B40F09E80079F3B78002B7C
:10FF800000F0998002962B695B6D002B7CD00AA84B
:10FF90008DF840A0CDE90A86CDE90C66CDE90E6664
:10FFA00005F04DFC041E4EDBDDF82C80454568D184
:10FFB0000E9C38462146FCF7F1FE2B699B6D002B09
:10FFC00050D0002853D0B146DFF8F4A1214638467E
:10FFD000FCF7E4FE002845D02B6911AA21462846EB
:10FFE0009B6D984700283DDB139B03F47043B3F5EA
:10FFF000804F31D13846FBF765F923780646DDF8A6
:020000040803EF
:1000000008B001934BB9BBF1000F04D05846FAF782
:1000100023FE019B02933446D8E70346224651460D
:1000200002A8CDF80890FBF733FBBBF1000F02D01C
:100030005846FAF711FE029E002EECD16FF00B0429
:10004000404605F033FC0F9808B1FAF705FE029818
:10005000E0B1FAF701FE19E02B699B6C13B1214660
:100060002846984721463846FCF798FE08B90024F0
:10007000E6E72B692246394628465B6D98470446D9
:10008000DEE76FF01104DBE76FF05704284605F058
:100090000DFC089818B1FAF7DFFD00230893002C37
:1000A00080F28B806442F1F77DFA04604FF0FF30FC
:1000B00021B0BDE8F08F00240126414F0A9411A819
:1000C0008DF85C60CDE91184CDE91344CDE9154488
:1000D00005F0B5FB002840DB12988542029009D15B
:1000E0000024284605F0E2FB169808B1FAF7B4FDA3
:1000F0000A98ADE7C38903F00F03032B04D16FF017
:10010000110405F0D3FBEFE703690BB18368F3B18A
:1001100005F0CCFB4846FBF7D5F8DDF828A00346F0
:10012000424639460AA80A94FBF7B2FABAF1000F20
:1001300002D05046FAF790FDDDF828801698B8F105
:10014000000F34D00028BAD0FAF786FDB7E7404652
:1001500005F0EFFB029805F0A9FBFFF70DFB041E6D
:10016000C2DB02AA40F2FF114046FFF76BFB0028FA
:100170001ADBAA684846029B9A60EA89DA812A69F2
:100180001A616A695A6105F0D4FB041E08DA14F199
:10019000100F05D0404605F0CCFBFFF70FFBA3E79F
:1001A0000024AC602C60F8E76FF01004F5E76FF006
:1001B0000B0499E76FF0150474E7002078E700BF9F
:1001C0008C3A160870B5002388B006460693019055
:1001D00001A8CDE90233CDE9043301238DF81C30A9
:1001E00005F02DFB041E0CDA6442069818B1FAF7EC
:1001F00033FD00230693F1F7D5F904604FF0FF308B
:100200002DE0029DEA892B6902F00F02032A0CD12E
:1002100063B11B6D43B3059928469847002818DA47
:100220004442284605F042FBDFE7FBB9AB68FBB967
:10023000FFF7A2FA041E01DA6442F2E7304605F045
:1002400078FB0446FFF7BAFA002C02DA14F1100F1B
:10025000F2D1284605F02AFB069810B9002008B014
:1002600070BDFAF7F9FCF9E75824DAE71424D8E767
:100270005A24D6E730B50C46054685B03C2200210D
:100280002046F1F718F92B69002B31D09B6813B188
:100290004FF49273A3602B69DB681BB1A36843F032
:1002A0009203A360EA89A36802F00F02032A03D134
:1002B00043F48043A36015E0022A16D143F4C043FF
:1002C000A3602B6973B11B6963B101A928469847E4
:1002D000002807DB9DF8043023B1BDF90C20029BF8
:1002E0005343A361002005B030BD43F40053E1E760
:1002F00044F22413DEE7F0B50E4689B0174698B3F2
:1003000091B303789BB30023019001A80693CDE934
:100310000233CDE9043301238DF81C3005F08FFA48
:10032000041E11DB029DEB8903F00F03032B12D196
:100330002B69B3B19B6DA3B1324605992846984706
:100340000446284605F0B2FA069808B1FAF784FC8C
:10035000204609B0F0BD3A4631462846FFF78AFFED
:10036000EEE76FF05704ECE76FF00D04F0E76FF085
:100370000104EDE710B50122FFF7BDFF041E05DA09
:100380006442F1F70FF904604FF0FF34204610BDCE
:1003900010B50022FFF7AFFF041E05DA6442F1F743
:1003A00001F904604FF0FF34204610BD70B5002302
:1003B00088B006460693019001A8CDE90233CDE945
:1003C000043301238DF81C3005F039FA041E2ADBB2
:1003D000029DEB8903F00F03032B12D12A6982B12E
:1003E000936C002B3ED0059928469847041E17DBD6
:1003F000284605F05BFA069888BB0024204608B022
:1004000070BDAA688ABB012B13D12B69DB69BBB114
:1004100028469847041E03DBFFF7AEF9041E12DAE4
:10042000284605F043FA06980028E7D0FAF714FCAE
:10043000E4E7022B02D12B699B69E8E7002BEBD0A4
:100440006FF00504ECE7304605F073FA0446FFF759
:10045000B5F9002CCCDA14F1100FE1D1C8E7FAF7A6
:10046000FBFBCAE76FF05704DAE76FF05904D7E7F0
:1004700010B5FFF79BFF041E06DA6442F1F792F80D
:1004800004604FF0FF3010BD0020FCE710B404689A
:10049000A40708D583685BB11B694BB1DB683BB12E
:1004A0005DF8044B18476FF00C005DF8044B704783
:1004B0006FF00800F9E737B515460C4659B101A9A8
:1004C000FFF794F8002804DB2A4621460198FFF73D
:1004D000DDFF03B030BD6FF01500FAE710B5FFF790
:1004E000EAFF041E05DA6442F1F75CF804604FF09D
:1004F000FF34204610BDB1F5417F08B5C36805D172
:1005000059681046FCF755FC002008BD6FF0180034
:10051000FBE770B5C56806460C462868002954D02C
:10052000292A52D9C38903F00F03032B0BD1036986
:100530000A4629465B6B9847002842DB73682A20ED
:100540000133736040E0A96800293CD029221831AA
:10055000601CFCF736FC00232370AB681A696AB193
:10056000DB8903F00F03013B062B07D8DFE803F01C
:100570001D041B1F2123190006232370AB689A68F2
:100580000AB91B690BB904232370FFF7F5F8AC68AF
:100590006368AB608BB9FFF711F9204605F086F967
:1005A000CCE70923E9E70423E7E70223E5E7032390
:1005B000E3E70523E1E70723DFE79A8901329A8120
:1005C000E9E7831C00D1002070BD6FF01500FBE748
:1005D00070B5C468D4E90056EB8903F00F03032B10
:1005E00010D12B691B6B43B90024284605F05EF936
:1005F0003046FAF731FB204670BD21462846984721
:100600000446F2E7A06808B105F050F92046FAF771
:1006100023FBE9E72DE9F04306468DB089461746EE
:10062000002A48D1D0F80C804468D8F80050EB89F3
:1006300003F00F03032B20D1A1420CDA2B699B6B33
:100640002BB96FF0850420460DB0BDE8F0833C4621
:10065000414628469847A14503DC002CF3DB746033
:10066000F1E72B6901AA414628465B6B98470028B1
:1006700001DB0134EFE70446EFE7A142BABFAD6802
:100680001446D8F80850FFF777F80DB1A1450FD1FF
:10069000D8F80870C8F8085015B1AB890133AB81A0
:1006A000FFF78CF8002FD8D0384605F0FFF8D4E7D4
:1006B00001346D68E9E7012A0CBF44686FF0150446
:1006C000C1E7FFECF7B5856806460F46EB8903F0F6
:1006D0000F03032B19D12B6923B3DC6A14B35B6BB3
:1006E00003B301AA2846A047041E0BDB019B1D6033
:1006F000019D3846FCF7AAFA68600D48C6E9020574
:1007000005F08DF8204603B0F0BD0C20FAF7BCFAD6
:10071000034650B1019000240560A868986005F078
:100720007EF8E5E76FF05704ECE76FF00B04E9E7BC
:10073000B8040024C3685968FFF7C4BF2DE9F34724
:10074000061E884614461F465FDB12B905F0D2FD2F
:100750000446022E1ADC4FF49873A46873435C338A
:100760001C4404F1280304F594726660A36163627B
:10077000A4F82881C4E907230C2384F82A31002F28
:1007800041D10025284602B0BDE8F08701A93046D6
:10079000FEF72CFF051E08DB019B9868A8B14146B7
:1007A000FFF79DFA30B16FF00C05002FEAD000235F
:1007B0003B60E7E74FF49870D4F80890FAF764FAD2
:1007C000044628B96FF00B05EFE76FF00105ECE781
:1007D00009F1540A5046F1F795F9051E03DA20464F
:1007E000FAF73AFAE1E7D9F8F0334BB11C6050461A
:1007F000C9F8F043F1F7D6F92046FCF748F8B0E71E
:10080000C9F8EC43F3E73C60BBE76FF00805CCE7C1
:100810002DE9F34107460E4690461D46FEF7ACFF14
:10082000041E12DB01AA41463846FFF70BF8041EEE
:1008300009DB019B0024DA8922F00F0242F0010259
:10084000C3E90465DA81FEF7B9FF204602B0BDE8CE
:10085000F08138B50546FEF78FFF041E05DB2846FC
:1008600005F067F80446FEF7A9FF204638BD2DE9DC
:10087000F34107460E4690461D46FEF77DFF041ED7
:1008800012DB01AA41463846FEF7DCFF041E09DBF5
:10089000019B0024DA8922F00F0242F00202C3E930
:1008A0000465DA81FEF78AFF204602B0BDE8F081D8
:1008B0002DE9F047074694B088461646264DDFF8E6
:1008C0009C90DFF89CA02846F1F756F900281ADB27
:1008D000D9F8004028460134C9F80040F1F762F920
:1008E00024F07F435246102101A8FAF7DEFE0122D0
:1008F00005A901A8FFF7FFFC0028E4DA01A8FCF72E
:10090000A5F9054628B96FF00B04204614B0BDE8E0
:10091000F08786F0020201464046C2F3400206F02C
:1009200073FC041E0ADB26F03C0229463846FFF71A
:1009300095FA041E284605DAFFF738FD2846FAF72F
:100940008BF9E2E7FFF732FD041EF7DB28460024AF
:10095000FAF782F9D9E700BFD40400243C50002400
:100960007150160870B50E468AB019460023154618
:100970000446009368B9484C216829B12846FCF721
:100980000DFA30BB656835BB6FF00E0420460AB027
:1009900070BD6A4604F0E2FF002818DA6946204676
:1009A00005F016F80028E6DB09E00834216831B1CB
:1009B0002846FCF7F3F90028F7D165685DB96FF0B8
:1009C000120400980028E1D004F070FFDEE7334CF9
:1009D000ECE70834D0E7FEF7CFFE041EF1DB00237E
:1009E00003A8039608938DF82430CDE90433CDE9AC
:1009F000063304F024FF002817DB0498C389019014
:100A00001B0704D1EB6BCBB96FF0150426E06FF038
:100A1000130404F04BFFFEF7D1FE08980028D0D055
:100A2000FAF71AF900230893CBE701AA40F2FF1165
:100A30003046FEF707FF041EE4DAECE7009810B139
:100A4000838901338381EB6B02AA0E999847041EB8
:100A50000BDA009B13B19A89013A9A81019804F04C
:100A600025FF304604F065FFD5E7019AD38915616B
:100A700023F00F0343F00303D381029B5361FEF77E
:100A80009DFE009808B104F011FF089808B90024F1
:100A90007CE7FAF7E1F8FAE7A8891708C889170888
:100AA00013B5049C0094FFF75DFF041E05DA644251
:100AB000F0F778FD04604FF0FF34204602B010BD1F
:100AC0002DE9F041002388B08846074600930028AE
:100AD0005BD08DF81C30CDE9010301A8CDE90333CB
:100AE000CDE9053304F0ABFE041E27DB029DEB8944
:100AF00003F00F03032B45D12B691B6C002B41D056
:100B0000FEF73AFE061E34DB2B69424669466869E9
:100B10001B6C9847041E29DB26D1EB8923F00F03B9
:100B2000EB81AB68C5E9044483B1AB89013BAB8180
:100B3000FEF744FE009808B104F0B8FE069808B12C
:100B4000FAF78AF8204608B0BDE8F081384604F08C
:100B5000F0FE0646FEF732FE16B116F1100F08D170
:100B6000284604F0A3FEE5E76FF00F042646FEF7E3
:100B700025FE284604F09AFE009808B104F096FE7F
:100B80003446DBE76FF01506F3E76FF00D04D9E7A5
:100B900010B5FFF795FF041E05DA6442F0F702FD79
:100BA00004604FF0FF34204610BD38B5C3681B7990
:100BB0001B0715D483685D69284601F00CFF041EED
:100BC00007DB284601F05DFF044628461CB101F012
:100BD00005FF204638BD6FF0570401F0FFFEF8E72F
:100BE0006FF01F04F5E7F8B514460D463C220021CE
:100BF00006462046F0F75FFCEA7A11072FD412F080
:100C0000010F14BF4FF492734FF4DB73D2064CBF45
:100C100043F4804343F40043A3602F8BE88A3946B2
:100C200001F00EFF6062698A8F4202D0002001F05D
:100C300007FFE061298AE88901F002FFE062EB69C1
:100C40000020A36196F84920316912FB01F212B22B
:100C50001344A286013B93FBF2F3A363F8BD6FF04C
:100C60000100FBE72DE9F0414569A4B00F4690462D
:100C7000284601F0B0FE061E71DB284601F001FF98
:100C80000446002835D13A460CA9284601F0A6F9B9
:100C9000044670BB9DF86530002B64D11AAE06ACDB
:100CA0000FCE0FC496E80300BDF868306A4684E8AA
:100CB0000300E96C1746194401F10B0301F11B0411
:100CC0001868083353F8041C1646A34203C632467C
:100CD000F6D1186842460CA9306028461B7933715A
:100CE00001F07CF9831C044608D0002808BF6FF08F
:100CF00010042846264601F071FE30E00CA9284673
:100D000001F030FB064688BB0CA9284601F007FD20
:100D1000041EEEDBBDF8682004ACEB6C13440B330F
:100D20003A46083303CAA24243F8080C43F8041CAD
:100D30001746F5D1106806A91860284612791A716D
:100D4000012385F8453001F0C9FB041ED1DB28469C
:100D500002F0F2F9041ECCDB284601F03FFE3046DB
:100D600024B0BDE8F0816FF01104C2E70446C0E78B
:100D700070B545690E46284601F02DFE041E0DDBB8
:100D8000284601F07EFE044628B901223146284655
:100D900001F02CFD0446284601F020FE204670BDDF
:100DA00070B545690E46284601F015FE041E0DDBA0
:100DB000284601F066FE044628B902463146284618
:100DC00001F014FD0446284601F008FE204670BDDF
:100DD00070B545690E46284601F0FDFD041E09DB8D
:100DE000284601F04EFE044630B14FF0FF3428464D
:100DF00001F0F4FD204670BD95F84730B168022B34
:100E000009D089B9F060E8692346C6E90403284699
:100E100001F0E4FDEEE7EB698B4205D1F360284673
:100E2000E96901F07AFEEFE72846F16001F075FE0E
:100E30000223EAE7F8B5836806460F465D6928464F
:100E400001F0C9FD041E1BDB284601F01AFE044612
:100E500098B9F6682846316901F096FE041E0CDB4D
:100E60002B692846E96C5A1E338903EA62133A4615
:100E700001EB4311FFF7B7FE0446284601F0AEFD33
:100E80002046F8BD2DE9F04F456999B00E46284639
:100E900001F0A1FD071EC0F29D80284601F0F1FD82
:100EA000044658B932466946284601F097F8831C33
:100EB000044608D0002808BF6FF0100428462746D3
:100EC00001F08CFD86E06946284601F04BFA0746A2
:100ED000002840F0908001462846D5F828A002F06E
:100EE00037F8B0F10008C0F28880B8F1010F40F384
:100EF00086804146284601F010FEB0F10009C0F29C
:100F00008180284601F016FE041ED7DBEE6C4FF000
:100F1000010B2A6939463046C5F82890F0F7CBFA1C
:100F200095F849305B4559D84FF02033C6F8013069
:100F3000C6F80530A6F809302E2333701023F3725B
:100F400001F04FFD06F1200283B283461146F38182
:100F5000F382030C33823383334653F8040B9342FA
:100F600041F8040BF9D12E234FEA18491FFA88F8EB
:100F7000514686F821302846A6F81490A6F81A8023
:100F8000149BEA69934208BF00231A0C7387B28648
:100F9000012685F8456001F0F7FD041E8EDB5B46F7
:100FA00010226946284601F0DBFB041E86DBBDF8F3
:100FB00038202846EB6C1344A3F81A80A3F8149049
:100FC00085F8456002F0B8F8041EFFF677AF2846B2
:100FD00001F004FD384619B0BDE8F08F012309EB9C
:100FE0000B023146284601F081FD041EFFF666AF74
:100FF0000BF1010B94E7044660E744465EE76FF0AF
:101000001B045BE74C4659E770B546690D46304610
:1010100001F0E1FC041E21DB304601F032FD041E2C
:1010200019DB1C220021281DF0F745FA44F6445331
:1010300005F1100130462B6096F849303269534370
:10104000AB6002F0EEF8041E05DBF36AEB602B697F
:101050006B6128236B60304601F0C0FC204670BDF8
:1010600070B50D461646044680B301F0B4FC002866
:101070002BDB636843B1F2071ED51A7942F00802F0
:101080001A711B68002BF8D126683EB133691BB179
:101090005B680BB13046984705B12E60E06C10B12B
:1010A000216921F183FE04F10800F0F70FFD2046CD
:1010B000F9F7D2FD002008E0204601F08FFC002E59
:1010C0000CBF6FF00F006FF0570070BD6FF0150090
:1010D000FBE7084608B5F9F7BFFD002008BD2DE97C
:1010E000F041466998B0182088461746F9F7CCFDBC
:1010F0000446002841D0304601F06DFC051E35DB6A
:10110000304601F0BEFC054668BB424669463046A3
:1011100000F064FF002825DB9DF835307BB1149B7F
:10112000A360159BE360169B2361179B63613046A8
:101130003C6001F053FC284618B0BDE8F081BDF8D2
:101140003820F36C1344DA7AD20613D59A8A3046E3
:10115000598B41EA0241C4E9021101F0DEFC02238D
:101160002061E3E70546304601F038FC2046F9F7F8
:1011700073FDE0E76FF01305F5E76FF00B05DAE7B5
:10118000F8B51746054618B96FF012052846F8BDA0
:101190000369002BF8D01B683BB95020F9F774FDA8
:1011A000044630B96FF00B05F0E798470028F4D0FB
:1011B000EAE700220646114646F8085B3046FAF791
:1011C000A0F90121204601F0F5FC054630B130467A
:1011D000F0F77CFC2046F9F73FFDD7E720463C605E
:1011E00001F0FCFBD2E72DE9F84345690E461746AE
:1011F000284601F0F0FB041E22DB284601F041FCEA
:101200000446D0B9804606F1080978703169A1B169
:10121000B8F1000F11D1284601F0B6FC002839DBE7
:101220002B695A1E736903EA6213EA6C590102EBD7
:101230004313525C3AB96FF00104284601F0CEFB2B
:101240002046BDE8F883E52ADB7A1CD0190703D5D0
:10125000520618D50F2B16D13A463146284601F0D2
:1012600078F980B92B694FF001085A1E736903EAB7
:101270006212EB6C03EB4213DB7A13F0100F14BF16
:10128000042308233B704946284601F093FD0028BB
:10129000BCD0D0E70446D0E7F8B5C6680F4633792E
:1012A0001A073DD483685D69284601F094FB041E4B
:1012B00023DB284601F0E5FB0446D8B973799B0788
:1012C00029D57369BB4215D01EDD3169284601F06E
:1012D0005BFC002822DB2B69E96C5A1E338903EA88
:1012E000621301EB431157B9284601F0B8FE0028FC
:1012F00014DB7761284601F071FB2046F8BD3A46C1
:10130000284601F06DFEF2E73A463146284601F0E4
:10131000B7FF0028ECE76FF00C04EBE70446E9E7C1
:101320006FF01F04E9E72DE9F041C6680F463379F5
:101330001B073BD48368D3F81480404601F04BFB75
:10134000051E30DB404601F09CFB054640BB2820D3
:10135000F9F78AFC044640B1D8F8100021F124FDC9
:10136000606228B92046F9F777FC6FF00B0517E0AB
:10137000257173796371B379A37133892381F3681C
:10138000E3603369236173696361B369A361F369DE
:10139000FC60C4E90735D8F804302360C8F804407D
:1013A000404601F01BFB2846BDE8F0816FF01F05A9
:1013B000F9E7F0B5C66889B033791A0759D483685C
:1013C0005D69284601F007FB041E4FDB284601F04B
:1013D00058FB0446002846D133795B0743D5314694
:1013E000284601F061FE041E3DDB3169284601F00C
:1013F000CBFB041E37DB2B69EC6C5A1E338903EAE6
:1014000062136A4604EB43141746234604F1200E88
:101410001868083353F8041C94467345ACE803007D
:101420006246F5D1E37A43F02003E3727369E36126
:10143000B3696383B6F91A30A38201F0D2FAE0826D
:10144000000C2022394620832046337923F0040300
:101450003371FBF782FC10B1012385F84530284633
:1014600001F06AFE0446284601F0B8FA204609B0A9
:10147000F0BD6FF01F04F9E72DE9F041D0E9023526
:101480000646D3F814802B7913F008041ED1FFF719
:1014900090FFD8F80420074652B1AA4204D12A6826
:1014A0002CB9C8F8042003E014461268F4E722605F
:1014B000686A18B1D8F8101021F178FC2846F9F7BD
:1014C000CBFB00233846F360BDE8F0810027EFE74F
:1014D0002DE9F843C5680E4680462B79190700F1BF
:1014E0009880012A07D0022A17D032B16FF0150474
:1014F0002046BDE8F88343681E44D8F808305F6989
:10150000D8F804303A6996FBF2F193FBF2F3994272
:1015100005D1C8F804600024EAE76B69ECE73846B7
:1015200001F059FA041EE3DB384601F0AAFA04463A
:1015300000285CD12946384601F0B6FD041E56DB72
:101540006B69B34204DA6A7912F0020F08BF1E46D3
:101550000023C8F8043097F84930AC69AB7184B9FE
:10156000002E06DC6B799A0745D4384601F036FA2E
:10157000D1E72146384601F0EBFC041E37DBAC61B5
:10158000F0D097F849903B6903FB09F9B145EC604D
:1015900019D86B79214638469B0710D501F0D8FC45
:1015A0000028044623DB0DD0FB6A83422ED9D8F8ED
:1015B0000430A6EB09064B44C8F80430E6E701F016
:1015C00099FBEDE74E46D8F80420294638463244C8
:1015D000C8F8042001F037FE3B69013B3342C1D01B
:1015E000EA692946384601F075FD041EBADA384624
:1015F00001F0F4F97CE7D8F804306A699342C1BF7E
:101600006B612B7943F004032B71AEE76FF01B0481
:10161000EDE76FF01F046BE72DE9F74FC46817463D
:101620008046894623791A0700F1CA8083685D697C
:10163000284601F0D0F9011E28DB284601F021FAE6
:101640000146002838D163799B0740F1B080002F14
:10165000C0F2B0806FF000436269DB1B9A4200F376
:10166000A980E369B3B12E694FF0000BD8F80430BC
:10167000013EDA461E402FBBD8F804302846626986
:101680009342C8BF636101F0A9F95146084603B00F
:10169000BDE8F08FA16939B9284601F059FCA06175
:1016A000E06095F84930A3712146D8F80420284617
:1016B00001F0C9FD011ED6DA2846019101F08EF92C
:1016C0000199E3E7A37993B9E168284601F040FC6A
:1016D000011EF1DB012970DDEB6A8B426DD9E160FF
:1016E000284695F84930A37101F017FAE0612B699B
:1016F000BB42B7FBF3F266D8002E66D1BBF1000FF8
:1017000035D1A37921462846934228BF1346019339
:1017100001F000FD019B4946E269284601F0E6F927
:10172000011E019B05DA11F10E0F4FF0010BC3D121
:10173000DDE7A279D21AA271E2691A44E2612A694C
:101740005A43237943F0040323719144D8F80430B9
:101750009244BF1A1344C8F804302E69013E1E405B
:1017600089E7D8F8043062693B4493422DD321467F
:10177000284601F099FC011E9EDBE36923622A6979
:101780004946606A921B304497422ABFA3793A4681
:1017900003F1FF33019221BFA371E3690133E361D8
:1017A000EFF71EFD2379019A43F00703CCE76FF0B2
:1017B0000C0181E76FF01A017EE76FF01B017BE7F8
:1017C0006FF01F0162E7002ECBD02146E269284668
:1017D00001F080FC011ED2DA6EE72DE9F74FC468F4
:1017E00016468046894623791A0700F1A18083684E
:1017F0005D69284601F0EFF8011E1EDB284601F066
:1018000040F9014618BB6379DB0740F18B80D8F8BB
:1018100004206769E369BF1AB74228BF374683B11E
:101820002E694FF0000BD8F80430013EDA461E4016
:101830009FB9284601F0D2F85146084603B0BDE8EA
:10184000F08F2146284601F0FEFC011EE8DA28460A
:10185000019101F0C3F80199EFE7A3798BB9E16831
:10186000284601F047FA012801465EDDEB6A834213
:101870005BD9E060284601F050F9E06195F8493005
:10188000A3712B69BB42B7FBF3F22FD876BBBBF138
:10189000000F2BD1A37921462846934228BF134637
:1018A000019301F037FC019B4946E269284601F0AB
:1018B00006F9011E019B05DA11F10E0F4FF0010B25
:1018C000C5D1DEE7A279D21AA271E2691A44E261B7
:1018D0002A695A43D8F8043091449244BF1A1344F9
:1018E000C8F804302E69013E1E40A1E72146E26996
:1018F000284601F0EFFB011EA9DB2A694846616A10
:10190000921B314497422ABFA3793A4603F1FF3331
:10191000019221BFA371E3690133E361EFF760FC3A
:10192000019AD7E76FF00C0191E76FF015018EE790
:101930006FF01F0181E72DE9F043836899B00746F6
:1019400088465D691646284601F045F8041E7DDB91
:10195000284601F096F80146002840F08780602272
:101960006846EFF7A8FD42466946284600F036FB78
:10197000044610BB9DF83530002B79D1BDF83830C6
:10198000EA6C02EB030999F80B30DC0670D406F020
:101990000C020C2A6FD0B0071ED5D9076ED406F002
:1019A0002203222B18D14946284601F058FB041E79
:1019B00012DA284601F012F848E0821CF9D17307C8
:1019C000F7D56946284600F000FF041EF1DBBDF89C
:1019D0003830EA6C02EB03092820F9F755F9804604
:1019E00040B1286921F1E0F9C8F8240028B940463F
:1019F000F9F732F96FF00B04DBE788F8056006F0C1
:101A00001206AB6A2846C8F81030179BA8F80830B1
:101A1000B9F81420B9F81A3043EA0243C8F818306C
:101A2000C8F80C3095F8493088F80630D9F81C30E1
:101A3000C8F81430C7F80C806B68C8F80030C5F8D7
:101A4000048000F0CBFF122E04D00024204619B0F1
:101A5000BDE8F0830022D8F814103846FFF738FDAF
:101A6000041EF2DA4046F9F7F7F8EFE70446A0E77C
:101A70006FF014049DE76FF010049AE76FF00C0408
:101A800097E7F0B5456999B00F461646284600F02D
:101A9000A2FF041E19DB284600F0F3FF044688B9B4
:101AA0003A466946284600F099FA002818DB9DF866
:101AB00035306BB13C2221463046EFF7FCFC44F256
:101AC000B613B360284600F089FF204619B0F0BD78
:101AD000BDF838303246E96C28461944FFF783F8E0
:101AE0000446EFE7034600F10B010020C20142EA81
:101AF000500213F8010B50FA82F29942D0B2F5D19C
:101B00007047F8B504460D4600EB42062F7807B142
:101B10000135204600F056FFC0B2B84205D117B1DA
:101B20000234A642F2D1012000E00020F8BD70B5D9
:101B300004460D4600EB42062046023400F042FF08
:101B400005F8010BA642F7D170BD2DE9F843814697
:101B50000C468F6D01F1290801F15006A16D484630
:101B600001F012F800280EDBD9F81030E56D013BCA
:101B700005EA6315D9F84C306D01ADB258195B5DBB
:101B80001BB96FF00100BDE8F883E52B12D0C37AD2
:101B90001B070FD40B224146FBF7DFF850B9D9F8E9
:101BA0002820636DE26325872364E76462646587A8
:101BB000A364E8E73146484601F0FCF80028CDD0A0
:101BC000DFE710B598B0044660226846EFF708FBDF
:101BD000159B694620461493139B16930023179375
:101BE000FFF7B3FF18B010BD38B5044600EB410550
:101BF000204602344FF6FF7100F0E8FEA542F7D10F
:101C000038BD70B504460D4600EB4206204602344E
:101C100015F8011B00F0DAFEA642F7D170BDFFEC0B
:101C20002DE9F04F0D2589B0074608460C46FBF715
:101C3000DCF8002604F1FF3AB0FBF5F5EDB205EB58
:101C4000450303EBC30303EBC303184410F0FF0B7E
:101C50001EBF0BF1010301355FFA83FB534618BF2A
:101C6000EDB25A78591C002A5DD1C4F101021A4420
:101C7000002E5DD0311B0136521A531E0A464FF01A
:101C8000000904F129014FF000084A4501914FF085
:101C9000203184F83490C4BF99461346C4F82D10FF
:101CA0004FF00602C4F829102163CABF31464946E5
:101CB000264616F8010B002844D03D283AD81F28A4
:101CC0000BD9A0F1200EDFF80CC35FFA8EFE2CFAC0
:101CD0000EFC1CF0010F18BF5F200292CDE903310A
:101CE000FBF708FB029A08F1010CA044062A88F8C9
:101CF0002900DDE903315FD1013B002B02DDBCF19E
:101D0000060F0ED17E22A4448CF82920312288F8B7
:101D10002B2001B3B9F1000F1DDD0E464FF0080C6A
:101D20000B22E046C5E72E2A08BF0E460B4698E771
:101D30003346A4E75D283DD07C283BD05B2808BF14
:101D40005F20CAE7062A06D1A0447E2388F82930FE
:101D5000312388F82A30636C3846A16C4FF00108B3
:101D6000A365638F61655B09E36500F0D6FEA36D33
:101D7000181A3B695A11E36D02FB0033E365019BBE
:101D800013F8012F7E2A20D121463846FFF719FF8C
:101D9000064610B3B11C6CD10198FFF7A3FEA16DEC
:101DA0000590384600F0F0FE061E65DA304609B0B0
:101DB000BDE8F08F5F2090E709F1FF39B9F1000F1E
:101DC000C9DDBCF10B0FACD1C5E708F10108B8F1D2
:101DD000070FD5D16FF01506E8E7238F1AF8012F0A
:101DE0001ABB08F12901A8F10200DFF8ECC1214477
:101DF00086421FDB08F1010908F12B0A214638460B
:101E0000FFF7DFFE06460028C4D1C1454FF030037E
:101E100023D004EB0A004A4610F8011D382914D8D3
:101E20002244013182F82910E8E703EB43139BB207
:101E30005340D3E7B200013643FA02F202F00F0238
